:020000040000FA
:100000000C9468070C9499070C9499070C94990721
:100010000C9499070C9499070C9499070C949907E0
:100020000C9499070C9499070C9499070C949907D0
:100030000C9499070C942F8A0C9499070C949907A7
:100040000C9499070C942A880C9499070C9499079E
:100050000C9499070C9499070C9499070C94568763
:100060000C9499070C94AD7F0C94837F0C949907A2
:100070000C9499070C9499070C9499070C94990780
:100080000C94FC870C9499070C9499070C9499078D
:100090000C9499070C9499070C9499070C94A68CCE
:1000A0000C9499070C9499070C94CE870C9499079B
:1000B0000C9499070C9499070C9499070C94A087B9
:1000C0000C9499070C9499070C9499070C94990730
:1000D0000C9499070C9499070C944D7F0C94237FF2
:1000E0000C9499070C94B6910C9485110C942119D9
:1000F0000C941D760C9410080C9484080C940874CD
:100100000C940F120C9466140C9477190C94687468
:100110000C942E130C94A0070C947D750C9456121D
:100120000C9473200C9470750C949E1E0C947108A2
:100130000C94C0070C94A2750C944D130C948F75FD
:100140000C940A760C94A7750C94CA110C946C75D7
:100150000C94CB150C94AA740C9481750C94CE2736
:100160000C94E0150C9477750C9426080C949575F6
:100170000C94D3130C945A740C9480080C94077448
:100180000C9477130C9417730C941E120C94CA08D9
:100190000C9447990C9409740C9437740C948775DB
:1001A0000C9461080C949B080C94F7740C94F1184F
:1001B0000C94AC170C9494080C94C50D0C946B7EA5
:1001C0000C94ED130C9424760C947C080C9470150C
:1001D0000C944F140C949E080C9462750C946F0848
:1001E0000C9468750C94A0110C9474080C94198CE0
:1001F0000C947B170C94816C0C9423170C940A7448
:100200000C9474750C94CF0D0C949D750C9441173F
:100210000C9499750C9425110C940E140C9446743E
:100220000C94FB750C9406740C944B080C94EB988E
:100230000C94E7080C944C190C9465080C94400835
:100240000C9492150C94A3750C948B750C94191541
:100250000C942A080C9451764E414E494E495459FB
:10026000494E46CDCCCC3D0AD7233C17B7D1387781
:10027000CC2B329595E6241FB14F0A000020410097
:1002800000C84200401C4620BCBE4CCA1B0E5AAEE1
:10029000C59D7400407A10F35A00A0724E180900F0
:1002A00010A5D4E80000E87648170000E40B5402DB
:1002B0000000CA9A3B000000E1F505000080969816
:1002C00000000040420F000000A086010000001066
:1002D0002700000000E803000000006400000000A8
:1002E000000A00000000000100000000002C76D889
:1002F00088DC674F0823DFC1DFAE59E1B1B796E56F
:10030000E3E453C63AE651997696E8E6C28426EBD2
:10031000898C9B62ED407C6FFCEFBC9C9F40F2BAE5
:10032000A56FA5F490055A2AF75C936B6CF9676D7D
:10033000C11BFCE0E40D47FEF520E6B500D0ED90D2
:100340002E0300943577050080841E080000204E9F
:100350000A000000C80C333333330F986E12831138
:1003600041EF8D2114893BE65516CFFEE6DB18D10F
:10037000844B381BF77C1D901DA4BBE424203284E1
:10038000725E228100C9F124ECA1E53D27436F6E26
:1003900074656E742D547970653A20746578742F85
:1003A00068746D6C0D0A0D0A3C68313E4550494336
:1003B000204641494C3C2F68313E00485454502F50
:1003C000312E302034303020426164205265717506
:1003D0006573740D0A004163636573732D436F6E1B
:1003E00074726F6C2D416C6C6F772D4F72696769F9
:1003F0006E3A202A0D0A436F6E74656E742D54791F
:1004000070653A20005365727665723A20576562CE
:100410006475696E6F2F312E370D0A0048545450A1
:100420002F312E3020323030204F4B0D0A00436FD9
:100430006E6E656374696F6E3A20636C6F73650DE1
:100440000A436F6E74656E742D547970653A20613D
:1004500070706C69636174696F6E2F782D77777730
:100460002D666F726D2D75726C656E636F64656459
:1004700000506F7374206661696C65640055706C20
:100480006F6164204661696C65643A2000234E6F99
:100490002073656E736F7220666F722074656D7065
:1004A00020262068756D696469747921004E6F207B
:1004B00053656E736F72210020666F722074656DD4
:1004C0007020262068756D69646974792100235352
:1004D000656E736F72204572726F72200053656E85
:1004E000736F72204572726F7221002357726F6EA4
:1004F000672073656E736F7220666F722074656D0E
:100500007020262068756D696469747921005772BE
:100510006F6E672053656E736F7221004320483DF4
:1005200000543D00202020202020202020202020BA
:1005300020202020002020202020202020202020DB
:1005400020202020200020202020202020202020CB
:1005500020202020202000202020202020202020BB
:1005600020202020202000202020202020202020AB
:100570002020202020200054696D657374616D7007
:100580002075706C6F6164206661696C65640053EE
:10059000657474696E6720636C6F636B2074696D3A
:1005A0006500236572726F72202D20004950206112
:1005B0006464726573733A2000416E676C65400035
:1005C000496E76616C696420534D20737465707355
:1005D0002070657220616E676C653D00534D20731D
:1005E000746570732070657220616E676C653D0084
:1005F0003C703E54696D653A20003C2F68333E0ADA
:10060000003C62723E4254206E616D653D003C626A
:10061000723E506174683D003C68333E5379737498
:10062000656D3A2056657273696F6E3D0050617258
:10063000616D657465727320726573657420646F93
:100640006E6521002F6F652F736D6C69676874701C
:100650006F2F73332F00616E676C6520646972655C
:100660006374696F6E3A200043757272656E742010
:10067000534D206973202300534D3A5461626C65D9
:100680002073746570732070657220616E676C658D
:100690003D00534D3A506F6C6172697A65722073F8
:1006A000746570732070657220616E676C653D00C3
:1006B0002344485450494E3D00234448543D0023B0
:1006C0006E65743D424C4500236E65743D57694626
:1006D0006900236E65743D42540023667470207572
:1006E0007365726E616D653A003A0023486F7374EA
:1006F0002073657276657220495020616E642050C7
:100700006F72743A002354696D6520736572766563
:10071000722049503A002352656C617920646576F5
:10072000696365733A002352656C61792073746163
:10073000747573206C6162656C733A200023526596
:100740006C6179207374617465733A002352656C2F
:1007500061792070696E733A00234E6F2E206F66A8
:1007600020636F6E74726F6C2072656C6179733D7B
:1007700000234E6F2E206F662072656C6179733D89
:1007800000234C6F67676572204E616D653A2000EB
:1007900046696E64696E6720576946692049500052
:1007A0004E45543D426C7565746F6F7468204C45BE
:1007B000004E45543D426C7565746F6F7468004E11
:1007C00045543D57694669005344206F70656E205B
:1007D0006661696C004E6577206461746120636FA7
:1007E0006C6C656374696F6E207374617274656498
:1007F0000043757272656E742073657474696E67F8
:10080000733A0053797374656D2072657365742053
:100810006174200023445320546865726D6F6D65C8
:100820007465722063616C696272617465642066CC
:100830006F72202300496E76616C696420616E6777
:100840006C6520666F722000207374657073207071
:10085000657220616E676C653D002073746570730E
:100860002070657220616E676C653D005461626C3A
:100870006520536574203000235475726E74616274
:100880006C6520536574203000506F6C6172697A1A
:1008900065722053657420300023506F6C6172695B
:1008A0007A6572205365742030005461626C652053
:1008B000536574203000235475726E7461626C65E8
:1008C00020536574203000506F6C6172697A6572D4
:1008D0002053657420300023506F6C6172697A6513
:1008E0007220536574203000576946692049503A98
:1008F00000234C6F67676572204E616D653A20007A
:100900004C4F474745520056455253494F4E0052AF
:1009100065626F6F74696E672E2E2E005245424FCE
:100920004F540053657276657220506F7274207553
:100930007064617465640053504F52543D004950D7
:100940002075706461746564005349503D00235400
:10095000696D652053657276657220495020757007
:10096000646174656400545349503D004352454CE2
:1009700041590044485450494E3D0074696D65200A
:10098000696E74657276616C3D0054494D455354EF
:10099000414D503D0054494D455354414D50002365
:1009A00077656273657276657220626567696E73DA
:1009B0000053657474696E67204950005365747400
:1009C000696E6720446576696365204950202E2E44
:1009D0002E00506F6C6172697A65722053657420C5
:1009E000300023506F6C6172697A657220536574B0
:1009F00020300054657374204C616D70732F466114
:100A00006E73006572726F72206F70656E696E67CB
:100A10002066696C653A20004C616D70204D6F74E2
:100A20006F72002354696D652020202020204461CE
:100A3000746520202020205365636F6E64732050FE
:100A40006F6C6172697A6572205461626C652054C2
:100A5000286F43292048282529202000696E6974C1
:100A60002E20646F6E652E00534420696E69742ECB
:100A7000206661696C65642100696E69742E206668
:100A800061696C656421002323204F452057656C04
:100A9000636F6D6520232300496E697469616C6919
:100AA0007A696E6720534420636172642E2E2E0093
:100AB00075706C6F616420627920465450206661C5
:100AC000696C6564210075706C6F616420627920C7
:100AD000465450204F4B210053797374656D207339
:100AE00074617274696E672E2E2E003C703E4C61EC
:100AF0006D7020616E64204D6F746F722044726956
:100B00007665727320537461747573EFBC9A3C2FD1
:100B1000703E003C21646F63747970652068746D69
:100B20006C3E3C68746D6C3E3C686561643E3C6D37
:100B300065746120636861727365743D22757466C3
:100B40002D38223E3C7469746C653E4F6E6C696E44
:100B500065206578706572696D656E74202D205012
:100B60006F6C6172697A6174696F6E206566666523
:100B7000637473206F66206C696768743C2F7469B6
:100B8000746C653E3C2F686561643E3C626F6479BD
:100B90003E3C68313E4F6E6C696E652065787065CD
:100BA00072696D656E74202D20506F6C6172697A68
:100BB0006174696F6E2065666665637473206F6625
:100BC000206C696768743C2F68313E003C68343E95
:100BD000436F707972696768742843293230323004
:100BE0002D323032322E50726F662E205945554EBE
:100BF0004720596175205975656E3C2F68343E3C1D
:100C00002F626F64793E3C2F68746D6C3E003C68C7
:100C1000313E43616E6E6F74206765742073656E3C
:100C2000736F722072656164696E6773213C2F680F
:100C3000313E007C3C3E5E2B3D3F2F5B5D3B2C2AD2
:100C4000225C00000020002300260029002C002F39
:100C50000032000001000003010601090100000A42
:100C60000B02090C0D0E0807030401000000000030
:100C70000000000000000000000000000000000074
:100C80000000000000000000001211100000000031
:100C90000000000000000000000000000000000054
:100CA00000000053797374656D207265737461720E
:100CB00074656421002053797374656D20726573C7
:100CC00074617274656421004E6574776F726B2075
:100CD0006D61696E7461696E6564206174200023C2
:100CE00023436F6D6D616E6440000000220025009B
:100CF00028002B002E003100340002010000050105
:100D000008010B0100002100240027002A002D000B
:100D10003000330001010000040107010A01010253
:100D200010202008081020401020408002010201FD
:100D300008040201010204081020408080402010B5
:100D4000080402018004020180402010080402010E
:100D50000804020101020408102040800102040876
:100D6000102040800505050507050808080802024F
:100D700002020A0A08080404040401010101010135
:100D800001010303030303030303040707070C0C18
:100D90000C0C0C0C0C0C02020202060606060606DF
:100DA00006060B0B0B0B0B0B0B0B417070656E6487
:100DB000206D6561732E200053696E676C65206D30
:100DC0006561732E200053617665206D65617375D2
:100DD000726520746F3A00202020202020202020DF
:100DE0002020202020202000000001000100101001
:100DF000020001000100B000000016000000280001
:100E000000001000000020000000010001000000B0
:100E100000000000000000000000000000000000D2
:100E200000000000000000000000FF000000FFFFC5
:100E30000000FFFF0000FFFF0000CFBF0000C7BFA2
:100E40000000C3BF0000C1BF0000C0BF0000000021
:100E50000000C0BF0000C1BF0000C3BF0000C7BF8B
:100E60000000CFBF0000FFFF0000FFFF00000000F8
:100E70000000000000000000000000000000000072
:100E80000000000000000000000000000000000062
:100E90000000000000000000000000000000000052
:100EA000000000000000000000000000000055737A
:100EB00065722D6167656E743A202A0D0A44697364
:100EC000616C6C6F773A202F0D0A00004799EB9800
:100ED00011241FBECFEFD1E2DEBFCDBF00E00CBFBB
:100EE00019E0A0E0B2E0EEECFAE601E00BBF02C0D0
:100EF00007900D92AE3CB107D9F725E1AEECB9E011
:100F000001C01D92AC3EB207E1F717E0C7E6D7E09B
:100F100000E006C021970109802FFE010E946EB2F9
:100F2000C636D10780E00807A9F70E94FF9C0C9401
:100F300055B50C9400008EBD0DB407FEFDCF08958D
:100F4000DC015996ED91FC913097B9F08389948931
:100F5000A589B6894285538564857585841B950B63
:100F6000A60BB70B811520E89207A105B10538F053
:100F70008FEF9FE7A0E0B0E0089590E080E0089553
:100F8000CF93DF931F92CDB7DEB76983DC01ED917C
:100F9000FC910280F381E02D41E050E0BE016F5FE3
:100FA0007F4F19950F90DF91CF910895FC0120811B
:100FB0002EBD9B012150310941F051810DB407FE36
:100FC000FDCF4EB55EBD4193F5CF61507109860FDF
:100FD000971F0DB407FEFDCF2EB5FC0120830895A9
:100FE000E091480CF091490C90818091470C8095DC
:100FF0008923808308958EBD00000DB407FEFDCFC8
:101000008EB5089590E020914A0C233339F40C9664
:10101000982F990F990F990F80E008954896F8CF6F
:10102000CF93DF931F92CDB7DEB76983DC01ED91DB
:10103000FC910280F381E02D41E050E0BE016F5F42
:101040007F4F19950F90DF91CF910895FC01818D0D
:10105000928D0895CF93DF931F92CDB7DEB769834A
:10106000DC01ED91FC910280F381E02D41E050E044
:10107000BE016F5F7F4F19950F90DF91CF9108955B
:10108000FC019485FB018485981303C081E09830AE
:1010900008F080E00895CF93DF931F92CDB7DEB7BD
:1010A0006983DC01ED91FC910280F381E02D41E048
:1010B00050E0BE016F5F7F4F19950F90DF91CF9188
:1010C0000895FC01768765870895DC01ED91FC9118
:1010D000068CF78DE02D199591E089270895862FCC
:1010E000089581E08627089521E0FC0184858830F9
:1010F00008F020E0822F0895FC01848595850895ED
:10110000FC0184899589089522E134E0FC01318352
:101110002083FB014089518962897389FC014283E4
:101120005383648375830895DC01ED91FC91048CF5
:10113000F58DE02D199490E080E00895FC01818DFB
:10114000928D009711F00C94588F089561E0FC0186
:1011500084810C94E37FCF93DF93EC018FEF8EBDFE
:101160002FEF8F819885AC014F5F5F4F58874F837A
:101170008130924028F40DB407FEFDCF2EBDF1CF93
:101180000DB407FEFDCFCE010E94A6081E82DF919E
:10119000CF910895CF93DF93EC01E98DFA8D3097CD
:1011A00049F481E090E09B838A8390E080E0DF91C6
:1011B000CF91089513821282898D9A8D0E94279073
:1011C000E98DFA8D22813381232B59F7F0CFCF920D
:1011D000DF92EF92FF920F931F93CF93DF93CDB7E0
:1011E000DEB7AF970FB6F894DEBF0FBECDBF7C0160
:1011F0006A0102E114E01A8309831C861B8688EECB
:1012000093E0A0E0B0E08D879E87AF87B88B8CE934
:1012100093E09A878987188F0F8B198E1A8E1B8EF1
:101220001C8E88E089A31BA70AA71CA61DA61EA6C4
:101230001FA68091190E90911A0EA0911B0EB091CD
:101240001C0E8EA39FA3A8A7B9A78B839C83AD83F5
:10125000BE8318861F82AE01465D5F4FCE010196A8
:101260000E94F68481309105B1F4D701ED91FC9193
:101270000488F589E02D1DA30CA38CA59DA5AEA522
:10128000BFA58EA39FA3A8A7B9A7A601BE016C5DA9
:101290007F4FC7011995AF960FB6F894DEBF0FBE0A
:1012A000CDBFDF91CF911F910F91FF90EF90DF9015
:1012B000CF9008959F92AF92BF92CF92DF92EF921C
:1012C000FF920F931F93CF93DF935C017B018B0100
:1012D000D0E0C0E0F80191908F016501CC0EDD1ED9
:1012E000C6010E94A6B0981621F0692DC6010E9481
:1012F000AEB02196C233F1E0DF0761F7C701DF919D
:10130000CF911F910F91FF90EF90DF90CF90BF9002
:10131000AF909F900895FF920F931F93CF93DF9309
:10132000F82ECAEADBE08E0161E0D80112968C91BA
:101330000E9400816091690BF80182810E94E37F25
:1013400064EF71E080E090E00E9456810E5F1F4FD5
:10135000FBE0003B1F0741F7FF2009F447C0609105
:101360006B0B8A810E94E37F68EE73E080E090E07F
:101370000E94568160916B0B8C810E94E37F68EE26
:1013800073E080E090E00E9456816091690B8A8151
:101390000E94E37F68EE73E080E090E00E94568157
:1013A00022968BE0CE3AD807D1F668EE73E080E063
:1013B00090E00E945681C1EDD2E00CEA1BE0E99179
:1013C000F991D8018C910E5F1F4FEE0FFF1FE75967
:1013D000F44F60810E94E37F68EC70E080E090E071
:1013E0000E945681B2E0C73DDB0749F7DF91CF91FC
:1013F0001F910F91FF90089581E08093EF028091FB
:10140000F002882341F088E08093DF1160E084EDF2
:1014100091E10C94EC8B08958091F0028823F9F00F
:101420008091EF028823D9F081E00E94308C8BE319
:101430009FE10197F1F760E080E00E94418C67E650
:1014400075E084ED91E10E94F37E61E080E00E940E
:10145000418C67E575E084ED91E10C94F37E08958D
:101460000F931F93CF93DF932091F002222309F46F
:101470005CC02091EF02222309F457C0EA018C01DD
:101480006F3F7F4FF1F461E080E00E94418CB80132
:1014900084ED91E10E94D17E66E475E084ED91E1F6
:1014A0000E94F37E61E0F80184810E94418CBE01BC
:1014B000DD0F880B990BDF91CF911F910F910C9449
:1014C00056810E942584AB01BC0180919B0A9091BA
:1014D0009C0AA0919D0AB0919E0A8C599F4FAF4FD4
:1014E000BF4F84179507A607B707F8F461E080E0BF
:1014F0000E94418CB80184ED91E10E94D17E65E3A8
:1015000075E084ED91E10E94F37E61E0F801848151
:101510000E94418C0E94258460939B0A70939C0AD0
:1015200080939D0A90939E0AC2CFDF91CF911F9125
:101530000F910895CF93DF93EC010E94588F882379
:1015400011F01D8281E0DF91CF9108953F924F927B
:101550005F926F927F928F929F92AF92BF92CF9243
:10156000DF92EF92FF920F931F93CF93DF93CDB74C
:10157000DEB72C970FB6F894DEBF0FBECDBF5C016F
:10158000DC015B968D909C905C9716964D905D90DB
:101590006D907C901997411451046104710409F411
:1015A00068C0BFEF4B1A5B0A6B0A7B0A312CF4014F
:1015B00081859285A385B4859C01AD012F5F3F4F46
:1015C0004F4F5F4F29873A874B875C8773016201D2
:1015D0001D821E821F821886F40181859285A38553
:1015E000B4852D813E814F815885281739074A07D8
:1015F0005B0708F056C089859A85AB85BC858C153C
:101600009D05AE05BF0550F482E0C82ED12CE12C1B
:10161000F12C92E0492E512C612C712C9E012F5FF0
:101620003F4FB701A601C4010E946C8E8823C9F107
:1016300089819A81AB81BC81892B8A2B8B2B09F103
:10164000260137019FEF491A590A690A790A2D8143
:101650003E814F8158852F5F3F4F4F4F5F4F2D8306
:101660003E834F8358873FEFC31AD30AE30AF30A36
:10167000B3CFF4014080518062807380332433946F
:1016800096CFC414D504E604F70409F70FEF1FEF53
:101690002FEF3FE0B701A601C4010E94CA8D81115E
:1016A00019C080E02C960FB6F894DEBF0FBECDBFF8
:1016B000DF91CF911F910F91FF90EF90DF90CF902E
:1016C000BF90AF909F908F907F906F905F904F9062
:1016D0003F900895F50146815781608571854115D8
:1016E00051056105710539F097018601C4010E9419
:1016F000CA8D8823B1F2D5011696CD92DD92ED9276
:10170000FC921997332051F0D701C6010196A11D13
:10171000B11DF40180839183A283B383F50187898E
:10172000908DA18DB28D892B8A2B8B2B39F4C78A92
:10173000D08EE18EF28E84818068848381E0B2CF86
:101740008FEF0E949B078EB508958F929F92AF9264
:10175000BF92FF920F931F93CF93DF93EC01F62E6E
:1017600049015A018E81882319F0CE010E94AB08ED
:1017700060E08C810E94E37F8CE291E00E94DB8438
:101780008F2D80640E949B0708E110E0D501C40101
:10179000002E04C0B695A795979587950A94D2F721
:1017A0000E949B0708501109083F8FEF180771F737
:1017B00085E9FF2021F088E0F8120DC087E80E943B
:1017C0009B0710E00E94A00B8A8787FF06C01F3F7F
:1017D00021F01F5FF7CF8FEFF2CFDF91CF911F91F5
:1017E0000F91FF90BF90AF909F908F900895AF9210
:1017F000BF92CF92DF92EF92FF920F931F93CF93FE
:10180000DF93EC016901C801820F931F8130924080
:1018100050F58E81882379F088819981AA81BB81D6
:1018200084179507A607B70731F48F819885C816E6
:10183000D90608F042C0488359836A837B838B852D
:10184000833039F089E0440F551F661F771F8A9552
:10185000D1F79A01AB0161E1CE010E94A50B88236B
:1018600089F083E08D83CE010E94A60880E0DF919D
:10187000CF911F910F91FF90EF90DF90CF90BF908D
:10188000AF9008950E9425845B010E94A00B8A8777
:101890008F3F69F40E9425846A197B096D3271407B
:1018A000A0F38FE08D83CE010E94A608DCCF8E3F8F
:1018B000B1F418861F8281E08E838FEF8EBD2FEFEB
:1018C0008F8198858C159D0560F40DB407FEFDCFC2
:1018D0002EBD8F819885019698878F83F1CF8DE0FB
:1018E000E1CFC8010197F7012FEFAF014E195F0952
:1018F0004817590738F40DB407FEFDCF3EB53193B4
:101900002EBDF3CF0DB407FEFDCF2EB5E80EF91EA8
:10191000F70120838F819885080F191F18870F837F
:101920008985882319F00115124030F08E818823B3
:1019300019F0CE010E94AB0881E099CF0F931F935D
:10194000CF93DF93EC01890182E1411551056105D7
:10195000710599F08B85833039F089E0440F551F6C
:10196000661F771F8A95D1F79A01AB0168E1CE0116
:101970000E94A50B882319F084E08D8338C08EEF78
:101980008EBDF801C8019E5F0DB407FEFDCF20811A
:101990002EBD0DB407FEFDCF21812EBD3296E81776
:1019A000F90791F70DB407FEFDCF8FEF0E949B075B
:1019B0008FEF0E949B070E94A00B8A878F71853052
:1019C00089F488E592E00E94DB848823A9F020E076
:1019D00030E0A9016DE0CE010E94A50B882371F0D3
:1019E00084E1CBCF81E18D83CE010E94A608CE0198
:1019F0000E94A60880E00AC085E1BFCF0E94A00B2C
:101A00008111EECFCE010E94A60881E0DF91CF9137
:101A10001F910F910895FC01DB0112968D919C910D
:101A200013979383828384E793E091838083149652
:101A30008C911497848315968C91159785831696AF
:101A40004D915D916D917C91199746835783608785
:101A500071871A964D915D916D917C911D9742878A
:101A60005387648775871E964D915D916D917C912A
:101A7000519746875787608B718B52968C915297FE
:101A8000828B53964D915D916D917C915697438BCE
:101A9000548B658B768B57964D915D916D917C91B2
:101AA0005A97478B508F618F728F5B968D919C9167
:101AB000948F838F0895DC015996ED91FC913097B6
:101AC00021F081E09581911101C080E00895CF93CC
:101AD000DF93EC01898D9A8D009741F00E949A0A5C
:101AE000898D9A8D0E942DB31A8E198EDF91CF9118
:101AF0000895EF92FF920F931F93CF93DF93EC0122
:101B00007B018A011B821A8288EE93E0A0E0B0E09C
:101B10008C839D83AE83BF8384EF93E09983888316
:101B20008DE190E00E9491B29A8F898F009779F0B1
:101B30002DE1F701DC0101900D922A95E1F74CE0CF
:101B400050E0B801CE010C960E94FCB4188EDF91D3
:101B5000CF911F910F91FF90EF900895CF93DF9356
:101B60001F92CDB7DEB741E050E0BE016F5F7F4FFF
:101B70000E943392019731F4898190E00F90DF91B8
:101B8000CF9108958FEF9FEFF9CFFC01818D928D5A
:101B9000009711F00C94AE0D8FEF9FEF08950F9307
:101BA0001F93CF93DF93EC01898D9A8D10E000E0B5
:101BB000009799F00E94AE0D8C010F3F100769F05D
:101BC000898D9A8DFC0142855385648575854150C8
:101BD0005109610971090E94938FC801DF91CF916A
:101BE0001F910F910895E091480CF091490C80816C
:101BF0009091470C892B80830895AF92BF92CF922A
:101C0000DF92EF92FF920F931F93CF93DF9300D059
:101C10001F92CDB7DEB78C016B017A0180914A0C1F
:101C20008333E9F45B016801C40ED51EC016D106EA
:101C3000A9F10E94F0078FE00E94FB07812F0E940C
:101C4000FB07802F0E94FB070F5F1F4F80E00E9461
:101C5000FB07F50181935F010E94F30DE7CF843309
:101C600069F50E94F00719830A838F2D8F778B8384
:101C7000EC8264E070E0CE0101960E94D607A701D5
:101C800070E060E0C6010E94CCB4E114F10421F0E0
:101C9000B701C6010E94D6070E94F30DC7010F903D
:101CA0000F900F900F90DF91CF911F910F91FF90A8
:101CB000EF90DF90CF90BF90AF9008950E94F00713
:101CC0000F3F110509F030F419820A831B8263E08B
:101CD00070E0D1CF17FD0BC019820A8333E016954F
:101CE00007953A95E1F7007E08600B83F0CFC801B5
:101CF00026E0969587952A95E1F7807E19830A83D9
:101D00000115104C18F480618B83E1CF8861FCCF02
:101D1000CF93DF931F92CDB7DEB720914B0C30E00D
:101D2000322F2227260F371F90E0982F882741E077
:101D300050E0BE016F5F7F4F820F931F0E94FD0D29
:101D400089810F90DF91CF910895AF92BF92CF928A
:101D5000DF92EF92FF920F931F93CF93DF9300D008
:101D600000D01F921F92CDB7DEB78C017B016A01B4
:101D700080914A0C8333E1F45801A40EB51EA016DD
:101D8000B10609F46FC00E94F00780EF0E94FB07C4
:101D9000812F0E94FB07802F0E94FB070F5F1F4FC0
:101DA000F70181917F010E94FB070E94F30DE7CFAD
:101DB0005B01A40EB51E8433C1F40E94F0071983A1
:101DC0000A838D2D80688B83CC8264E070E0CE0125
:101DD00001960E94D607AE14BF0409F441C0F70172
:101DE00081917F010E94FB07F6CF0E94F0070F3F11
:101DF000110509F028F419820A8384E08B830CC052
:101E000017FD17C019820A8333E0169507953A9596
:101E1000E1F7007E0C600B8386E0C816D104A0F5C4
:101E2000F701DE011496EA15FB0599F081918D9377
:101E3000FACFC80126E0969587952A95E1F7807E2E
:101E400019830A830115104C10F48461D7CF8C617B
:101E5000D5CFB6016D5F7F4FCE0101960E94D607A8
:101E60000E94F30DC60128960FB6F894DEBF0FBE90
:101E7000CDBFDF91CF911F910F91FF90EF90DF9039
:101E8000CF90BF90AF90089563E070E0CE010196CF
:101E90000E94D607F70181917F010E94FB07AE14D3
:101EA000BF04C1F7DDCFCF93DF931F92CDB7DEB76D
:101EB00041E050E0BE016F5F7F4F90E080E00E9404
:101EC000FD0D89810F90DF91CF910895CF93DF931E
:101ED000C4E1D0E00E94530F882361F061E070E01C
:101EE00080E090E00E9456812197A1F780E0DF9189
:101EF000CF91089581E0FBCFCF93DF931F92CDB7B1
:101F0000DEB7898341E050E0BE016F5F7F4F90E014
:101F100080E00E94A50E0F90DF91CF91089563E0BD
:101F200070E00C94880EDA01E0914B0CF0E0FE2F8B
:101F3000EE27E60FF71F90E0982F8827A901BD0133
:101F40008E0F9F1F0C94A50ECF93DF931F921F92AD
:101F5000CDB7DEB779836A8322E030E0AE014F5F10
:101F60005F4F60E170E00E94930F0F900F90DF9140
:101F7000CF910895CF93DF931F921F92CDB7DEB715
:101F800079836A8322E030E0AE014F5F5F4F64E007
:101F900070E00E94930F0F900F90DF91CF91089502
:101FA000CF93DF931F92CDB7DEB720914B0C30E07B
:101FB000322F2227260F371F90E0982F882749833A
:101FC00041E050E0BE016F5F7F4F820F931F0E9480
:101FD000A50E0F90DF91CF910895CF93C82F462F74
:101FE00061E070E00E94D00F61E070E08C2F0E94F1
:101FF000880E8111F9CFCF910895DA01E0914B0C51
:10200000F0E0FE2FEE27E60FF71F90E0982F8827CD
:10201000A901BD018E0F9F1F0C94FD0D6F927F9241
:102020009F92AF92BF92CF92DF92EF92FF920F9367
:102030001F93CF93DF931F921F92CDB7DEB7982ED9
:102040008B013A01690122E030E0AE014F5F5F4F42
:1020500064E270E00E94FD0FE980FA80FE24EF2424
:10206000FE24E00EF11E9701377040914A0C092DB5
:1020700010E0C801433309F04CC00896982F882718
:10208000990F990F990F820F931F473309F446C098
:10209000A9014C0D5D1D4130584008F43FC060E07F
:1020A00078E05B01A21AB30AA501B3010E94A50E54
:1020B000A6014A195B09B3016A0D7B1D80914A0C88
:1020C000833349F5085F1F4F000F000F000F80E0BA
:1020D000902F0E94A50EEC0CFD1CF982EA8222E0F2
:1020E00030E0AE014F5F5F4F64E270E0892D0E94E7
:1020F000930F0F900F90DF91CF911F910F91FF9051
:10210000EF90DF90CF90BF90AF909F907F906F90B7
:1021100008954096B3CF005F1F4FD6CFA601B301FD
:10212000D8CFEF92FF921F93CF93DF931F921F920E
:10213000CDB7DEB7182F22E030E0AE014F5F5F4F22
:1021400060E270E00E94FD0FE980FA80FE24EF2437
:10215000FE2422E030E0AE014F5F5F4F60E270E0AE
:10216000812F0E94FD0F89819A81982789279827BE
:10217000E816F90689F487E0189FF0011124E3506E
:10218000F44FF582E482C7010F900F90DF91CF9159
:102190001F91FF90EF9008957C01DBCFFF920F938A
:1021A0001F93CF93DF931F921F92CDB7DEB7F82E08
:1021B00022E030E0AE014F5F5F4F66E270E00E94C8
:1021C000FD0F09811A8110270127102722E030E036
:1021D000AE014F5F5F4F66E270E08F2D0E94FD0FF2
:1021E00089819A819827892798270817190749F420
:1021F000C8010F900F90DF91CF911F910F91FF9029
:1022000008958C01E3CF44E050E0BC018FE090E002
:102210000C94A50E08951F93CF93DF93182F80E59C
:1022200091E00E948D77812F0E949110EC01812F07
:102230000E948F0F873121F08C3111F0D0E0C0E087
:10224000CE01DF91CF911F910895FC0184858830E4
:1022500010F40C940B1190E080E00895CF92DF927F
:10226000EF92FF921F93CF93DF93182F7B01EA0128
:102270004130584010F0C0E0D8E080E591E00E9485
:102280008D77812F0E9491106C01812F0E948F0FFA
:10229000873111F08C3121F5CC16DD0670F380E525
:1022A00091E00E948D779E01A70170E060E0812F90
:1022B0000E940E1060E270E0812F0E94ED0F62E03C
:1022C00070E0812F0E94880E84FD0DC0812F0E9436
:1022D0008F0F8823B9F080E591E00E948D77EFCFD2
:1022E000D0E0C0E0DCCF40E162E070E0812F0E94EE
:1022F000D00FCE01DF91CF911F91FF90EF90DF9033
:10230000CF900895D0E0C0E0F4CF0F931F93CF9308
:10231000DF938C01EA01FC018485883048F40E9437
:102320002E11892B39F481E090E0F80193838283A8
:10233000D0E0C0E0CE01DF91CF911F910F910895C1
:10234000CF92DF92EF92FF920F931F93CF93DF9381
:102350008B017A016C0129EBC20ED11CF601408180
:10236000EC012A96442349F050E0BC0167567F4FA8
:10237000CE010E948511F6011082A701B801CE019D
:10238000DF91CF911F910F91FF90EF90DF90CF9051
:102390000C948511CF93DF93EC01C754DF4FE88194
:1023A00021E02E0F2883E80FF92FF11DE756FF4F8C
:1023B0006083203249F4BC0167567F4F40E250E011
:1023C0000A960E948511188281E090E0DF91CF91FA
:1023D00008951F93CF93DF931F92CDB7DEB7182FC9
:1023E00080E591E00E948D77812F0E94020827E00E
:1023F000129FF0011124E350F44F22813381377092
:1024000041E050E0BE016F5F7F4F820F931F0E943B
:10241000FD0D89810F90DF91CF911F910895FC01EF
:10242000808D883040F4218D328D232B21F00E9445
:10243000E91190E008958FEF9FEF0895CF93DF9318
:10244000FC012485283028F08FEF9FEFDF91CF919A
:102450000895EC010190F081E02D0084F185E02DDC
:102460001995892B89F38C850E94E91190E0EECFB4
:102470001F93CF93DF93182F87E0189FE00111245B
:10248000C350D44F88819981009761F480E591E031
:102490000E948D77812F0E94CE102E81821B910980
:1024A00099838883DF91CF911F910895FC018485E2
:1024B000883010F40C94381290E080E008954F9228
:1024C0005F927F928F929F92AF92BF92CF92DF9254
:1024D000EF92FF920F931F93CF93DF931F921F9260
:1024E000CDB7DEB7782E6B014A01A82EB12C27E0BC
:1024F000829FC0011124FC01E350F44F7F01008151
:10250000118180E591E00E948D770815190554F43A
:10251000872D0E94CE10F70126818C01021B110924
:10252000118300830115110519F5872D0E948F0F66
:10253000843159F0882349F001E010E08C3111F426
:1025400010E000E0119501951109C8010F900F905E
:10255000DF91CF911F910F91FF90EF90DF90CF907F
:10256000BF90AF909F908F907F905F904F90089515
:10257000801691060CF4840187E08A9DF0018B9D02
:10258000F00D1124E350F44FE280F380C114D10424
:1025900051F12701F7E05F22872D0E940208840D88
:1025A000951D20914A0C273309F453C09801240D3E
:1025B000351D2130384008F44CC020E038E0490196
:1025C00084189508A401B6010E94FD0D2601480C4F
:1025D000591C6801C818D908872D0E940208A60155
:1025E000B2010E94FD0DE00EF11E87E08A9DF00110
:1025F0008B9DF00D1124E350F44FF382E282208191
:102600003181201B310B318320838681800F912FF4
:10261000911D8A3F910510F4232BF1F487E08A9DE8
:10262000F0018B9DF00D1124E350F44F1682F982D6
:10263000EA8222E030E0AE014F5F5F4F68E270E077
:10264000872D0E94930F60E470E0872D0E94ED0FAC
:102650007CCFA801B601C5CF868377CFCF93DF9318
:10266000FC01218D328D2115310529F48FEF9FEF6B
:10267000DF91CF910895EC01808D4217530708F048
:10268000A9010E945F121816190684F7298D3A8D48
:10269000281B390B3A8F298FEBCF0F931F93CF93C2
:1026A000DF931F92CDB7DEB7FC01218D328D232B36
:1026B00041F48FEF9FEF0F90DF91CF911F910F911A
:1026C00008958C0141E050E0BE016F5F7F4FFC0137
:1026D000808D0E945F12181619065CF7F801818D33
:1026E000928D0197928F818F898190E0E4CF0F9333
:1026F0001F93CF93DF9300D000D01F921F92CDB7CE
:10270000DEB78C01D80159964D915C915A974115CD
:10271000510551F0ED91FC91048CF58DE02D70E0A8
:1027200060E0C8011995EECFF801808D0E94381243
:10273000892BB1F148E050E0BE016F5F7F4FD801B7
:1027400058968C910E945F1218161906F4F4D8015D
:10275000509684E0FE01319601900D928A95E1F742
:102760008D8190E0982F88272E81820F911DF8018E
:10277000958B848B8F81282F30E0322F22278885FC
:10278000820F932F911D928F818F28960FB6F89408
:10279000DEBF0FBECDBFDF91CF911F910F91089586
:1027A00090E080E0F2CFCF93DF931F92CDB7DEB7FA
:1027B00041E050E0BE016F5F7F4FFC0184850E94C5
:1027C0005F121816190634F4898190E00F90DF919A
:1027D000CF9108958FEF9FEFF9CFFC01848588306A
:1027E00010F40C945F1290E080E00895CF93C82F0E
:1027F00080E591E00E948D7768E070E08C2FCF91AA
:102800000C94ED0FCF93C82F80E591E00E948D7757
:1028100060E170E08C2FCF910C94ED0FCF92DF929E
:10282000EF92FF920F931F93CF93DF9300D000D0CE
:10283000CDB7DEB78C016B017A01FC01808D883049
:1028400010F40E94021482E194E09A838983F601D5
:1028500082819381A481B5818B839C83AD83BE8368
:10286000B701CE0101960E940D7AF801808F883061
:10287000A0F4F586E486128E118E81E026960FB6BE
:10288000F894DEBF0FBECDBFDF91CF911F910F91A6
:10289000FF90EF90DF90CF90089580E0EFCFCF933F
:1028A000DF93EC01888D883020F40E94021488E0C8
:1028B000888FDF91CF910895CF93C82F80E591E065
:1028C0000E948D778C2FCF910C948F0FEF92FF92F7
:1028D0000F931F93CF93DF937C0180914A0CD4E038
:1028E000833309F0D8E005E31CE0C0E0F801219152
:1028F00031918F01F701848195812817390729F0DB
:10290000CF5FDC13F3CF80E006C08C2F0E945C14F5
:102910008431B1F781E0DF91CF911F910F91FF904A
:10292000EF9008959F92AF92BF92CF92DF92EF9275
:10293000FF920F931F93CF93DF93EC017B01809164
:102940004A0C811121C01B821A8288EE93E0A0E01C
:10295000B0E08C839D83AE83BF8386EC93E0998344
:10296000888388E08C8788EE93E09E878D87CE01F0
:10297000DF91CF911F910F91FF90EF90DF90CF905B
:10298000BF90AF909F90089534E0932E833311F061
:1029900028E0922E85E3C82E8CE0D82E10E098E037
:1029A000B92EA12CD6012D913D916D01F7018481A5
:1029B00095812817390791F4812F0E945C14082F04
:1029C000873111F08C3139F5812F0E943812892B13
:1029D00059F50C3119F4812F0E94F6131F5F9112E3
:1029E000E1CFA11008C0D701ED91FC910084F185E1
:1029F000E02DC70119951B821A8288EE93E0A0E0B2
:102A0000B0E08C839D83AE83BF8386EC93E0998393
:102A10008883BC86A8CF843149F08111DFCFF601CD
:102A2000329711821082DACFB12ED8CFAA24A39484
:102A3000D5CF8F929F92AF92BF92CF92DF92EF92BB
:102A4000FF920F931F93CF93DF93CDB7DEB72F97EE
:102A50000FB6F894DEBF0FBECDBF5C014B017A010B
:102A600080914A0C8823C9F104E0833309F008E01F
:102A7000B501CE0101960E94921485E3C82E8CE028
:102A8000D82E10E0F601219131916F01F50184817A
:102A900095812817390751F4812F0E945C148731E2
:102AA00029F4A701B401812F0E942E111F5F011389
:102AB000E9CFC7012F960FB6F894DEBF0FBECDBF8A
:102AC000DF91CF911F910F91FF90EF90DF90CF900A
:102AD000BF90AF909F908F900895F12CE12CE9CF9B
:102AE000CF93DF93EC018C858830D0F40E945C1486
:102AF000843189F0882379F0883169F021E08C31C4
:102B000059F4E881F9810084F185E02DCE01199511
:102B100021E0892B09F420E0822FDF91CF910895E5
:102B200080E0FBCFCF92DF92EF92FF92CF93DF93C3
:102B3000EC018C85883068F40E94F6130E9425848D
:102B40006B017C018C850E945C14811109C088E0B6
:102B50008C87DF91CF91FF90EF90DF90CF90089519
:102B600061E070E080E090E00E9456810E94258440
:102B7000AB01BC014C195D096E097F098D859E85ED
:102B8000B0E0A0E0481759076A077B07D8F28C85A8
:102B90000E940214DCCFCF93DF93EC018C85883048
:102BA00060F40E945C14873111F08C3131F48C8513
:102BB0000E940B118115984088F3DF91CF91089501
:102BC000CF92DF92EF92FF920F931F93CF93DF93F9
:102BD000CDB7DEB7AF970FB6F894DEBF0FBECDBF4F
:102BE0008C016B017A0182E194E09A8389831B82D4
:102BF0001C821D821E821C861B8648EE53E060E00C
:102C000070E04D875E876F87788B2CE933E03A87D9
:102C10002987988F8F8B198E1A8E1B8E1C8E28E019
:102C200029A39BA78AA71CA61DA61EA61FA6D8017E
:102C30001C968C91883060F40E945C14882321F0EB
:102C4000F80184850E94F61388E0D8011C968C93C5
:102C50008091190E90911A0EA0911B0EB0911C0E2E
:102C60008EA39FA3A8A7B9A78B839C83AD83BE83A4
:102C700018861F82AE01465D5F4FB601CE010196F8
:102C80000E94F6840097C1F0D801ED91FC91068472
:102C9000F785E02D82E194E09DA38CA38CA59DA5F2
:102CA000AEA5BFA58EA39FA3A8A7B9A7A701BE01E4
:102CB0006C5D7F4FC8011995AF960FB6F894DEBFD3
:102CC0000FBECDBFDF91CF911F910F91FF90EF907D
:102CD000DF90CF9008958F929F92AF92BF92CF9244
:102CE000DF92EF92FF920F931F93CF93DF9300D069
:102CF00000D000D01F92CDB7DEB790914A0C911151
:102D000015C018E0812F2A960FB6F894DEBF0FBECB
:102D1000CDBFDF91CF911F910F91FF90EF90DF908A
:102D2000CF90BF90AF909F908F90089528E0F22EA3
:102D3000933311F494E0F92E6B01082F80E591E0B4
:102D40000E948D779E012F5F3F4F5901490110E08E
:102D5000812F0E948F0FF40181934F018823C1F0CE
:102D60001F5FF112F5CFF12CF50191915F019D31BB
:102D700049F0983139F09A51923020F0F3941F11B4
:102D8000F3CFBFCF60E170E08F2D0E94ED0F1F2DBC
:102D9000E12EF12CF701EE0FFF1FEB5CF34F1182D8
:102DA000108283EE93E00197F1F7402F70E060E02E
:102DB000812F0E94D00F4FEF62E070E0812F0E94C0
:102DC000D00FB601CD2889F48091900290919102A4
:102DD00001968115F0EC9F0798F1909391028093F2
:102DE00090026091900270919102812F0E94BA0F1F
:102DF00061E070E0812F0E94ED0F27E02E9DC00161
:102E00002F9D900D11249C012350344F7901F9011D
:102E10001182108222E030E0AE01475F5F4F68E22E
:102E200070E0812F0E94FD0F89859A859827892758
:102E30009827F7019383828316821582148262CFCA
:102E400080E090ECCACF0F931F93CF93DF93EC01F8
:102E50008B01888D883010F40E940214B80182E042
:102E60000E946B16888F883050F41D870C871A8E4D
:102E7000198E81E0DF91CF911F910F91089580E02D
:102E8000F9CF9F92AF92BF92CF92DF92EF92FF92D3
:102E90000F931F93CF93DF938C015B01942EE52E4C
:102EA000FC01C688D788F08C80E591E00E948D7780
:102EB0008F2D0E949110C92DDE2D8C179D0708F4CF
:102EC000EC019E01A501B6018F2D0E940E10F801A4
:102ED000868997898C0F9D1F978B868BCE01DF91FA
:102EE000CF911F910F91FF90EF90DF90CF90BF9007
:102EF000AF909F900895CF93FC01C08D80E591E045
:102F00000E948D7760E270E08C2F0E94ED0F62E0EE
:102F100070E08C2F0E94880E84FD16C062E070E085
:102F20008C2F0E94880E83FF0AC048E162E070E0A7
:102F30008C2F0E94D00F80E090E0CF91089580E523
:102F400091E00E948D77E3CF40E162E070E08C2F4A
:102F50000E94D00F81E0F0CFFF920F931F93CF9389
:102F6000DF93EB01FC01178A168A2A81211109C01F
:102F70002B81211106C02C81211103C02D81222318
:102F800001F141155105E9F08A01FC01F08C80E561
:102F900091E00E948D77AE014E5F5F4F24E030E0FC
:102FA0006CE070E08F2D0E94930FB8018F2D0E946E
:102FB000A40F81E090E0DF91CF911F910F91FF90DE
:102FC000089580E0F7CF7F928F929F92AF92BF9249
:102FD000CF92DF92EF92FF920F931F93CF93DF93E5
:102FE000CDB7DEB7A6970FB6F894DEBF0FBECDBF44
:102FF0008C01762E942E852E20E2A22ECE010196F3
:103000007C01DC01EA2D1D92EA95E9F76801F3E401
:10301000CF0ED11C82E194E09AA389A38FEF8BA3FA
:103020008CA38DA38EA343E450E0BE016F5D7F4F60
:10303000C6010E94AC17019609F4BFC081E08983E4
:103040008A8386E0B82EBB821C82D80114966D91CB
:103050007D918D919C9117970E9476B26D837E83AE
:103060008F83988789869A8680E890E09C878B87F3
:103070004CE150E0B701C6010E944117FE013796AE
:103080008AE1DF011D928A95E9F74801B8E08B0ECD
:10309000911CF401D70101900D92BA94E1F740E13F
:1030A00050E0B701C6010E944117F7011192AA949E
:1030B000E9F796E0A92EB12C40E250E0B701C60135
:1030C0000E944117F1E0AF1AB108B1F783E6898396
:1030D00092E89A8393E59B838C8385E38D8381E0DB
:1030E0008E837F829DE3988797E099878A8786E021
:1030F000F401DE011B9601900D928A95E1F78CE0B8
:10310000898B8A8B64E174E0CE0143960E94E7B418
:10311000D8011B966C91CE0149960E94D278F80195
:103120006485CE014B960E94D278D8011D966C9191
:10313000CE014D960E94D2784EE150E0B701C60113
:103140000E944117B3E07B121EC082E3898384E0B2
:103150008A83F80196859B8397859C8390899D83BC
:1031600091899E8396E39F838887828D8987838D4B
:103170008A87848D8B87858D8C874CE050E0B701E2
:10318000C6010E94411787E3898386E08A8391E024
:103190009B8393E09C838D838FE08E838AE38F8370
:1031A0008BE388878FEF898749E050E0B701C6013C
:1031B0000E944117C6010E947B17A6960FB6F8948D
:1031C000DEBF0FBECDBFDF91CF911F910F91FF905A
:1031D000EF90DF90CF90BF90AF909F908F907F90B7
:1031E00008950F931F93CF938C01FC016481758127
:1031F00081E20E946B16C82F8830F8F480E591E0D8
:103200000E948D778C2F0E948F0F833131F08C2F8D
:10321000CF911F910F910C94F61362E070E08C2F08
:103220000E94ED0FF80184819581EC2FF0E0EE0F04
:10323000FF1FEB5CF34F91838083CF911F910F9120
:1032400008950F931F93CF93DF931F921F92CDB7D3
:10325000DEB7FC0124852830E0F48C0180E591E0A4
:103260000E948D7722E030E0AE014F5F5F4F60E15A
:1032700070E0F80184850E94FD0F89819A8198276A
:10328000892798270F900F90DF91CF911F910F9171
:10329000089590E080E0F6CF0F931F93CF93DF93D4
:1032A0001F921F92CDB7DEB7FC0124852830E0F4D1
:1032B0008C0180E591E00E948D7722E030E0AE0144
:1032C0004F5F5F4F64E070E0F80184850E94FD0F5E
:1032D00089819A819827892798270F900F90DF91ED
:1032E000CF911F910F91089590E080E0F6CFCF929B
:1032F000DF92EF92FF921F93CF93DF93EC017B015C
:103300006A018C85883048F40E945C14882319F087
:103310008C850E94F61388E08C87F7018281938167
:10332000A481B5810097A105B10551F490E080E03A
:10333000DF91CF911F91FF90EF90DF90CF90089594
:103340008F3F9F4FAF4FBF4F89F370E060E081E246
:103350000E946B16182F8C87883040F780E591E02B
:103360000E948D77A7014E5F5F4F24E030E06CE054
:1033700070E0812F0E94930FB601812F0E94A40F4D
:1033800064E070E0812F0E94ED0F0E9425846B01A4
:103390007C018C850E945C14873111F18C3101F124
:1033A000882321F20E942584AB01BC014C195D09E0
:1033B0006E097F098D859E85B0E0A0E08417950792
:1033C000A607B70738F061E070E080E090E00E9467
:1033D0005681DFCF8C850E94021488E08C87A6CFAF
:1033E00081E090E0A5CFCF93DF93EC0182E194E000
:1033F000998388831A821B821C821D8280E591E05A
:103400000E948D77BE016E5F7F4F44E050E08FE0F9
:1034100090E00E94FD0DCE01DF91CF9108954F9273
:103420005F926F927F928F929F92AF92BF92CF9254
:10343000DF92EF92FF920F931F93CF93DF93EC01F4
:10344000181619061CF44C0104972CF0C1E0D0E0CA
:1034500063E0862E912C8E01000F111F7E01EE0C71
:10346000FF1CEE0CFF1C8C169D060CF4B3C09701DC
:103470002C5B3D4F5901F90180819181A281B3817B
:10348000970121523D4F6901181619061A061B06AD
:103490003CF50E947D88F6014080518062807380F7
:1034A0006419750986099709F50140805180628089
:1034B0007380461657066806790658F41082118202
:1034C000128213820E947D88F60160837183828359
:1034D000938321960E5F1F4FF4E0EF0EF11CC3CFD4
:1034E000980129523D4F3901F9018081918198015C
:1034F00021533D4F5901F9012081318182179307F2
:10350000C1F0880F991FFC01E759F44F6081F80161
:10351000E655F44F80810E94E37FF3018081918121
:10352000F501918380836CE271E080E090E00E947D
:103530005681F60180819181A281B3811816190606
:103540001A061B0634F60E947D88F601208131811F
:1035500042815381621B730B840B950BF701E1547D
:10356000FD4F20813181428153812617370748075B
:10357000590708F0AECFF601108211821282138231
:1035800098012C5A3D4F6901F90180819181F50123
:10359000208131818217930709F49BCF880F991FEF
:1035A000FC01E759F44F6081F801E655F44F808142
:1035B0000E94E37FF60180819181F50191838083F0
:1035C000F301918380836CE271E080E090E00E94DF
:1035D00056817FCFDF91CF911F910F91FF90EF9098
:1035E000DF90CF90BF90AF909F908F907F906F9023
:1035F0005F904F900895CF93DF93FC012481358134
:10360000232B69F0EC01BC0185E29DE00E94DF7E86
:10361000BE0188E89CE0DF91CF910C94DF7EDF91C2
:10362000CF910895CF93DF93FC0124813581232B23
:1036300069F0EC01BC0185E29DE00E94D17EBE01F3
:1036400088E89CE0DF91CF910C94D17EDF91CF91FF
:1036500008958F929F92AF92BF92CF92DF92EF9296
:10366000FF920F931F93CF93DF938C01862F0B3024
:10367000110509F09FC090915D11992309F0F8940C
:1036800062E10E948981EC0180915D11882309F03B
:103690007894209701F180E090ECA9E7B4EC809356
:1036A000501190935111A0935211B09353118093E4
:1036B000541190935511A0935611B0935711CE3FCA
:1036C0008FEFD80709F4A9C0CF3FDC0709F462C027
:1036D000CCEFDFEF30C1C0915811E09059116E2D41
:1036E00070E090E080E00E9489AF2DEC3CEC4CEC67
:1036F0005DE30E94E8AF4B015C016C2F70E090E04D
:1037000080E00E9489AF9B01AC01C501B4010E9419
:1037100030B1609350117093511180935211909376
:103720005311D0915A11F0905B116D2F6F7770E0AB
:1037300090E080E00E9489AF4B015C016F2D70E04A
:1037400090E080E00E9489AF2DEC3CEC4CEC5DE316
:103750000E94E8AF9B01AC01C501B4010E9430B1E9
:10376000D7FD26C060935411709355118093561164
:1037700090935711CE0DCD0FCF0D81E090E02091A9
:103780005C11C21302C090E080E0892B09F493C061
:10379000CFEFDFEFCE01DF91CF911F910F91FF901F
:1037A000EF90DF90CF90BF90AF909F908F90089553
:1037B0009058D8CFCFEFDFEF0631110509F0BBC02D
:1037C00090915D11992309F0F89461E00E9489813C
:1037D000EC0180915D11882309F07894209701F124
:1037E00080E090ECA9E7B4EC8093501190935111D4
:1037F000A0935211B093531180935411909355118B
:10380000A0935611B0935711CF3FDC0719F22097C0
:1038100009F451C0229609F05BCFCEEFDFEF8BC0E9
:10382000C0915911D091581160915811709159114E
:1038300076276727762790E080E00E9487AF2DECFF
:103840003CEC4CEC5DE30E94E8AF60935011709348
:1038500051118093521190935311E0905B11F090AD
:103860005A116F2D6F77762F6E2D90E080E00E94B9
:1038700087AF2DEC3CEC4CEC5DE30E94E8AFF7FC2D
:1038800018C0609354117093551180935611909302
:1038900057118C2F8D0F8E0D8F0DC1E0D0E09091C0
:1038A0005C11891302C0D0E0C0E0D195C195D10967
:1038B000ABCF9058E6CFC0905011D0905111E0900E
:1038C0005211F090531120E030E048EC52E4C7016F
:1038D000B6010E9444B2D0E0C0E0181614F4CBEF59
:1038E000DFEF20E030E0A901C701B6010E9482AFFE
:1038F00087FF02C0CAEFDFEFC0905411D09055117E
:10390000E0905611F090571120E030E048EC52EC76
:10391000C701B6010E9482AF87FF02C0C9EFDFEF87
:1039200020E030E040EF52E4C701B6010E9444B20B
:1039300018160CF483C00C30110509F02BCF81E070
:103940008093830C8CE58093850C1092840C1092EC
:10395000860C60E082EC9DE00E94517681E00E943E
:10396000FC8A0E9431816B017C0180917D0C811168
:1039700068C081E080937D0C80937C0C9FEF9093D6
:103980007B0C10927A0C94E09093790C8093580CF5
:103990008091580C886B8093580C8091570C813023
:1039A00009F028C11092570C0E9431816B017C01F3
:1039B0008091580C8093BB0080917F0C9091800C7B
:1039C000A091810CB091820C892B8A2B8B2BA1F0BA
:1039D0000E94318100917F0C1091800C2091810C0C
:1039E0003091820C6C197D098E099F090617170703
:1039F0002807390708F446C08091BC0083FDD8CF62
:103A000085EC8093BC000E9431816B017C01809128
:103A10007D0C813009F4F0C080917A0C853008F07B
:103A20000DC180917A0CA9E5BCE0E2EBFBE090E0EF
:103A3000981769F12D9121939F5FFACFC8EFDFEFBF
:103A40007ACF80917F0C9091800CA091810CB091E5
:103A5000820C892B8A2B8B2B09F487CF0E94318112
:103A600000917F0C1091800C2091810C3091820C80
:103A70006C197D098E099F09061717072807390752
:103A800008F073CF80917E0C0E94DB8A80E0109258
:103A9000460C8093450C082F10E0CEEFDFEF882313
:103AA00009F478CECDEFDFEF053011050CF472CEBE
:103AB000CEE8DAE082EC9DE00E940A7688872196C3
:103AC000CE018E589A4080179107A4F3C091960AB0
:103AD0000091970A602F70E090E080E00E9489AF2B
:103AE0002DEC3CEC4CEC5DE30E94E8AF6B017C01FB
:103AF0006C2F70E090E080E00E9489AF9B01AC01E8
:103B0000C701B6010E9430B16B017C01C0928E0AE0
:103B1000D0928F0AE092900AF092910AD091980A7E
:103B20001091990A6D2F6F7770E090E080E00E940D
:103B300089AF4B015C01612F70E090E080E00E9452
:103B400089AF2DEC3CEC4CEC5DE30E94E8AF9B01AF
:103B5000AC01C501B4010E9430B1D7FD71C06093C2
:103B6000920A7093930A8093940A9093950AC00FD7
:103B7000CD0FC10F80919A0AC8130ACE20E030E021
:103B800048EC52E4C701B6010E9444B2D0E0C0E064
:103B9000181614F4CBEFDFEF20E030E040EA50E4F9
:103BA000C701B6010E9482AF87FF02C0CAEFDFEFF4
:103BB000C090920AD090930AE090940AF090950AEF
:103BC00020E030E040EF51ECC701B6010E9482AF27
:103BD00087FF02C0C9EFDFEF20E030E040EF52E4A2
:103BE000C701B6010E9444B218160CF0D3CDC8EF3D
:103BF000DFEFD0CD85EE05CF80917F0C9091800CCA
:103C0000A091810CB091820C892B8A2B8B2B09F40B
:103C1000FECE0E94318100917F0C1091800C20918A
:103C2000810C3091820C6C197D098E099F09061751
:103C300017072807390708F0EACE24CF85E0F3CE2E
:103C400090588DCFCF93DF93FB0122813381DC012C
:103C500013963C932E931297448155816681778108
:103C600014964D935D936D937C9317974085518582
:103C70006285738518964D935D936D937C931B9726
:103C80001C96EF012C969C01275E3F4F49914D9366
:103C9000A217B307D9F7218D328DFC01328F218F06
:103CA000DF91CF9108950F931F93CF93DF938C01F2
:103CB000EB01FE0164912196662349F0D801ED9154
:103CC000FC910190F081E02DC8011995F2CFDF91B0
:103CD000CF911F910F910895EF92FF920F931F9331
:103CE000CF93DF93EC017B018A016CE174E00E94C9
:103CF000531E65E074E0CE010E94531E66ED73E032
:103D0000CE010E94531EB701CE010E94C97E67E713
:103D100079E0CE010E94C97E0115110521F0B8019C
:103D2000CE010E94C97E67E779E0CE01DF91CF9195
:103D30001F910F91FF90EF900C94C97ECF93DF936A
:103D4000EC016BEB73E00E94531E65E074E0CE0162
:103D50000E94531E6DE873E0CE01DF91CF910C9469
:103D6000531ECF93DF93EC01FB01248135810E9428
:103D7000C47DCE01DF91CF910895EF92FF920F9312
:103D80001F93CF93DF9300D000D0CDB7DEB78C0167
:103D90007B016DE174E00E94AF7D8AE0E816F104DA
:103DA0002CF462ED76E0C8010E948A7CB701CE0156
:103DB00001960E94FD7ABE016F5F7F4FC8010E948D
:103DC000947CCE0101960E94107DC80126960FB604
:103DD000F894DEBF0FBECDBFDF91CF911F910F9141
:103DE000FF90EF9008952F923F924F925F926F92C3
:103DF0007F928F929F92AF92BF92CF92DF92EF927B
:103E0000FF920F931F93CF93DF93CDB7DEB7C258C6
:103E1000D1090FB6F894DEBF0FBECDBF6C015B01B8
:103E200088EE482E83E0582E612C712C04EF13E0AD
:103E30009BE5892E912C8C0E9D1E8CE0880E911C8A
:103E40001B019FEF291A390AD6015996ED90FC9073
:103E5000F7018581823008F493C082859385A4851B
:103E6000B5858F719927AA27BB27892B8A2B8B2B86
:103E700009F086C040E250E0BE016F5F7F4FC7018E
:103E80000E943392803209F07BC08981882309F433
:103E900077C0853E79F38E3269F38C8583FDEACF56
:103EA00022961FAE1EAE229784E793E09FAF8EAF9F
:103EB00024961FAE2497BE016F5F7F4FE0E080E045
:103EC0004EE2DB019D91BD019032A1F0883049F4B2
:103ED00026E730E02C0F3D1F2E0F311DD9014C93EA
:103EE000EF5F26E730E02C0F3D1F2E0F311DD9016B
:103EF0009C93EF5F8F5F8B3021F786E790E08C0F0C
:103F00009D1F8E0F911DFC011082D60159966D9157
:103F10007C9121E0AE014A585F4FCE01CE960E94BF
:103F20003A93882369F1BE01625C7F4FCE0181968E
:103F30000E940B0DAE014A585F4FBE016F5D7F4F6F
:103F4000CE01855A9F4F0E94790DCE01855A9F4F11
:103F50000E945B0D882309F4ACC0F12CFA141B04F9
:103F60002CF569E0CE0101960E947B7DCE01019681
:103F70000E94121BCE0101960E94107DF394EECF99
:103F80006F961FAE1EAE6F97A3964CAE5DAE6EAE33
:103F90007FAEA3976D961FAF0EAF6D97E6961FAEDF
:103FA0001EAEE697A8961FAEA897CFCFB401CE015C
:103FB00001960E94AF7DCE0101960E94121BCE0198
:103FC00001960E94107DE696EEADFFADE697309724
:103FD00009F447C08581823008F443C068E674E084
:103FE000CE0101960E94AF7DCE0101960E94FB1A80
:103FF000CE0101960E94107D6F968EAD9FAD6F979A
:104000009C838B83A3968CAD9DADAEADBFADA397C6
:104010008D839E83AF83B887A7968CAD9DADAEADE3
:10402000BFADA79789879A87AB87BC871A83098317
:104030008DE0F401DE011D9601900D928A95E1F765
:10404000E6968EAD9FADE6979B8F8A8FB101CE012C
:1040500001960E94F31ECE01855A9F4F0E94670D64
:10406000F3CE6BE174E0CE0101960E94AF7DCE01EC
:1040700001960E94121BCE0101960E94107DE696C9
:10408000EEADFFADE69740E050E0BA01309721F089
:104090004389548965897689CE0101960E94297BDE
:1040A000CE0101960E94FB1ACE0101960E94107D5E
:1040B000D2CFCE57DF4F0FB6F894DEBF0FBECDBFC5
:1040C000DF91CF911F910F91FF90EF90DF90CF90F4
:1040D000BF90AF909F908F907F906F905F904F9028
:1040E0003F902F900895CF92DF92EF92FF920F931F
:1040F0001F93CF93DF93CDB7DEB7C455D1090FB669
:10410000F894DEBF0FBECDBF65965FAF4EAF65972B
:104110002091DB0B3091DC0B2F5F3F4F3093DC0B9A
:104120002093DB0B2091F80B2111C1C08B016C0196
:1041300081E08093F80B1092DC0B1092DB0B6DE1A9
:1041400074E0CE01895B9F4F0E94AF7D6DE174E00A
:10415000CE01835B9F4F0E94AF7D50E040E06EE157
:1041600074E0C6010E946C1E0130110509F08EC07A
:104170006DE174E088EE9FE00E94F37A6DE174E0F7
:1041800084EC9FE00E94F37A6596EEADFFAD6597F3
:104190008081882309F474C000E210E09E012F5F43
:1041A0003F4F40E250E0BE016F5D7F4FCE018D5A20
:1041B0009F4F0E94D477049739F3BE016F5D7F4F04
:1041C000CE018F5B9F4F0E94AF7DBE016F5B7F4F23
:1041D000CE01895B9F4F0E94D77CCE018F5B9F4FA2
:1041E0000E94107DBE016F5F7F4FCE018F5B9F4F9E
:1041F0000E94AF7DBE016F5B7F4FCE01835B9F4FFF
:104200000E94D77CCE018F5B9F4F0E94107D2D9620
:104210008EAD9FAD2D970297029730F467E374E05F
:1042200084EC9FE00E94F37ABE01695B7F4F88EEC9
:104230009FE00E94947C63968EAD9FAD6397892B1F
:1042400009F4A2CF63E476E0CE018F5B9F4F0E941A
:10425000AF7DBE01635B7F4FCE018F5B9F4F0E949E
:104260002B7C60E476E00E94157CBC0188EE9FE028
:104270000E94947CCE018F5B9F4F0E94107D84CF63
:1042800068EE7FE084EC9FE00E94947C1092F80B33
:10429000CE01835B9F4F0E94107DCE01895B9F4FB3
:1042A0000E94107D0FB6F894DEBF0FBECDBFCC5A72
:1042B000DF4F0FB6F894DEBF0FBECDBFDF91CF91B9
:1042C0001F910F91FF90EF90DF90CF9008950F9383
:1042D0001F93CF93DF9300D000D0CDB7DEB72091EE
:1042E0006D0B2223A9F08C0168EC77E0CE010196DA
:1042F0000E94AF7DB801CE0101960E942B7CBC01CB
:1043000085E29DE00E94DF7ECE0101960E94107D35
:1043100026960FB6F894DEBF0FBECDBFDF91CF91CA
:104320001F910F9108950F931F93CF93DF93CDB7F4
:10433000DEB72C970FB6F894DEBF0FBECDBF8C0151
:104340000E94278ABC01C8010E94BD1E0E941F8ACC
:10435000BC01CE0107960E94BD1E60E077E0CE0151
:1043600001960E94AF7DBE01695F7F4FCE0101962D
:104370000E942B7CBC01C8010E94947CCE01019656
:104380000E94107DCE0107960E94107D60E476E0C9
:10439000C8010E948A7C0E94178ABC01CE01019646
:1043A0000E94BD1EBE016F5F7F4FC8010E94947CBA
:1043B000CE0101960E94107D6EE374E0C8010E9458
:1043C0008A7C0E940F8ABC01CE0101960E94BD1E0C
:1043D000BE016F5F7F4FC8010E94947CCE010196A1
:1043E0000E94107D6EE374E0C8010E948A7C0E94E6
:1043F000058ABC01CE0101960E94BD1EBE016F5F01
:104400007F4FC8010E94947CCE0101960E94107DCE
:10441000C8012C960FB6F894DEBF0FBECDBFDF915A
:10442000CF911F910F9108950F931F93CF93DF9317
:10443000CDB7DEB72C970FB6F894DEBF0FBECDBF59
:104440008C010E94278ABC01C8010E94BD1E0E94E7
:104450001F8ABC01CE0107960E94BD1E60E077E076
:10446000CE0101960E94AF7DBE01695F7F4FCE01F4
:1044700001960E942B7CBC01C8010E94947CCE0155
:1044800001960E94107DCE0107960E94107D0E9429
:104490007D880E940C896091D20B70E0CE01079656
:1044A0000E94BD1E60E077E0CE0101960E94AF7DC4
:1044B000BE01695F7F4FCE0101960E942B7CBC013B
:1044C000C8010E94947CCE0101960E94107DCE010D
:1044D00007960E94107D60E476E0C8010E948A7C05
:1044E0000E94178ABC01CE0101960E94BD1EBE012A
:1044F0006F5F7F4FC8010E94947CCE0101960E949D
:10450000107D6EE374E0C8010E948A7C0E940F8ACD
:10451000BC01CE0101960E94BD1EBE016F5F7F4FA0
:10452000C8010E94947CCE0101960E94107D6EE32A
:1045300074E0C8010E948A7C0E94058ABC01CE01F9
:1045400001960E94BD1EBE016F5F7F4FC8010E9491
:10455000947CCE0101960E94107DC8012C960FB666
:10456000F894DEBF0FBECDBFDF91CF911F910F91A9
:104570000895CF92DF92EF92FF920F931F93CF9304
:10458000DF9300D000D0CDB7DEB77C01FB01848182
:1045900095818A01081B190B101611069CF0C701A2
:1045A0000E94947DC70126960FB6F894DEBF0FBE19
:1045B000CDBFDF91CF911F910F91FF90EF90DF90D2
:1045C000CF900895CE0101960E94A67DCC24C3947D
:1045D000D12C60E476E0CE0101960E948A7CFFEF48
:1045E000CF1ADF0A0C151D05A4F7BE016F5F7F4FC0
:1045F000C7010E94947DCE0101960E94107DD2CF0A
:10460000DF92EF92FF920F931F93CF93DF93CDB77B
:10461000DEB762970FB6F894DEBF0FBECDBF8C0138
:1046200010929F0A6DE174E0CE010D960E94AF7D5D
:10463000FF24F39485E29DE00E94687420919F0A14
:10464000181619067CF521112DC085E29DE00E9407
:1046500046748A3009F07EC089899A89892B09F4C9
:1046600081C0F0929F0A60E474E0CE0101960E943E
:10467000AF7DBE01635F7F4FCE0101960E942B7C10
:10468000BC01CE0107960E94A67DCE0107960E942E
:104690006721CE0107960E94107DCE0101960E94EF
:1046A000107D60C0F12CE12CDD24D394222309F489
:1046B00060C089899A89019709F045C06FED74E05F
:1046C000CE0107960E94AF7DBE01695F7F4FCE018C
:1046D0000D960E94FA7BF12C811115C060E574E003
:1046E000CE0101960E94AF7DBE016F5F7F4FCE016C
:1046F0000D960E94FA7BFF24F3948111F12CCE01D8
:1047000001960E94107DCE0107960E94107DFF2029
:10471000A1F050E040E0BE01635F7F4FCE01019603
:104720000E94B11EBE016F5F7F4F8BE89FE00E9429
:10473000D77CCE0101960E94107D64E170E080E09C
:1047400090E00E945681BE01635F7F4FC8010E94C6
:10475000947D8EC08D3009F47FCF682FCE010D96E9
:104760000E94687C6AE070E080E090E00E945681E0
:1047700061CF88E89CE00E9468741816190614F549
:1047800088E89CE00E9446748A30A9F08D3099F048
:1047900090919F0A91110FC0682FCE010D960E9433
:1047A000687C8FEFE81AF80A65E070E080E090E03E
:1047B0000E945681DECF89899A89892BA9F3D092EC
:1047C0009F0AF2CF64E170E080E090E00E945681A1
:1047D000EF2809F43FC089899A89892BD9F1809102
:1047E0006D0B882389F168EC77E0CE0101960E9479
:1047F000AF7DBE016F5F7F4FCE010D960E94FA7BA9
:10480000F82ECE0101960E94107DF1101DC069E4C2
:1048100074E0CE0101960E94AF7DCE0101960E9408
:10482000121BCE0101960E94107DBE01635F7F4F77
:10483000CE0101960E94A67DCE0101960E94FB1A30
:10484000CE0101960E94107D64E170E080E090E06E
:104850000E94568189899A8920919F0A21112BCF24
:10486000009709F028CF6DE174E0C8010E94AF7D88
:10487000CE010D960E94107DC80162960FB6F89485
:10488000DEBF0FBECDBFDF91CF911F910F91FF9083
:10489000EF90DF9008950F931F93CF93DF93CDB7E1
:1048A000DEB72C970FB6F894DEBF0FBECDBF2C89B4
:1048B0003D89FE017496AAEABBE090E080E0329662
:1048C0002817390734F0408151814D935D9301964B
:1048D000F6CFCE5BDE4F88819981C254D140281734
:1048E00039070CF01CC2DC01AA0FBB1FA655B44F40
:1048F000880F991FFC01E855F44F80819181019642
:104900008D939C938C8D9D8D90936A0B8093690BF6
:104910008E8D9F8D90936C0B80936B0BAD968FADAE
:10492000AD97BE0164597F4F8F3209F001C2CE01AD
:1049300007960E94AF7D62E574E0CE0101960E9469
:10494000AF7DBE01695F7F4FCE0101960E942B7C37
:10495000BC018CE791E10E94C07CCE0101960E94CF
:10496000107DCE0107960E94107D6CE771E1CE01AB
:1049700001960E94A67DCE0101960E94FB1ACE01EF
:1049800001960E94107D68E674E0CE0101960E94B7
:10499000AF7DBE016F5F7F4F8CE791E10E94DA7BB4
:1049A000182FCE0101960E94107D409180115091E8
:1049B0008111112309F4C3C1BA01625071098CE756
:1049C00091E10E94C97B682FCE0101960E947B7DF8
:1049D000BE016F5F7F4F8EE591E10E94D77CCE01D3
:1049E00001960E94107D6EE470E1CE0107960E9450
:1049F000AF7D6AE674E0CE0101960E94AF7DBE01F4
:104A0000695F7F4FCE0101960E942B7CBC0186E737
:104A100091E10E94C07CCE0101960E94107DCE01E2
:104A200007960E94107D24968FAD24971F928F9336
:104A300023968FAD23971F928F9322968FAD229747
:104A40001F928F9321968FAD21971F928F9380E7AE
:104A500094E09F938F938AE99BE09F938F930E94AA
:104A600025B5CE52DF4F88819981C25DD0409093A9
:104A70008D0280938C02BE016C527F4FCE01019655
:104A80000E94AF7DBE016F5F7F4F80E791E10E9482
:104A9000D77CCE0101960E94107DBE0161527F4FEE
:104AA000CE0101960E94AF7DBE016F5F7F4F8AE607
:104AB00091E10E94D77CCE0101960E94107D409129
:104AC0006E1150916F11425051096AE671E1CE01A9
:104AD00001960E94B11ECE0101960E94617B6C5925
:104AE00060939702CE0101960E94107DCC5EDE4F4E
:104AF000688179818A819B81C451D1400E9489AFAC
:104B00000FB6F894DEBF0FBECDBF9B01AC010E9473
:104B100049B2882389F08CE390E0A0E0B0E0CC5E5D
:104B2000DE4F88839983AA83BB83C451D140CD5E75
:104B3000DE4F1882C351D140CD5EDE4F8881C35114
:104B4000D140882399F0CC5EDE4F88819981AA817B
:104B5000BB81C451D14080936E0290936F02A093A9
:104B60007002B093710281E08093500CC85EDE4FFA
:104B7000688179818A819B81C851D1409B01AC01B8
:104B80000E9449B2882361F080E090E0A0E7B2E49F
:104B9000C85EDE4F88839983AA83BB83C851D14006
:104BA000C45EDE4F68817981CC51D140072E000C64
:104BB000880B990B0E9489AF9B01AC010E9449B2FE
:104BC000882341F082E090E0C45EDE4F99838883C1
:104BD000CC51D140CE5BDE4F68817981C254D14047
:104BE000072E000C880B990B0E9489AF9B01AC012A
:104BF0000E9449B2882341F083E090E0CE5BDE4F13
:104C000099838883C254D140C45CDE4F08811981E6
:104C1000CC53D140B801012E000C880B990B0E9497
:104C200089AF9B01AC010E9449B2811103C01016EB
:104C3000110644F080E590E0C45CDE4F99838883E0
:104C4000CC53D140C45CDE4F88819981CC53D14094
:104C500090933F0280933E0288E2FE01E551FF4FB0
:104C6000AEE6BBE001900D928A95E1F7CE5CDE4F97
:104C700088819981AA81BB81C253D1408093290246
:104C800090932A02A0932B02B0932C02CA5CDE4FB1
:104C900088819981AA81BB81C653D1408093250226
:104CA00090932602A0932702B0932802C65CDE4FA1
:104CB00088819981CA53D14090935D0280935C02B0
:104CC000CC5BDE4F68817981C454D140072E000C43
:104CD000880B990B0E9489AF9B01AC010E9449B2DD
:104CE000882341F088E390E0CC5BDE4F9983888392
:104CF000C454D140CC5BDE4F88819981C454D140EB
:104D000090938F0280938E022C960FB6F894DEBF9C
:104D10000FBECDBFDF91CF911F910F91089580916C
:104D2000AE0B9091AF0B9093B10B8093B00BEACD8B
:104D3000CE0107960E94AF7D67E574E0FECD41503D
:104D400051096CE771E1CE0101960E94B11EBE01CE
:104D50006F5F7F4F8EE591E10E94D77CCE01019677
:104D60000E94107D6CE771E1CE0101960E94A67D44
:104D700068E674E0CE0101960E94157CBC018CE7C8
:104D800091E10E94C07C2BCEDF92EF92FF920F93B5
:104D90001F93CF93DF93CDB7DEB762970FB6F8942A
:104DA000DEBF0FBECDBF2091F002222379F120910A
:104DB000EF02222359F17A018C016F3F7F4FA1F559
:104DC00060E080E00E94418CD12CB80184ED91E13B
:104DD0000E94D17E64E275E084ED91E10E94F37E51
:104DE000F801848160E08D0D0E94418C0E94258431
:104DF0006093530C7093540C8093550C9093560C05
:104E0000B701FF0C880B990B0E94568162960FB672
:104E1000F894DEBF0FBECDBFDF91CF911F910F91F0
:104E2000FF90EF90DF90089560E080E00E94418C59
:104E30000E94258428EE33E040E050E00E94CCB090
:104E4000CA01B90120E831E541E050E00E94EEB02E
:104E5000AB01BC0120E0CE0101960E944E7DBE0157
:104E60006F5F7F4FCE0107960E94A67D62EB78E0D0
:104E7000CE0107960E94157CBC01CE010D960E94C2
:104E8000A67DCE0107960E94107DCE0101960E945C
:104E9000107DBE01635F7F4F84ED91E10E94D17E62
:104EA000D98860E08D2D0E94418CCE010D960E9424
:104EB000107D8BCFCF93DF9300D000D0CDB7DEB77E
:104EC0000E940C0ACE0101960E9493214AE050E014
:104ED0006FEF7FEFCE0101960E94C426CE010196AE
:104EE0000E94107D61E080E00E94418CCE0101961D
:104EF0000E94F31964ED71E1CE0101960E946B7E70
:104F00006CE774E084ED91E10E94C97E0E942584E3
:104F10006093E50B7093E60B8093E70B9093E80B9F
:104F200026960FB6F894DEBF0FBECDBFDF91CF91AE
:104F300008950F931F93CF93DF9300D000D0CDB788
:104F4000DEB78C01CE0101960E9493214AE050E029
:104F50006FEF7FEFCE0101960E94C426CE0101962D
:104F60000E94107DB801CE0101960E94A67D4AE004
:104F700050E06FEF7FEFCE0101960E94300ACE0124
:104F800001960E94107D26960FB6F894DEBF0FBEE4
:104F9000CDBFDF91CF911F910F910895EF92FF92B6
:104FA0000F931F93CF93DF9300D01F92CDB7DEB73F
:104FB0008C017B01FB0184858830A8F082E194E0BC
:104FC000F801918380831282138214821582C801B2
:104FD0000F900F900F900F90DF91CF911F910F9135
:104FE000FF90EF90089580E591E00E948D7724E096
:104FF00030E0AE014F5F5F4F6CE070E0F7018485F9
:105000000E94FD0FBE016F5F7F4FC8010E94177F96
:10501000DECF3F924F925F926F927F928F929F92DC
:10502000AF92BF92CF92DF92EF92FF920F931F93B6
:10503000CF93DF93CDB7DEB7EA970FB6F894DEBF14
:105040000FBECDBF7C012A013B0169010E9425846E
:105050004B015C0187010D5B1F4FC8010E94771354
:10506000181619069CF00E942584681979098A0986
:105070009B09461657066806790608F466C162E37E
:1050800070E080E090E00E945681E7CF42E250E07D
:10509000BE016F5F7F4FC8010E942E13898182304D
:1050A000D1F0312C832DEA960FB6F894DEBF0FBEF7
:1050B000CDBFDF91CF911F910F91FF90EF90DF90C7
:1050C000CF90BF90AF909F908F907F906F905F90A8
:1050D0004F903F900895F801848995898334910514
:1050E00001F76D817E818F8198850E9476B24B0198
:1050F0005C01F60180829182A282B38246E050E098
:10510000B701685F7F4FCE014D960E94A4B4892BF2
:1051100041F6F70180819181A281B38188169906B9
:10512000AA06BB0608F4BDCF84819581A681B7810C
:1051300088159905AA05BB0508F4B3CF89899A8912
:10514000AB89BC8986879787A08BB18B4EEC50E0EA
:1051500070E060E0C8010E942E13312CC7018296D6
:1051600098AB8FA7F701B696FAABE9AB08969CAB64
:105170008BAB67019AE1C90ED11CBD96FEABEDABBE
:10518000C701429698AF8FABFD97FAAFE9AF4701E1
:10519000FEE18F0E911CF801818D928D1816190673
:1051A0000CF080CFC8010E944D138333910509F4A0
:1051B000B2C014F58130910509F464C044F4892B20
:1051C00051F3C8010E944D13AC01552775C08330BF
:1051D000910509F462C00697A1F7C8010E944D131A
:1051E000B82E44E050E0B401C8010E942E13EB2D0C
:1051F000E450FF0BAF0160C08A33910509F45FC032
:1052000084F585339105B1F1C697D9F6C8010E949E
:105210004D135C01B601CE0189960E94177F8BA5C4
:105220009CA5ADA5BEA5892B8A2B8B2BB1F0EDA932
:10523000FEA94080518062807380B601CE018396C2
:105240000E94177F8DA19EA1AFA1B8A5A501481608
:1052500059066A067B0609F0B8CF44E050E0B60173
:1052600018C08B33910509F440C08F3F910509F4B4
:1052700092CFA7CFC8010E944D13C8010E944D13C1
:10528000382E89CFC8010E944D1344E050E06FA929
:1052900078ADC8010E942E137ECFC8010E944D1325
:1052A000B82E44E050E069AD7AADC8010E942E13DB
:1052B0008B2D8450990BAC0170E060E0EACFC801FF
:1052C0000E944D1344E050E069A97AA9C8010E94E8
:1052D0002E13F70166A177A180A591A50E9476B251
:1052E00066A377A380A791A756CFC8010E944D134C
:1052F00044E050E06BA97CA9C8010E942E13F7017D
:1053000062A573A584A595A50E9476B262A773A72E
:1053100084A795A740CFC8010E944D1344E050E0F8
:105320006FA578A9C8010E942E13F70162A173A18D
:1053300084A195A10E9476B262A373A384A395A3CE
:1053400066A777A780AB91AB26CF33243A94AACE39
:105350002F923F924F925F926F927F928F929F9285
:10536000AF92BF92CF92DF92EF92FF920F931F9373
:10537000CF93DF9300D000D0CDB7DEB78C010E9471
:10538000EDA62FEC37E040E050E00E94EEB0DC01EB
:10539000CB010196A11DB11DF80184839583A683DD
:1053A000B78380839183A283B3835801F3E4AF0E64
:1053B000B11CC5010E944F1464E470E0C5010E9455
:1053C0002317882309F445C10E9425842B013C0141
:1053D000480182E4880E911C48EEC42E43E0D42E8E
:1053E000E12CF12C52E0252E1E821D82D4018C91DD
:1053F0008330B1F1811166C0F80184819581A68165
:10540000B7810196A11DB11D84839583A683B783BF
:105410000E9425846419750986099709A7019601D8
:105420000E94CCB0A90161E0C8010E94E31781E0AD
:10543000D4018C938D819E810197C1F20E942584B5
:105440006419750986099709D801D6962D913D9161
:105450004D915C91D997261737074807590720F6D1
:10546000C5010E944F14F80184819581A681B781FE
:105470000196A11DB11D84839583A683B7830E94E5
:105480002584F801FE9660837183828393838D81E6
:105490009E8126960FB6F894DEBF0FBECDBFDF917A
:1054A000CF911F910F91FF90EF90DF90CF90BF9021
:1054B000AF909F908F907F906F905F904F903F90B4
:1054C0002F9008958430F1F4F80184819581A681AC
:1054D000B7810196A11DB11D84839583A683B783EF
:1054E0000E9425846419750986099709A701960108
:1054F0000E94CCB0A90163E0C8010E94E317D40167
:105500002C9298CF813051F5F80142AD53AD64AD86
:1055100075AD9E012F5F3F4FC8010E940928382EAC
:10552000F2E08F1390C089819A81AB81BC81F80130
:1055300084839583A683B7830E94258464197509A3
:1055400086099709A70196010E94CCB0A90163E0E2
:10555000C8010E94E317D4013C926CCF823009F05D
:1055600069CFF80142AD53AD64AD75AD9E012F5FBB
:105570003F4FC8010E940928382EF5E08F135DC007
:10558000E3E0D401EC93F80182A193A1A4A1B5A119
:10559000892B8A2B8B2B41F484E893E0A0E0B0E0C8
:1055A00082A393A3A4A3B5A3F80186A197A1A0A564
:1055B000B1A5892B8A2B8B2B61F482A193A1A4A185
:1055C000B5A1B695A7959795879586A397A3A0A70C
:1055D000B1A7F80182A593A5A4A5B5A5892B8A2B0F
:1055E0008B2BA9F482A193A1A4A1B5A1AC01BD010B
:1055F00023E076956795579547952A95D1F7841BB3
:10560000950BA60BB70B82A793A7A4A7B5A7F80184
:1056100086A197A1A0A5B1A586A797A7A0ABB1AB7E
:1056200082A593A5A4A5B5A582AB93ABA4ABB5AB5E
:1056300081E090E09E838D83FDCE96E0891303C0C8
:10564000D4011C92F7CEBFEF3B12F4CEF4011082CE
:10565000F1CE1E821D821BCF8F929F92AF92BF927E
:10566000EF92FF920F931F93CF93DF9300D000D060
:10567000CDB7DEB700914C0C10914D0CF12CE12C04
:105680000115110509F4DAC00E9425844B015C0163
:1056900078012EE3E20EF11CF70180819181A28155
:1056A000B381A5019401281B390B4A0B5B0BCA017E
:1056B000B901683E33E0730781059105A0F128EE3A
:1056C00033E040E050E00E94CCB0861A970AA80A66
:1056D000B90AD7018D929D92AD92BC921397F801B1
:1056E00086A597A5A0A9B1A949015A01880C991CC2
:1056F000AA1CBB1C88159905AA05BB0508F0B0C0FB
:1057000016A617A610AA11AAF80182A993A9A4A9FE
:10571000B5A988159905AA05BB0508F0AAC012AA63
:1057200013AA14AA15AAF80186A597A5A0A9B1A93C
:10573000892B8A2B8B2B09F0A5C0EE5BFF4F808154
:10574000833009F09FC084E08083C8010E94A829AB
:1057500001967C01F80182A993A9A4A9B5A9892B76
:105760008A2B8B2BA1F4EE5BFF4F8081833011F0ED
:1057700081110DC01082F8013E9684E1DF011D9277
:105780008A95E9F7C8010E94A82903967C01B2E036
:10579000EB16F10429F0E4E0EE16F10409F04EC036
:1057A00080E591E00E948D7760914C0C70914D0CDA
:1057B000625F7F4FCE0101960E94177FCE01039654
:1057C0000E94031160914C0C70914D0C6A5E7F4FEA
:1057D000CE0101960E94177F44E050E0BE016D5F4C
:1057E0007F4F81E090E00E94A50E60914C0C70917B
:1057F0004D0C6E5E7F4FCE0101960E94177F44E0F4
:1058000050E0BE016D5F7F4F85E090E00E94A50EE5
:1058100060914C0C70914D0C625E7F4FCE010196F1
:105820000E94177F8B819C81AD81BE818093190E70
:1058300090931A0EA0931B0EB0931C0EC7012696D0
:105840000FB6F894DEBF0FBECDBFDF91CF911F9191
:105850000F91FF90EF90BF90AF909F908F90089521
:10586000821B930BA40BB50B86A797A7A0ABB1AB7C
:105870004BCF821B930BA40BB50B82AB93ABA4ABAA
:10588000B5AB51CFF12CE12C65CFEF92FF920F9386
:105890001F93CF93DF93CDB7DEB7E8970FB6F89499
:1058A000DEBF0FBECDBF6DE174E0CE0187960E94D2
:1058B000AF7D6DE174E0CE018D960E94AF7D82E0F8
:1058C000E82EF12C2496FFAEEEAE249786E0EBEFA7
:1058D000F2E0DE01D39601900D928A95E1F786E021
:1058E000FE01F396DE01AC5BBF4F01900D928A95ED
:1058F000E1F72C961FAE1EAE2C9701E010E02E961D
:105900001FAF0EAF2E9788E0E1E0F3E0DE0159967D
:1059100001900D928A95E1F788E0FE017996DE010B
:10592000A25BBF4F01900D928A95E1F788E1E9E013
:10593000F3E0DE01119601900D928A95E1F788E17E
:10594000FE013196DE01AA5ABF4F01900D928A9551
:10595000E1F78091210390912203A0912303B0915C
:105960002403E2968CAF9DAFAEAFBFAFE29760E885
:1059700074E0CE0187960E94F37A60E0CE018796AC
:105980000E94687C4BA55CA5BE016E587F4FCE017E
:1059900087960E94AC7864E476E0CE018D960E94F2
:1059A0009B7C66ED74E08EE591E10E94F37A60E005
:1059B000CE018D960E94687C49A95AA9BE016656FF
:1059C0007F4FCE018D960E94AC786DE174E0CE01E0
:1059D00087960E94F37A6DE174E0CE018D960E9465
:1059E000F37AC250DF4F19821882CE5FD040809187
:1059F0008C0290918D02C050DF4F99838883C050F4
:105A0000D14080E090E0A0E7B2E4CA5BDE4F88833B
:105A10009983AA83BB83C654D140C65BDE4FF9820B
:105A2000E882CA54D14080E090E0A0E2B2E4C45BD6
:105A3000DE4F88839983AA83BB83CC54D14080E016
:105A400090E0A4E3B2E4C05BDE4F88839983AA832D
:105A5000BB83C055D14084EB90E0CC5ADE4F998394
:105A60008883C455D14088E790E0CA5ADE4F9983B5
:105A70008883C655D1408CE291E0A0E0B0E0C85ADE
:105A8000DE4F88839983AA83BB83C855D140C45A0B
:105A9000DE4F19830883CC55D140C25ADE4FF982BC
:105AA000E882CE55D14060E080E791E10E94687CB9
:105AB00060E08AE691E10E94687C40917411509107
:105AC0007511BE016E5F7E4F80E791E10E94AC7858
:105AD00040916E1150916F11BE01635F7E4F8AE657
:105AE00091E10E94AC7888E2EEE6FBE0DE01A75E81
:105AF000BE4F01900D928A95E1F78CE390E0A0E013
:105B0000B0E0CE5BDE4F88839983AA83BB83C25407
:105B1000D140CF5BDE4F1882C154D14084EE98E370
:105B2000AEE8B2E4C05ADE4F88839983AA83BB8370
:105B3000C056D14084EE98E3AEE8B1E4CC59DE4FD4
:105B400088839983AA83BB83C456D140C859DE4F4A
:105B500019830883C856D14080E590E0C659DE4FCE
:105B600099838883CA56D14083E090E0C059DE4FC4
:105B700099838883C057D14088E390E0CE58DE4FA8
:105B800099838883C257D14084EF91E09093670254
:105B900080936602BE016E5B7F4F0E945A0964EFDC
:105BA00071E080E090E00E9456816DE276E0CE01E7
:105BB00081960E949D7DCE0181960E94FB1ACE01A6
:105BC00081960E94107DCE018D960E94107DCE019F
:105BD00087960E94107DE8960FB6F894DEBF0FBE40
:105BE000CDBFDF91CF911F910F91FF90EF9008955E
:105BF0009F92AF92BF92CF92DF92EF92FF920F935C
:105C00001F93CF93DF93CDB7DEB7C859D1090FB635
:105C1000F894DEBF0FBECDBF5C017B016A0166E771
:105C200070E1CE0189579F4F0E94AF7D68E674E016
:105C30008E010F5F1F4FC8010E94AF7DB801CE01DA
:105C400089579F4F0E94FA7B982EC8010E94107DB1
:105C5000911014C068E674E0C8010E94AF7DBE01D7
:105C600069577F4FC8010E942B7CBC01CE01895728
:105C70009F4F0E94C07CC8010E94107DB501CE01DB
:105C800083579F4F0E94AF7D68E874E0E114F104F0
:105C900071F066E974E021E0E216F10441F061EA96
:105CA00074E032E0E316F10411F069EA74E0CE0129
:105CB00089579F4F0E948A7C60E0CE0189579F4F91
:105CC0000E94687CB601C8010E94A67D6AE0C801F6
:105CD0000E947C7CBC01CE018D569F4F0E94A67D08
:105CE000C8010E94107DC557DF4F48815981CB58AC
:105CF000D040B801CE0189579F4F0E94AC78809167
:105D0000510C882399F161EB74E0CE018F579F4FBE
:105D10000E94AF7DCE018F579F4F0E94121BCE0174
:105D20008F579F4F0E94107DBE0169577F4FCE0154
:105D30008F579F4F0E94A67DCE018F579F4F0E9485
:105D4000121BCE018F579F4F0E94107DB801CE01CC
:105D50008F579F4F0E94AF7DCE018F579F4F0E945C
:105D6000121BCE018F579F4F0E94107DCC56DF4FE4
:105D70008881C459D0408F93CD56DF4F8881C35955
:105D8000D0408F93C257DF4F8881CE58D0408F9339
:105D9000C357DF4F8881CD58D0408F9381EC94E07A
:105DA0009F938F938EECE82E89E0F82EFF92EF926E
:105DB0000E9425B540913E0250913F026AE97BE086
:105DC0008DEF9FE00E94E0150FB6F894DEBF0FBE86
:105DD000CDBF019709F07CC01F930F9387EC94E02F
:105DE0009F938F9304ED1AE01F930F930E9425B5A4
:105DF000B8018DEF9FE00E94B57E8AE99BE09F93FA
:105E00008F9388ED94E09F938F931F930F930E943D
:105E100025B5B8018DEF9FE00E94B57E6EE274E07B
:105E20008DEF9FE00E94F37E67E779E08DEF9FE0C2
:105E30000E94107EF70101900020E9F7CF018F5CEE
:105E400099409F938F9381EE94E09F938F931F933C
:105E50000F930E9425B5B8018DEF9FE00E94B57E9B
:105E6000B7018DEF9FE00E94C97E62E370E080E0A1
:105E700090E00E9456818DEF9FE00E9492150FB630
:105E8000F894DEBF0FBECDBF11E0CE018D569F4FFF
:105E90000E94107DCE0183579F4F0E94107DCE013E
:105EA00089579F4F0E94107D812FC856DF4F0FB634
:105EB000F894DEBF0FBECDBFDF91CF911F910F9140
:105EC000FF90EF90DF90CF90BF90AF909F9008959C
:105ED00061E774E0CE018F579F4F0E949D7DCE01F8
:105EE0008F579F4F0E94FB1ACE018F579F4F0E94E2
:105EF000107D6DE774E0CE018F579F4F0E949D7D0E
:105F0000CE018F579F4F0E94121BCE018F579F4F7C
:105F10000E94107D6EEC79E0CE018F579F4F0E945A
:105F2000AF7DCE018F579F4F0E94FB1ACE018F5736
:105F30009F4F0E94107D10E0A8CFEF92FF920F9329
:105F40001F93CF93DF93CDB7DEB768970FB6F89462
:105F5000DEBF0FBECDBF81E08093F80B0E942C2BDB
:105F60008C0160ED77E080E090E00E9456818BE04C
:105F7000E82EF12C0D7F0130110571F481E0E81A53
:105F8000F10851F00E942C2B8C0160ED77E080E04D
:105F900090E00E945681EECF0E9414827C0168EE50
:105FA00073E080E090E00E9456810BE010E0EF2863
:105FB00099F40150110981F060ED77E080E090E004
:105FC0000E9456810E9414827C0168EE73E080E09A
:105FD00090E00E945681EBCF87EB9EE00E94F11883
:105FE0001092F80B0E945A276DE174E0CE010796DB
:105FF0000E94AF7D6CEA75E0CE010D960E949D7DFA
:10600000CE0143960E94F319888D1F928F938F893A
:106010001F928F938E891F928F938D891F928F93DA
:1060200080E794E09F938F9384ED9AE09F938F9302
:106030000E9425B564ED7AE0CE0101960E94AF7D05
:10604000BE016F5F7F4FCE0107960E94D77CCE01C5
:1060500001960E94107DBE01635F7F4FCE010196C5
:106060000E94A67DCE0101960E94121BCE010196D0
:106070000E94107DBE01695F7F4FCE0101960E9494
:10608000A67DCE0101960E94FB1ACE0101960E94C8
:10609000107DBE01695F7F4FCE0101960E94A67DF3
:1060A000AE014F5F5F4F63E070E080E092E00E94DE
:1060B000F82D182FCE0101960E94107D0FB6F8948E
:1060C000DEBF0FBECDBF11112BC062EA75E0CE015D
:1060D00001960E949D7DCE0101960E94121BCE0169
:1060E00001960E94107DBE01635F7F4FCE01019635
:1060F0000E94A67DCE0101960E94121BCE01019640
:106100000E94107D6AEC7FE0CE0101960E94A67D80
:10611000CE0101960E94FB1ACE0101960E94107DCD
:10612000CE010D960E94107DCE0107960E94107D33
:1061300068960FB6F894DEBF0FBECDBFDF91CF914A
:106140001F910F91FF90EF9008957F928F929F92F1
:10615000AF92BF92CF92DF92EF92FF920F931F9375
:10616000CF93DF93CDB7DEB762970FB6F894DEBF5B
:106170000FBECDBF6FE875E0CE0101960E949D7DF8
:10618000CE0101960E94FB1ACE0101960E94107D5D
:1061900004E010E030EAC32E3AE0D32E40E3E42ED0
:1061A00053EEB52E66E0A62E7CEE972EE1E3FE2E92
:1061B000FEE48F2EA4E37A2E68EB72E28DE99FE075
:1061C0000E942317F6018E2D11928A95E9F7B0925D
:1061D000A00AA092A20A9092A30AF092AC0A80921E
:1061E000AD0AF092AE0A7092AF0A60E472E0CE019E
:1061F00001960E94177F4BE750E0BE016F5F7F4F13
:106200008DE99FE00E94AC1740E350E060EA7AE03D
:106210008DE99FE00E9441178DE99FE00E947B1766
:1062200068EE73E080E090E00E9456818DE99FE087
:106230000E947713892B09F04FC00150110909F012
:106240007CC08091D00A9091D10AA091D20AB091DD
:10625000D30A892B8A2B8B2B09F089C06DE174E05E
:1062600088EE9FE00E94F37A68EE7FE0CE0101960F
:106270000E94A67DAE014F5F5F4F70E060E082E755
:1062800092E00E94F82D182FCE0101960E94107DF9
:1062900011110EC067E775E0CE0101960E949D7D49
:1062A000CE0101960E94FB1ACE0101960E94107D3C
:1062B00062960FB6F894DEBF0FBECDBFDF91CF91CF
:1062C0001F910F91FF90EF90DF90CF90BF90AF9014
:1062D0009F908F907F90089540E350E060EA7AE0CD
:1062E0008DE99FE00E942E136091C80A7091C90A3F
:1062F00076276727762790E080E0CB01772766270F
:106300000091CA0A1091CB0A10270127102730E00C
:1063100020E0602B712B822B932B7E508A4A93486E
:106320000E9458880E947D886093D00A7093D10A99
:106330008093D20A9093D30A84CF68EE73E080E012
:1063400090E00E9456814091D00A5091D10A60910C
:10635000D20A7091D30A2AE085E29DE00E941F7E56
:1063600067E779E085E29DE00E94107E25CF68EE28
:1063700073E080E090E00E9456810E947D886093E7
:10638000EF0B7093F00B8093F10B9093F20B0E9444
:106390007D886093E90B7093EA0B8093EB0B9093ED
:1063A000EC0BCE0101960E941422CE0101960E94B0
:1063B000FB1ACE0101960E94107D0E94178ABC0133
:1063C000CE0107960E94BD1E6EE374E0CE010796D3
:1063D0000E948A7C0E940F8ABC01CE0101960E9415
:1063E000BD1EBE016F5F7F4FCE0107960E94947C59
:1063F000CE0101960E94107D6EE374E0CE010796F7
:106400000E948A7C0E94058ABC01CE0101960E94EE
:10641000BD1EBE016F5F7F4FCE0107960E94947C28
:10642000CE0101960E94107D66EF74E0CE010196C8
:106430000E94AF7DBE01695F7F4FCE0101960E9431
:106440002B7CBC01CE010D960E94A67D4AE050E057
:106450006FEF7FEFCE010D960E94C426CE010D9600
:106460000E94107DCE0101960E94107DCE010796FC
:106470000E94107D68EE73E080E090E00E945681FB
:106480000E94278ABC01CE010D960E94BD1E0E946B
:106490001F8ABC01CE0101960E94BD1E60E077E01C
:1064A000CE0107960E94AF7DBE016F5F7F4FCE0188
:1064B00007960E942B7CBC01CE010D960E94947C15
:1064C000CE0107960E94107DCE0101960E94107D9C
:1064D0000E947D880E940C896091D20B70E0CE01F1
:1064E00001960E94BD1E60E077E0CE0107960E94F3
:1064F000AF7DBE016F5F7F4FCE0107960E942B7C60
:10650000BC01CE010D960E94947CCE0107960E949C
:10651000107DCE0101960E94107D6CEF74E0CE01DB
:1065200001960E94AF7DBE01635F7F4FCE01019651
:106530000E942B7CBC01CE0107960E94A67D4AE0FA
:1065400050E06FEF7FEFCE0107960E94C426CE0188
:1065500007960E94107DCE0101960E94107DCE010B
:106560000D960E94107D68EE73E080E090E00E943E
:106570005681CE0101960E9493214AE050E06FEFD0
:106580007FEFCE0101960E94C4268ECECF92DF927D
:10659000EF92FF920F931F93CF93DF93CDB7DEB7A8
:1065A00068970FB6F894DEBF0FBECDBF6DE174E003
:1065B000CE0143960E94AF7D61E877E0CE0101965F
:1065C0000E949D7DCE0101960E94121BCE01019674
:1065D0000E94107D69EE70E1CE0101960E94AF7DB0
:1065E000CE0101960E94FB1ACE0101960E94107DF9
:1065F00061E777E0CE0101960E949D7DCE01019674
:106600000E94121BCE0101960E94107D6CA17DA1FB
:10661000CE0101960E94FD7ACE0101960E94FB1ADE
:10662000CE0101960E94107D69E577E0CE010196CA
:106630000E949D7DCE0101960E94121BCE01019603
:106640000E94107DCE5ADE4F68817981C255D140BB
:10665000CE0101960E94FD7ACE0101960E94FB1A9E
:10666000CE0101960E94107D6CE477E0CE01019688
:106670000E949D7DCE0101960E94121BCE010196C3
:106680000E94107D0AEA1BE0EE24E394F12CCE5A1E
:10669000DE4F88819981C255D1408E159F050CF43B
:1066A0004AC0F80182819381C6979CF162E075E04F
:1066B000CE0101960E94AF7DCE0101960E94121B71
:1066C000CE0101960E94107DF801628173816653AC
:1066D0007109CE0101960E94FD7ACE0101960E94B9
:1066E000121BCE0101960E94107D60E476E0CE017F
:1066F00001960E94AF7DCE0101960E94121BCE0131
:1067000001960E94107DFFEFEF1AFF0A0E5F1F4FE8
:10671000BECF6DEB76E0CE0101960E94AF7DCE013B
:1067200001960E94121BCE0101960E94107DF80175
:1067300062817381CECF60E476E0CE0101960E9443
:10674000AF7DCE0101960E94FB1ACE0101960E94F8
:10675000107D6DE377E0CE0101960E949D7DCE0114
:1067600001960E94121BCE0101960E94107D60913D
:10677000690B70916A0BCE0101960E94FD7ACE01E1
:1067800001960E94121BCE0101960E94107D60E4CA
:1067900076E0CE0101960E94AF7DCE0101960E9467
:1067A000121BCE0101960E94107D60916B0B7091BF
:1067B0006C0BCE0101960E94FD7ACE0101960E94DB
:1067C000FB1ACE0101960E94107D66E277E0CE01B1
:1067D00001960E949D7DCE0101960E94121BCE0162
:1067E00001960E94107DBE01605D7F4FCE01019633
:1067F0000E94AF7DCE0101960E94121BCE01019630
:106800000E94107D60E476E0CE0101960E94AF7D8B
:10681000CE0101960E94121BCE0101960E94107DAE
:10682000BE016C5C7F4FCE0101960E94AF7DCE0110
:1068300001960E94FB1ACE0101960E94107D66E12E
:1068400077E0CE0101960E949D7DCE0101960E94C7
:10685000FB1ACE0101960E94107D8E010C5D1F4F28
:10686000EE24E394F12C680188E0C80ED11C8CA1C1
:106870009DA18E159F050CF449C0B701CE01079666
:106880000E94FD7A68EC77E0CE0101960E94AF7D10
:10689000BE01695F7F4FCE0101960E942B7CBC0137
:1068A000CE010D960E94A67DCE010D960E94121B70
:1068B000CE010D960E94107DCE0101960E94107DA2
:1068C000CE0107960E94107D60E077E0CE01019630
:1068D0000E94AF7DCE0101960E94121BCE0101964F
:1068E0000E94107DB801645E7F4FCE0101960E9428
:1068F000AF7DCE0101960E94FB1ACE0101960E9447
:10690000107DEFEFEE1AFE0A8601ADCF65E077E06D
:10691000CE0101960E949D7DCE0101960E94121B20
:10692000CE0101960E94107D7E01F2EBEF1AFEEF80
:10693000FF0A10E000E0F70161917F0170E0CE01F5
:1069400001960E94FD7ACE0101960E94121BCE0193
:1069500001960E94107D0330110571F064E075E02E
:10696000CE0101960E94AF7DCE0101960E94121BBE
:10697000CE0101960E94107D0F5F1F4F043011055C
:10698000D1F660E476E0CE0101960E94AF7DCE01A3
:1069900001960E94FB1ACE0101960E94107DC45BF5
:1069A000DE4F68817981CC54D140072E000C880BD2
:1069B000990B0E9489AF9B01AC010E9449B28823C8
:1069C00041F080E590E0C45BDE4F99838883CC542E
:1069D000D140C45BDE4F88819981CC54D1409093E3
:1069E0003F0280933E026BEE76E0CE0101960E945C
:1069F0009D7DCE0101960E94121BCE0101960E9440
:106A0000107D6AE97BE0CE0101960E94AF7DCE0148
:106A100001960E94121BCE0101960E94107D69EE24
:106A200076E0CE0101960E949D7DCE0101960E94E6
:106A3000121BCE0101960E94107D60913E02709162
:106A40003F02CE0101960E94FD7ACE0101960E947E
:106A5000FB1ACE0101960E94107D6AED76E0CE0110
:106A600001960E949D7DCE0101960E94121BCE01CF
:106A700001960E94107DBE016C5A7F4FCE01019697
:106A80000E94AF7DCE0101960E94FB1ACE010196B5
:106A90000E94107D66E075E0CE0101960E94AF7DF8
:106AA000CE0101960E94121BCE0101960E94107D1C
:106AB000BE0164587F4FCE0101960E94AF7DCE018A
:106AC00001960E94FB1ACE0101960E94107DC052D1
:106AD000DF4F88819981C05ED040892B71F462EDCF
:106AE00076E0CE0101960E949D7DCE0101960E9426
:106AF000FB1ACE0101960E94107DC052DF4F8881A3
:106B00009981C05ED040019771F468EC76E0CE01C7
:106B100001960E949D7DCE0101960E94FB1ACE0136
:106B200001960E94107DC052DF4F88819981C05E1E
:106B3000D040029771F46FEB76E0CE0101960E948F
:106B40009D7DCE0101960E94FB1ACE0101960E9406
:106B5000107D69EB76E0CE0101960E949D7DCE010D
:106B600001960E94121BCE0101960E94107DCE510B
:106B7000DF4F68817981C25ED040CE0101960E94CC
:106B8000FD7ACE0101960E94FB1ACE0101960E9469
:106B9000107D60EB76E0CE0101960E949D7DCE01D6
:106BA00001960E94121BCE0101960E94107DCC5AC4
:106BB000DE4F88819981C455D140C6970CF41FC11E
:106BC00062E075E0CE0101960E94AF7DCE01019694
:106BD0000E94121BCE0101960E94107DCC5ADE4FFE
:106BE00068817981C455D14066537109CE010196FF
:106BF0000E94FD7ACE0101960E94FB1ACE010196F9
:106C00000E94107D4091E10B5091E20B6091E30BEB
:106C10007091E40B21E0CE0107960E94187D61E19E
:106C200075E0CE0101960E94AF7DBE01695F7F4F86
:106C3000CE0101960E942B7C6CE175E00E94157CD0
:106C4000BC01CE010D960E94A67DCE010D960E943C
:106C5000FB1ACE010D960E94107DCE0101960E9476
:106C6000107DCE0107960E94107D4091DD0B509162
:106C7000DE0B6091DF0B7091E00B21E0CE010796F7
:106C80000E94187D61E275E0CE0101960E94AF7D01
:106C9000BE01695F7F4FCE0101960E942B7C6CE1A3
:106CA00075E00E94157CBC01CE010D960E94A67D68
:106CB000CE010D960E94FB1ACE010D960E94107D0A
:106CC000CE0101960E94107DCE0107960E94107D94
:106CD00062E976E0CE0101960E949D7DCE0101968B
:106CE0000E94121BCE0101960E94107D4091290244
:106CF00050912A0260912B0270912C0225E0CE0166
:106D000001960E94187DCE0101960E94FB1ACE01C9
:106D100001960E94107D68E776E0CE0101960E9400
:106D20009D7DCE0101960E94121BCE0101960E940C
:106D3000107D4091250250912602609127027091AA
:106D4000280225E0CE0101960E94187DCE01019611
:106D50000E94FB1ACE0101960E94107D68E676E043
:106D6000CE0101960E949D7DCE0101960E94121BCC
:106D7000CE0101960E94107D60916C0270916D02AF
:106D8000CE0101960E94FD7ACE0101960E94FB1A67
:106D9000CE0101960E94107D66E576E0CE01019657
:106DA0000E949D7DCE0101960E94121BCE0101968C
:106DB0000E94107DC65BDE4F68817981CA54D14044
:106DC000CE0101960E94FD7ACE0101960E94FB1A27
:106DD000CE0101960E94107DCE0143960E94107D47
:106DE00068960FB6F894DEBF0FBECDBFDF91CF918E
:106DF0001F910F91FF90EF90DF90CF9008956DEB72
:106E000076E0CE0101960E94AF7DCE0101960E94F0
:106E1000121BCE0101960E94107DCC5ADE4F688174
:106E20007981C455D140E2CE2F923F924F925F922A
:106E30006F927F928F929F92AF92BF92CF92DF928A
:106E4000EF92FF920F931F93CF93DF93CDB7DEB7EF
:106E5000EC970FB6F894DEBF0FBECDBF3C018B019F
:106E600070E060E00E94C97B8F8F6DE174E0CE011D
:106E700049960E94AF7D80916C0290916D020197BE
:106E800009F07AC082E090E00E94C38888E090E038
:106E9000909324028093230289E090E09093220251
:106EA000809321028091670B9091680B9093660B01
:106EB0008093650B80911D0290911E02A0911F028C
:106EC000B09120028093190290931A02A0931B02A2
:106ED000B0931C028091350290913602A091370246
:106EE000B09138028093390290933A02A0933B020A
:106EF000B0933C028091640B8093630B80915F0B95
:106F00009091600BA091610BB091620B80935B0B31
:106F100090935C0BA0935D0BB0935E0B8AE390E0C3
:106F200090931802809317028091E10B9091E20BED
:106F3000A091E30BB091E40B8093960B9093970B89
:106F4000A093980BB093990B809115029091160223
:106F500090931402809313028091290290912A0247
:106F6000A0912B02B0912C0280932D0290932E02BF
:106F7000A0932F02B093300280916C0290916D0229
:106F8000029709F07AC083E090E00E94C3888AE00B
:106F900090E090932402809323028BE090E0909302
:106FA0002202809321028091590B90915A0B909369
:106FB000660B8093650B80910F0290911002A09157
:106FC0001102B09112028093190290931A02A093B9
:106FD0001B02B0931C028091310290913202A09169
:106FE0003302B09134028093390290933A02A09315
:106FF0003B02B0933C028091580B8093630B8091CD
:10700000540B9091550BA091560BB091570B809358
:107010005B0B90935C0BA0935D0BB0935E0B8BE3CB
:1070200090E090931802809317028091DD0B90916D
:10703000DE0BA091DF0BB091E00B8093960B909349
:10704000970BA093980BB093990B80910D029091A0
:107050000E02909314028093130280912502909166
:107060002602A0912702B091280280932D029093CE
:107070002E02A0932F02B09330022F8D2335C1F43E
:107080001092660B1092650B80916D0B882371F046
:1070900068E275E0CE0101960E94AF7DCE010196B7
:1070A0000E94FB1ACE0101960E94107DE12CFCC0CB
:1070B000C8010197029708F038C281E090E0A0E093
:1070C000B0E08093190290931A02A0931B02B09330
:1070D0001C02D30114968D919C91029748F141E0D6
:1070E00050E0B301CE0101960E94B11EBE016F5F58
:1070F0007F4FCE0149960E94D77CCE0101960E9417
:10710000107DCE0149960130110581F50E94567B14
:1071100020E030E040E251E40E94E8AF0E940EB26D
:107120006093190270931A0280931B0290931C02C1
:10713000BF8D81E090E09093660B8093650BB13436
:1071400001F580916D0B882309F4B0CF6DE275E0F5
:10715000CE0101960E94AF7DCE0101960E94FB1ADE
:10716000CE0101960E94107DE12C6BC00E94567BDF
:1071700020912D0230912E0240912F025091300229
:10718000CBCFEF8DE63409F075C160E0809121022C
:107190000E94E37F64E670E080E090E00E94568108
:1071A00061E0809123020E94E37F64E670E080E06A
:1071B00090E00E94568160E0809121020E94E37F6E
:1071C00064E670E080E090E00E94568161E080918A
:1071D00023020E94E37F64E670E080E090E00E947A
:1071E000568102301105C1F4CE0149960E94567BAA
:1071F0009B01AC016091960B7091970B8091980B5D
:107200009091990B0E942FB16093960B7093970BFE
:107210008093980B9093990B80916D0B882371F05C
:1072200066E375E0CE0101960E94AF7DCE01019626
:107230000E94121BCE0101960E94107DEE24E39461
:10724000F12C80916D0B882379F1409119025091B6
:107250001A0260911B0270911C022AE0CE01019675
:107260000E944E7DBE016F5F7F4FCE0107960E9448
:10727000A67D6AE475E0CE0107960E94157CBC01EC
:10728000CE010D960E94A67DCE010D960E94FB1A9E
:10729000CE010D960E94107DCE0107960E94107DB2
:1072A000CE0101960E94107D8091190290911A02E0
:1072B000A0911B02B0911C02181619061A061B0693
:1072C0000CF0E7C53F8D363409F4EFC4323509F4CC
:1072D000F0C460E0809121020E94E37F64E670E0E8
:1072E00080E090E00E9456816E2D809123020E94E2
:1072F000E37F64E670E080E090E00E945681609158
:10730000650B809121020E94E37F61E070E080E0E4
:1073100090E00E94568160E0809121020E94E37F0C
:1073200068EC70E080E090E00E945681C12CD12C86
:107330007601C3948091190290911A02A0911B02C8
:10734000B0911C02C816D906EA06FB060CF0B3C4BD
:107350006091650B809121020E94E37F61E070E003
:1073600080E090E00E94568160E0809121020E94BE
:10737000E37F6091390270913A0280913B029091D3
:107380003C020E9456818091390290913A02A0916C
:107390003B02B0913C020B97A105B1050CF464C00F
:1073A00060912D0270912E0280912F0290913002F7
:1073B0009B01AC010E9430B10E940EB29B01AC0156
:1073C000C701B6010E94EEB0672B682B692B09F04C
:1073D0004BC0023011050CF447C069EB75E089E73A
:1073E0009FE00E949B7CC701B6010E9489AF20915B
:1073F0002D0230912E0240912F02509130020E94B6
:107400009CB1AB01BC0120E0CE0107960E94187D23
:1074100069E77FE0CE0101960E94A67DBE01695F0B
:107420007F4FCE0101960E942B7C6CE175E00E949B
:10743000157CBC0189E79FE00E94C07CCE010196CB
:107440000E94107DCE0107960E94107D69E77FE0C3
:10745000CE0101960E94A67DCE0101960E94992739
:10746000CE0101960E94107D4FEFC41AD40AE40A9F
:10747000F40A60CFFF8DF23509F076CE60E080919E
:1074800021020E94E37F64E670E080E090E00E94C9
:10749000568160E0809123020E94E37F64E670E001
:1074A00080E090E00E94568160E0809121020E947D
:1074B000E37F64E670E080E090E00E94568160E047
:1074C000809123020E94E37F64E670E080E090E018
:1074D0000E94568102301105C1F4CE0149960E94E6
:1074E000567B9B01AC016091960B7091970B80913C
:1074F000980B9091990B0E9430B16093960B70930A
:10750000970B8093980B9093990B80916D0B882328
:1075100009F4CCCD60E475E0CE0101960E94AF7D08
:10752000CE0101960E94121B1BCE0115110521F000
:107530000330110509F0BACD80916C0290916D0273
:1075400020E137E240E050E08130910521F420E471
:107550003CE940E050E02EA73FA748AB59AB21E003
:1075600030E03093660B2093650B30935D022093DF
:107570005C02029759F40330110541F480914411E3
:107580009091451190935D0280935C0240915C0262
:1075900050915D025DA74CA7551F5527551F5AAB4B
:1075A00081E090E090935D0280935C0260E08091C6
:1075B00021020E94E37F64E670E080E090E00E9498
:1075C00056816AA9809123020E94E37F64E670E0FD
:1075D00080E090E00E94568160E0809121020E944C
:1075E000E37F64E670E080E090E00E9456816AA943
:1075F000809123020E94E37F64E670E080E090E0E7
:107600000E9456818FEF9FEF909314028093130294
:10761000812C912C540118A619A61AA61BA61CA2EF
:107620001DA21EA21FA218A219A21AA21BA2212CDF
:10763000312C21011FAA18AE19AE1AAE1BAA1CAA22
:107640001DAA1EAA61E0809121020E94E37F61E0F1
:1076500070E080E090E00E94568160E0809121021D
:107660000E94E37F61E070E080E090E00E9456813C
:10767000C501B40126E030E040E050E00E94EEB0E9
:10768000672B682B692B09F0F8C0A2E0B0E0BCAF13
:10769000ABAFC12CD12C760180911702863308F054
:1076A000865320917B00982F9870277F922B909380
:1076B0007B008770806480937C0080917A00806476
:1076C00080937A0080917A0086FDFCCF80917800CB
:1076D00060917900762F682F072E000C880B990B8C
:1076E0000E9489AF9B01AC01C701B6010E9430B175
:1076F0006B017C0162E070E080E090E00E945681C6
:107700002BAD3CAD2130310509F0ADC020E030ECAF
:107710004FEF54E4C701B6010E949CB16B017C019C
:1077200080916D0B882399F12DEC3CEC4CE45EE3E9
:10773000C701B6010E9444B287FD29C022E0B7010B
:10774000A601CE0107960E94187D61E575E0CE0185
:1077500001960E94AF7DBE01695F7F4FCE01019609
:107760000E942B7CBC01CE010D960E94A67DCE010D
:107770000D960E94FB1ACE010D960E94107DCE013F
:1077800001960E94107DCE0107960E94107D2AE985
:1077900039E949E95EE3C701B6010E9444B287FDB9
:1077A00013C0211431044104510411F414012501C2
:1077B0008CA19DA1AEA1BFA1892B8A2B8B2B21F47B
:1077C0008CA29DA2AEA2BFA22DEC3CEC4CE45EE3E9
:1077D000C701B6010E9482AF18160CF449C02114EB
:1077E00031044104510409F448C028A139A14AA137
:1077F0005BA1232B242B252B69F488A599A5AAA589
:10780000BBA5892B8A2B8B2B09F401C188A299A2D5
:10781000AAA2BBA228A139A14AA15BA122163306C4
:107820004406550654F5809113029091140297FF77
:10783000F3C01092140210921302220E331E441E43
:10784000551ED201C101B595A795979587958FAB28
:1078500098AFA9AFBAAF18A219A21AA21BA2212CE5
:10786000312C21010AC0E1E0F0E0FCAFEBAF14CF16
:10787000211431044104510469F6E0901302F090A0
:10788000140292E0E916F10434F4F7FCE1C003308D
:10789000110509F0DDC08EA49FA4A8A8B9A8AAE08C
:1078A0008A0E911CA11CB11C8EA59FA5A8A9B9A9DF
:1078B00088169906AA06BB060CF4C4CEE2E0EE16C2
:1078C000F1040CF479C06BA97CA98DA99EA92FA9FC
:1078D00038AD49AD5AAD621B730B840B950B0E94FA
:1078E00089AF4B015C01B701FF0C880B990B0E941B
:1078F00089AF9B01AC01C501B4010E949CB120E09D
:1079000030E044EB53E40E949CB16B017C01C092D7
:107910002D02D0922E02E0922F02F092300220E04F
:1079200030E040E85FE30E9444B287FDABC0809145
:107930006C0290916D028130910509F08FC0C09268
:107940003C11D0923D11E0923E11F0923F11C09255
:107950002902D0922A02E0922B02F0922C026CEDC6
:1079600075E0CE0101960E949D7DCE0101960E9498
:10797000121BCE0101960E94107D40912D02509164
:107980002E0260912F027091300225E0CE01019607
:107990000E94187DCE0101960E94FB1ACE0101962D
:1079A0000E94107D84EF91E09093670280936602BD
:1079B0006EE170E10E945A090330110531F03AA9D5
:1079C000E32E0115110509F06FCCC3010E94567B0F
:1079D0006B017C01C092960BD092970BE092980BB2
:1079E000F092990B20E030E044EB53E4C701B6017C
:1079F0000E9444B287FD6AC020E030E044EB53E4CB
:107A0000C701B6010E942FB16B017C01EBCF88A6A4
:107A100099A6AAA6BBA6FACE0115110509F02DCF8D
:107A20000196909314028093130228A139A14AA1D0
:107A30005BA1220E331E441E551ED201C101B59515
:107A4000A795979587958BAB9CABADABBEAB03CFA2
:107A5000BFEF8B1A9B0AAB0ABB0A26CF029709F02D
:107A60007ECFC0924011D0924111E0924211F0922B
:107A70004311C0922502D0922602E0922702F09292
:107A800028026DCF60EC75E0CE0101960E949D7DCD
:107A9000CE0101960E94121BCE0101960E94107D1C
:107AA00040912D0250912E0260912F027091300270
:107AB00025E0CE0101960E94187DCE0101960E941C
:107AC000FB1ACE0101960E94107D76CF20E030E0B7
:107AD000A901C701B6010E9482AF87FF0BC020E059
:107AE00030E044EB53E4C701B6010E9430B16B01B2
:107AF0007C01ECCFC0925B0BD0925C0BE0925D0BF3
:107B0000F0925E0B48A459A46AA47BA48CA19DA109
:107B1000AEA1BFA1481A590A6A0A7B0A01151105CC
:107B2000D9F410925B0B10925C0B10925D0B1092CB
:107B30005E0BACA5BDA5C12CD12C7601C394812CC4
:107B4000912C5401B7FF1CC0812C912C5401CC24E2
:107B5000CA94DC2C760114C0ECA5FDA5C12CD12C57
:107B60007601C394F7FF04C0CC24CA94DC2C7601C0
:107B700080905B0B90905C0BA0905D0BB0905E0BC7
:107B800020912D0230912E0240912F02509130020F
:107B9000C501B4010E94E8AF4B015C01A301920151
:107BA000C701B6010E94BCB00E9489AF20E030E05E
:107BB00040E05FE30E94E8AF9B01AC01C501B40166
:107BC0000E942FB10E940EB26093190270931A02A4
:107BD00080931B0290931C0280916D0B882309F403
:107BE00041C02AE048A559A56AA57BA5CE010D96FE
:107BF0000E944E7D2AE04CA15DA16EA17FA1CE0125
:107C000007960E944E7D68E575E0CE0101960E94C0
:107C1000AF7DBE01695F7F4FCE0101960E942B7C34
:107C200060E476E00E94157CBE01635F7F4F0E9496
:107C30002B7CBC01CE0143960E94A67DCE014396CB
:107C40000E94FB1ACE0143960E94107DCE01019640
:107C50000E94107DCE0107960E94107DCE010D96E8
:107C60000E94107D8091190290911A02A0911B022E
:107C7000B0911C02B7FF15C0B095A0959095819565
:107C80009F4FAF4FBF4F8093190290931A02A0935A
:107C90001B02B0931C02EE24E394F12CF6E4FF8F58
:107CA00003CBE12C22E52F8FFFCAEE24E394F12CC5
:107CB00010CBE12C0ECB0230110524F40115110577
:107CC00009F0DFC061E080E00E94418C02301105C4
:107CD00024F40115110509F09CC0C090960BD090BA
:107CE000970BE090980BF090990B20E030E044EB7C
:107CF00053E4C701B6010E9444B287FD0BC020E0E7
:107D000030E044EB53E4C701B6010E942FB16B0190
:107D10007C01EBCF20E030E0A901C701B6010E9451
:107D200082AF87FF0BC020E030E044EB53E4C70193
:107D3000B6010E9430B16B017C01ECCFC092960B72
:107D4000D092970BE092980BF092990B80916C0275
:107D500090916D020197B1F461E175E089E79FE0D0
:107D60000E94F37A8091960B9091970BA091980BBB
:107D7000B091990B8093E10B9093E20BA093E30BEE
:107D8000B093E40B80916C0290916D020297B1F474
:107D900061E275E089E79FE00E94F37A8091960B9B
:107DA0009091970BA091980BB091990B8093DD0B5C
:107DB0009093DE0BA093DF0BB093E00B4091960BFA
:107DC0005091970B6091980B7091990B20E0CE0128
:107DD00007960E94187D69E77FE0CE0101960E9418
:107DE000A67DBE01695F7F4FCE0101960E942B7C6C
:107DF0006DE175E00E94157CBC0189E79FE00E945F
:107E0000C07CCE0101960E94107DCE0107960E9493
:107E1000107D0130110539F54091190250911A0277
:107E200060911B0270911C0221E0CE0107960E9416
:107E30004E7D60E675E0CE0101960E94AF7DBE01E9
:107E4000695F7F4FCE0101960E942B7CBC0189E7C0
:107E50009FE00E94C07CCE0101960E94107DCE0161
:107E600007960E94107D69E77FE0CE0101960E948F
:107E7000A67DCE0101960E949927CE0101960E940F
:107E8000107D1092190210921A0210921B02109289
:107E90001C0280916C0290916D028130910509F075
:107EA00083C08091650B9091660B9093680B8093D3
:107EB000670B8091190290911A02A0911B02B09158
:107EC0001C0280931D0290931E02A0931F02B09388
:107ED00020028091390290913A02A0913B02B09128
:107EE0003C028093350290933602A0933702B09300
:107EF00038028091630B8093640B80915B0B9091AF
:107F00005C0BA0915D0BB0915E0B80935F0B909327
:107F1000600BA093610BB093620B8091960B9091D4
:107F2000970BA091980BB091990B8093E10B9093D4
:107F3000E20BA093E30BB093E40B809113029091BA
:107F400014029093160280931502012B81F4809104
:107F50002D0290912E02A0912F02B09130028093B9
:107F6000290290932A02A0932B02B0932C02CE01F7
:107F700049960E94107DEC960FB6F894DEBF0FBEB6
:107F8000CDBFDF91CF911F910F91FF90EF90DF90C8
:107F9000CF90BF90AF909F908F907F906F905F90A9
:107FA0004F903F902F900895029709F78091650BAD
:107FB0009091660B90935A0B8093590B8091190204
:107FC00090911A02A0911B02B0911C0280930F02A3
:107FD00090931002A0931102B09312028091390283
:107FE00090913A02A0913B02B0913C028093310201
:107FF00090933202A0933302B09334028091630BCA
:108000008093580B80915B0B90915C0BA0915D0B62
:10801000B0915E0B8093540B9093550BA093560B2D
:10802000B093570B8091960B9091970BA091980B62
:10803000B091990B8093DD0B9093DE0BA093DF0B37
:10804000B093E00B809113029091140290930E0272
:1080500080930D02012B09F08ACF80912D0290911F
:108060002E02A0912F02B0913002809325029093AE
:108070002602A0932702B093280279CF6F927F92B5
:108080008F929F92AF92BF92CF92DF92EF92FF9228
:108090000F931F93CF93DF93CDB7DEB7C456D109AB
:1080A0000FB6F894DEBF0FBECDBF40E052EC61E0EA
:1080B00070E085E29DE00E94907740E855E260E044
:1080C00070E088E89CE00E94907761E088E00E9480
:1080D000008161E089E00E94008160E08AE30E9403
:1080E000008161E088E00E94E37F60E089E00E9417
:1080F000E37F61E08AE00E94008161E08BE00E9402
:10810000008160E08BE30E94008161E08AE00E94D0
:10811000E37F60E08BE00E94E37F0E94E98084EFD0
:1081200091E0909367028093660268ED7AE085E2C1
:108130009DE00E94F37E67E779E085E29DE00E9482
:10814000107E60ED77E080E090E00E94568185E24D
:108150009DE00E944674982E0EE110E091100BC035
:1081600085E29DE00E944674982E6EE170E080E00A
:1081700090E00E9456810150110981F780916602BA
:1081800090916702A0E5AA2EA1E1BA2EBEE1EB2EE6
:10819000B0E1FB2E9C012E5130416901C6018E0DCC
:1081A0009F1D0E94A6B0F70181937F01AE16BF0606
:1081B000A9F76091381170913911072E000C880BC6
:1081C000990B0E9489AF9B01AC010E9449B28823A0
:1081D00031F081E090E090933911809338116091F3
:1081E0003A1170913B11072E000C880B990B0E94DD
:1081F00089AF9B01AC010E9449B2882331F082E033
:1082000090E090933B1180933A11F5E79F16B1F0FF
:108210006091341170913511809136119091371120
:108220000E9489AF9B01AC010E9449B2811106C036
:1082300080911E1090911F108197E8F02DB73EB7E6
:10824000225331400FB6F8943EBF0FBE2DBFADB7DD
:10825000BEB7119682E391E0EEE1F0E101900D925C
:108260000197E1F70E94452C0FB6F894DEBF0FBED0
:10827000CDBFF5E79F2EEDB7FEB7E253F1400FB645
:10828000F894FEBF0FBEEDBFADB7BEB7119682E347
:1082900091E0EEE1F0E101900D920197E1F70E948B
:1082A0004B240FB6F894DEBF0FBECDBF35E7931653
:1082B00019F083E798121BC0EDB7FEB7E253F14007
:1082C0000FB6F894FEBF0FBEEDBFADB7BEB71196A7
:1082D00082E391E0EEE1F0E101900D920197E1F788
:1082E0000E94C6320FB6F894DEBF0FBECDBF66EC5B
:1082F0007AE080ED9FE00E949B7C60EB7AE08AEC64
:108300009FE00E949B7C0E94E980E7E2CE2ED12C68
:10831000E12CF12CB12CA12C882483948092830C25
:10832000C092850C1092840C1092860C81E00E9401
:10833000FC8A8111B0C1C092D8113FEFA31AB30AD1
:108340008FEFC81AD80AE80AF80A90E4C916D104CF
:10835000E104F10419F7AB2831F462E875E085E235
:108360009DE00E94B57E0E94E9801092D911809113
:10837000DD11823018F098E09093D9119091DE11C0
:10838000992339F0813029F48091D9118460809348
:10839000D91162E370E080E090E00E945681609124
:1083A000DF1184ED91E10E94EC8B68EE73E080E0D8
:1083B00090E00E94568160E384ED91E10E94008C80
:1083C0005BE4E52E56E4F52EC7010197F1F760E373
:1083D00084ED91E10E94008CC7010197F1F760E301
:1083E00084ED91E10E94008C83E592E00197F1F722
:1083F00060E284ED91E10E94008C8091D91180624D
:108400000E94308C84E08093DA118CE00E94308CE2
:1084100081E00E94308C6BE3E62E6FE1F62EC701FF
:108420000197F1F782E08093DB1186E00E94308CA7
:1084300082E00E94308CC7010197F1F780E40E942E
:10844000308C7EE5E72E72E0F72EF70161917F0117
:1084500084ED91E10E94198CF6E6EF16F2E0FF063A
:10846000A1F70E940C0A0E94FC0964E670E080E01B
:1084700090E00E94568168E97AE0CE0101960E9460
:108480009D7DCE0101960E94FB1ACE0101960E94AD
:10849000107D61E085E30E94008161E085E30E9438
:1084A000E37F61E08AE00E94008161E08AE00E944F
:1084B000E37F61E089E30E9400818091B00E803308
:1084C00008F050C061E089E30E9400818091B00E05
:1084D000282F30E0F901EE0FFF1FE20FF31FE35EDC
:1084E000F14F9081907C996390831092B10E10921D
:1084F000B20E2CE0622F0E944EB2829FB001112476
:108500009B01200F311FF901EE0FFF1FE20FF31F38
:10851000E35EF14F908196FD17C00F5F1F4F0C3047
:10852000110571F7813009F0CDC01092800082E012
:10853000809381001092850010928400B19A8091FE
:108540006F00826080936F00E091B00E8E2F90E0FC
:10855000FC01EE0FFF1FE80FF91FE35EF14F808172
:108560008064808368EC70E080E090E00E94568137
:1085700068EE73E080E090E00E94568167E87AE060
:10858000CE0101960E949D7D4AE050E06FEF7FEFA3
:10859000CE0101960E94C426CE0101960E94107D54
:1085A0001092D90D1092D70D1092D40D1092D30DB8
:1085B00084E08093D20D0E9425848B0161E080913C
:1085C000D20D0E9400818EEC9DE00E94A60860E022
:1085D00082E30E94008161E083E30E94008161E008
:1085E00084E30E94008161E085E30E94008161E0F4
:1085F00085E30E94E37F83E58CBD8DB58E7F8DBDC5
:10860000BAE0FB2E8FEF0E949B07FA94F110FACF8D
:1086100060E08091D20D0E94E37F20E030E0A9016C
:1086200060E08EEC9DE00E94A50BF82E8093D80DA3
:1086300021E0821709F472C00E942584601B710B2F
:10864000613D774050F381E08093D30D8EEC9DE047
:108650000E94A60869E77AE0CE0101960E949D7DFE
:10866000CE0101960E94FB1ACE0101960E94107D58
:1086700068E67AE0CE0101960E949D7D4AE050E0D6
:108680006FEF7FEFCE0101960E94300ACE01019676
:108690000E94107D58C1843009F052CE67E675E023
:1086A00085E29DE00E94C97E20E1B701A60185E236
:1086B0009DE00E941F7E67E779E085E29DE00E94D1
:1086C000107E3ECE823061F4109290008093910033
:1086D000109295001092940088BB8093710034CF63
:1086E000833069F41092A00082E08093A100109280
:1086F000A5001092A40089BB8093720025CF811140
:1087000023CF1092200182E0809321011092250155
:10871000109224018ABB8093730016CF2AEA31E0BD
:1087200040E050E068E08EEC9DE00E94A50B82FFE7
:108730002AC0F092D90D8091D90DC12CD12CE12CF9
:10874000F0E4FF2E823019F0C12CD12C760120E00C
:1087500030E0A90167E38EEC9DE00E94A50BA70124
:10876000960169E28EEC9DE00E94A50B8093D80DE6
:108770008823D1F00E942584601B710B613D7740F6
:1087800030F388E061CFA4E0FA2E0E94A00B809322
:10879000D80DFA94F110F9CF8A3A11F082E054CF53
:1087A00082E08093D90DC7CF8091D90D8230D1F46A
:1087B00020E030E0A9016AE38EEC9DE00E94A50B69
:1087C000882311F086E040CF0E94A00B807C803C83
:1087D00019F483E08093D90D0E94A00B0E94A00B96
:1087E0000E94A00B8EEC9DE00E94A6088DB58E7FA6
:1087F0008DBD8CB58C7F8CBD8CB58CBD81E00E940D
:10880000E478882309F49EC28091FD0D811122CF66
:108810008091F10D803109F09CC282E08093FD0DC2
:1088200010920F0E1092100E1092110E1092120E46
:108830008091F20D9091F30DB0E0A0E0E5E0880F9B
:10884000991FAA1FBB1FEA95D1F780930B0E909337
:108850000C0EA0930D0EB0930E0E8AED9DE090933A
:10886000140E8093130E81E08093FC0D1092FE0D88
:108870001092FF0D1092000E1092010E1092020E37
:108880001092030E1092040E1092050E1092060E16
:108890001092070E1092080E1092090E10920A0EF6
:1088A0006CE57AE0CE0101960E949D7DCE01019695
:1088B0000E94FB1ACE0101960E94107D41E068E6FD
:1088C00074E0CE0101960E94E494BE016F5F7F4F79
:1088D0008DE991E10E94221E80919F119091A0113B
:1088E0009C838B838091A1119091A211A091A311DF
:1088F000B091A4118D839E83AF83B8878091A51119
:108900009091A611A091A711B091A81189879A877B
:10891000AB87BC8784EF93E09A8389838DE0E9EA93
:10892000F1E1DE011D9601900D928A95E1F78091AB
:10893000B6119091B7119B8F8A8F70E060E0CE01E5
:1089400001960E94F31E68EE73E080E090E00E94C2
:10895000568143E162EB72E0CE0101960E94E494FD
:10896000BE016F5F7F4F88EB91E10E94221E63E2A0
:108970007AE08EEB9FE00E949B7C68E17AE08EEBD0
:108980009FE00E943E7C88EB91E10E945B0D882372
:1089900009F410C21EAE1DAE84E793E09CAF8BAF0E
:1089A00021961FAE219719A218A29F8F8E8F1BA20E
:1089B000812C712C7E019BE3E90EF11C08EF1DE078
:1089C00074E7A72E73E0B72E882D972DFC01EE5487
:1089D000FD4F20812F3209F40196DC01AE54BD4FCA
:1089E000FE01E85AFF4F30E020E06F014D914F3219
:1089F00049F0442339F001962F5F3F4F41932C30CB
:108A00003105A1F72C0D3D1DF9011082FC01EE543A
:108A1000FD4F20812F3209F40196882E792E8E5435
:108A20009D4FFC0160801C821B82BA82A9821E823B
:108A300021E0A601B801CE0101960E943A93882355
:108A400009F4D5C1CE0101960E949A0A6110A0C115
:108A50002DE0083F120719F0C8010E949A0A88EB1E
:108A600091E10E94670D66E970E080E090E00E946D
:108A7000568110924E0C04E610E091100BC085E276
:108A80009DE00E944674982E64E170E080E090E0E2
:108A90000E9456810150110981F763EF79E0CE0100
:108AA00001960E949D7D48EC50E070E060E0CE01B0
:108AB00001960E94300ACE0101960E94107D32E795
:108AC00081E0931280E00E948B0982E090E00E9496
:108AD000C3886CE271E080E090E00E94568183E000
:108AE00090E00E94C3886CE271E080E090E00E9418
:108AF000568101E010E010936D0200936C02109318
:108B00005D0200935C026AEA75E083E79FE00E94E1
:108B1000F37A63E77FE0CE0101960E94A67D62E0D2
:108B200070E0CE0101960E941437CE0101960E949A
:108B3000107D62EE79E0CE0101960E949D7DCE010E
:108B400001960E94FB1ACE0101960E94107D62EDF3
:108B500079E0CE0101960E949D7D48EC50E070E0E6
:108B600060E0CE0101960E94C426CE0101960E94CB
:108B7000107D62ED76E083E79FE00E94F37A63E781
:108B80007FE0CE0101960E94A67D63E070E0CE01F9
:108B900001960E941437CE0101960E94107D109319
:108BA0006D0200936C026CEB79E0CE0101960E949D
:108BB0009D7DCE0101960E94FB1ACE0101960E9476
:108BC000107D61EB79E0CE0101960E949D7D4AE027
:108BD00050E06FEF7FEFCE0101960E94C426CE01D8
:108BE00001960E94107D68EE73E080E090E00E94A4
:108BF00056810E949D2F0E94A5308DB79EB782534B
:108C000091400FB6F8949EBF0FBE8DBFADB7BEB7F3
:108C1000119682E391E0EEE1F0E101900D9201976F
:108C2000E1F70E94C6321092F70B81E89CE6909320
:108C3000280F8093270F2091490F0FB6F894DEBFBD
:108C40000FBECDBF2830D8F4822F90E0FC01EE0F8C
:108C5000FF1FEE0FFF1FE75DF04F4EEA55E0518317
:108C600040832F5F2093490F880F991F880F991F0A
:108C7000FC01E55DF04F83E790E2918380832091D2
:108C8000490F2830D8F4822F90E0FC01EE0FFF1F2F
:108C9000EE0FFF1FE75DF04F44EB55E0518340833B
:108CA0002F5F2093490F880F991F880F991FFC0190
:108CB000E55DF04F87E193E79183808387EB9EE04A
:108CC0000E94F1186FE979E0CE0101960E949D7D26
:108CD000CE0101960E94FB1ACE0101960E94107DE2
:108CE0001092F80B0E947D886093F90B7093FA0B39
:108CF0008093FB0B9093FC0B80911D118093500C83
:108D0000882351F00E947D886093EF0B7093F00BE5
:108D10008093F10B9093F20BCC59DF4F0FB6F89480
:108D2000DEBF0FBECDBFDF91CF911F910F91FF909E
:108D3000EF90DF90CF90BF90AF909F908F907F90FB
:108D40006F90089580E00E94E478882309F482CC33
:108D50005BCD803209F07ECC83E08093FD0D4091A5
:108D6000F40D5091F50D6091F60D7091F70D409353
:108D70000F0E5093100E6093110E7093120E2BE095
:108D80003EE08AED9DE00E94ED8E811166CD62CCC1
:108D900021E0A601B801C7010E943A93D82EFDE058
:108DA000083F1F0709F44DC0C8010E949A0AD1105C
:108DB0004DC024C063E07AE0CE0101960E949D7D03
:108DC000CE0101960E94121BCE0101960E94107DD9
:108DD00062EB72E0CE0101960E94AF7DCE0101965A
:108DE0000E94FB1ACE0101960E94107D42CEFDE04A
:108DF000083F1F0719F0C8010E949A0A68E975E048
:108E0000CE0101960E94AF7DCE0101960E94121BF9
:108E1000CE0101960E94107D62EB72E0CE010196B8
:108E20000E94AF7DCE0101960E94FB1ACE010196F1
:108E30000E94107D6EEB7FE088EB91E10E94DF7E67
:108E40000ECE8823D9F28E01025E1F4F902F812F04
:108E50008701E92EF82EB8CD2F923F924F925F9264
:108E60006F927F928F929F92AF92BF92CF92DF923A
:108E7000EF92FF920F931F93CF93DF93CDB7DEB79F
:108E8000E3970FB6F894DEBF0FBECDBF67E97FE072
:108E9000CE018E960E94A67D0EA51FA50115110577
:108EA00071F0D8018D918D01882349F0082E000CB6
:108EB000990B0E949CB4F80131978083F2CF68EB44
:108EC00075E0CE0101960E94AF7DBE016F5F7F4FBE
:108ED000CE018E960E94FA7B182FCE0101960E9439
:108EE000107D112309F401C145E050E067E97FE0FE
:108EF000CE0101960E94B11EBE016F5F7F4F83E7D6
:108F00009FE00E94D77CCE0101960E94107D83E7EE
:108F10009FE00E946C7B60E083E79FE00E94687C9A
:108F20004091770F5091780F66E770E183E79FE0FB
:108F30000E94AC7868E674E0CE0101960E94AF7D95
:108F4000BE016F5F7F4F83E79FE00E94FA7B182F7F
:108F5000CE0101960E94107D62E574E0111102C0FD
:108F600067E574E0CE0101960E94AF7D63E77FE084
:108F7000CE0101960E942B7CBC018CE791E10E94FE
:108F8000C07CCE0101960E94107D8CE791E10E9489
:108F90006C7B4091801150918111415051096CE7D7
:108FA00071E1CE0101960E94B11EBE016F5F7F4F3D
:108FB0008EE591E10E94D77CCE0101960E94107D42
:108FC0008EE591E10E94617B0E9489AF9B01AC011B
:108FD0000E9449B2882309F448C0609180117091C1
:108FE0008111625071098CE791E10E94C97B682F61
:108FF000CE0101960E947B7DBE016F5F7F4F8EE5A3
:1090000091E10E94D77CCE0101960E94107D68E616
:1090100074E0CE0101960E94AF7DBE016F5F7F4F6D
:109020008EE591E10E94FA7B182FCE0101960E94F5
:10903000107D1123D1F060918011709181116350E6
:1090400071098CE791E10E94C97B682FCE010196DE
:109050000E947B7DBE016F5F7F4F8EE591E10E9494
:10906000D77CCE0101960E94107D84EF91E0909311
:109070006702809366026EE170E10E945A0964E61D
:1090800070E080E090E00E94568180913D0288234C
:1090900071F067E97FE0CE0101960E94A67DCE01C6
:1090A00001960E946721CE0101960E94107DCE019B
:1090B0008E960E94107D81E0E3960FB6F894DEBF95
:1090C0000FBECDBFDF91CF911F910F91FF90EF9019
:1090D000DF90CF90BF90AF909F908F907F906F90D8
:1090E0005F904F903F902F9008956EEB75E0CE010A
:1090F00001960E94AF7DBE016F5F7F4FCE018E96BD
:109100000E94FA7B182FCE0101960E94107D112338
:1091100009F447C045E050E067E97FE0CE010196E1
:109120000E94B11EBE016F5F7F4F83E79FE00E94E8
:10913000D77CCE0101960E94107D83E79FE00E94BC
:109140006C7B60E083E79FE00E94687C4091770F32
:109150005091780F6EE470E183E79FE00E94AC7855
:109160006EE470E1CE014C960E94AF7D6AE674E039
:10917000CE0101960E94AF7DBE01645E7F4FCE019D
:1091800001960E942B7CBC0186E791E10E94C07C85
:10919000CE0101960E94107DCE014C960E94107D5A
:1091A00064CF64EC75E0CE0101960E94AF7DBE01F4
:1091B0006F5F7F4FCE018E960E94FA7B182FCE01F3
:1091C00001960E94107D1123E1F043E050E067E931
:1091D0007FE0CE0101960E94B11EBE016F5F7F4FFE
:1091E00083E79FE00E94D77CCE0101960E94107D0C
:1091F00063E77FE0CE0101960E94A67DCE01019635
:10920000CDCF68EC75E0CE0101960E94AF7DBE0126
:109210006F5F7F4FCE018E960E94FA7B182FCE0192
:1092200001960E94107D112301F144E050E067E9AE
:109230007FE0CE0101960E94B11EBE016F5F7F4F9D
:1092400083E79FE00E94D77CCE0101960E94107DAB
:1092500083E79FE00E94617B7093DD106093DC10D8
:1092600070938D0260938C0200CF6DEC75E0CE019F
:1092700001960E94AF7DBE016F5F7F4FCE018E963B
:109280000E94FA7B182FCE0101960E94107D1123B7
:1092900009F449C045E050E067E97FE0CE0101965E
:1092A0000E94B11EBE016F5F7F4F83E79FE00E9467
:1092B000D77CCE0101960E94107D83E79FE00E943B
:1092C000617B709339116093381184EF91E0909332
:1092D0006702809366026EE170E10E945A0964E6BB
:1092E00070E080E090E00E94568168EC77E0CE016B
:1092F00001960E94AF7D67E97FE0CE0101960E9452
:109300002B7CBC01CE014C960E94A67DCE014C96D2
:109310000E94FB1ACE014C960E94107DCE01019650
:109320000E94107DB2CE63ED75E0CE0101960E94E1
:10933000AF7DBE016F5F7F4FCE018E960E94FA7B9C
:10934000182FCE0101960E94107D1123E1F044E018
:1093500050E067E97FE0CE0101960E94B11EBE0198
:109360006F5F7F4F83E79FE00E94D77CCE0101961D
:109370000E94107D83E79FE00E94617B70933B1108
:1093800060933A11A2CF68ED75E0CE0101960E947C
:10939000AF7DBE016F5F7F4FCE018E960E94FA7B3C
:1093A000182FCE0101960E94107D1123A1F044E0F8
:1093B00050E067E97FE0CE0101960E94B11EBE0138
:1093C0006F5F7F4F83E79FE00E94D77CCE010196BD
:1093D0000E94107D84CF6DED75E0CE0101960E9454
:1093E000AF7DBE016F5F7F4FCE018E960E94FA7BEC
:1093F000182FCE0101960E94107D1123A1F047E0A5
:1094000050E067E97FE0CE0101960E94B11EBE01E7
:109410006F5F7F4F83E79FE00E94D77CCE0101966C
:109420000E94107D2CCE65EE75E0CE0101960E9463
:10943000AF7DBE016F5F7F4FCE018E960E94FA7B9B
:10944000182FCE0101960E94107D1111D8CF6DEE1C
:1094500075E0CE0101960E94AF7DBE016F5F7F4F28
:10946000CE018E960E94FA7B182FCE0101960E94A3
:10947000107D112321F081E00E948B0900CE67EF5F
:1094800075E0CE0101960E94AF7DBE016F5F7F4FF8
:10949000CE018E960E94FA7B182FCE0101960E9473
:1094A000107D112319F00E949D2FE9CD65E979E027
:1094B000CE0101960E949D7DBE016F5F7F4FCE0160
:1094C0008E960E94FA7B182FCE0101960E94107D85
:1094D000112309F485C06AE879E0CE0101960E9463
:1094E0009D7DBE016F5F7F4FCE018E960E94FA7BFD
:1094F000182FCE0101960E94107D112309F454C04B
:109500004AE050E067E97FE0CE0101960E94B11E7B
:10951000BE016F5F7F4F83E79FE00E94D77CCE0143
:1095200001960E94107D83E79FE00E94617B0E946C
:1095300058880E947D886093EF0B7093F00B8093A6
:10954000F10B9093F20B0E947D886093E90B70936E
:10955000EA0B8093EB0B9093EC0BCE014C960E94A0
:1095600014226EEF75E0CE0101960E94AF7DBE0120
:10957000645E7F4FCE0101960E942B7CBC01CE0120
:1095800082960E94A67DCE0182960E94FB1ACE0191
:1095900082960E94107DCE0101960E94107DCE0120
:1095A0004C960E94107D71CD4BE050E067E97FE062
:1095B000CE0101960E94B11EBE016F5F7F4F83E70F
:1095C0009FE00E94D77CCE0101960E94107D83E728
:1095D0009FE00E94617B60587F488F4F9F4FA7CFCD
:1095E00064E477E0CE0101960E94AF7DBE016F5F1B
:1095F0007F4FCE018E960E94FA7B182FCE010196E6
:109600000E94107D112309F46AC045E050E067E92B
:109610007FE0CE0101960E94B11EBE016F5F7F4FB9
:1096200083E79FE00E94D77CCE0101960E94107DC7
:109630000E947D886093EF0B7093F00B8093F10B89
:109640009093F20B83E79FE00E94617B60936E0230
:1096500070936F02809370029093710260931E1159
:1096600070931F11809320119093211120911D114F
:109670002093500C672B682B692B11F41092500C1F
:1096800084EF91E090936702809366026EE170E14F
:109690000E945A0964E670E080E090E00E945681E2
:1096A0006BE779E0CE0101960E949D7DCE01019687
:1096B0000E94121BCE0101960E94107D40916E0205
:1096C00050916F026091700270917102CE0101960B
:1096D0000E94297BCE0101960E94FB1ADBC16FE03C
:1096E00076E0CE0101960E94AF7DBE016F5F7F4F95
:1096F000CE018E960E94FA7B182FCE0101960E9411
:10970000107D1123D9F14AE050E067E97FE0CE01F6
:1097100001960E94B11EBE016F5F7F4F83E79FE0FD
:109720000E94D77CCE0101960E94107D83E79FE0C6
:109730000E94617B613071058105910519F481E01A
:1097400080931D1183E79FE00E94617B672B682B4C
:10975000692B11F410921D1180911D118093500CF2
:10976000882309F4B2CD0E947D886093EF0B70933B
:10977000F00B8093F10B9093F20BA7CD6AE176E0AA
:10978000CE0101960E94AF7DBE016F5F7F4FCE017B
:109790008E960E94FA7B182FCE0101960E94107DB2
:1097A0001123A1F048E050E067E97FE0CE01019687
:1097B0000E94B11EBE016F5F7F4F83E79FE00E9452
:1097C000D77CCE0101960E94107D8FCD63E276E0BA
:1097D000CE0101960E94AF7DBE016F5F7F4FCE012B
:1097E0008E960E94FA7B182FCE0101960E94107D62
:1097F000112321F145E050E067E97FE0CE010196B9
:109800000E94B11EBE016F5F7F4F83E79FE00E9401
:10981000D77CCE0101960E94107D83E79FE00E94D5
:10982000617B6130710521F481E08093510C2DCC76
:10983000672B09F02ACC1092510C27CC69E276E014
:10984000CE0101960E94AF7DBE016F5F7F4FCE01BA
:109850008E960E94FA7B182FCE0101960E94107DF1
:10986000112351F163E070E087E99FE00E94C97B1A
:10987000682FCE0101960E947B7DBE016F5F7F4FF6
:1098800083E79FE00E94D77CCE0101960E94107D65
:1098900083E79FE00E946C7B83E79FE00E94617BEF
:1098A0009B01215031092330310508F0EECB709334
:1098B0004D1160934C11D9CB6DE276E0CE0101964B
:1098C0000E94AF7DBE016F5F7F4FCE018E960E94DA
:1098D000FA7B182FCE0101960E94107D112309F406
:1098E0006AC066E070E087E99FE00E94C97B682F4C
:1098F000CE0101960E947B7DBE016F5F7F4F83E7A3
:109900009FE00E94D77CCE0101960E94107D83E7E4
:109910009FE00E946C7B60E083E79FE00E94687C90
:1099200083E79FE00E94617B6B01CB010197039766
:1099300008F0ABCB48E050E067E97FE0CE0101964C
:109940000E94B11EBE016F5F7F4F83E79FE00E94C0
:10995000D77CCE0101960E94107D83E79FE00E9494
:109960006C7B8091770F9091780F0997A8F028E091
:1099700030E050E040E063E77FE0CE0101960E94D6
:10998000C47DBE016F5F7F4F83E79FE00E94D77C5D
:10999000CE0101960E94107DB60113E0660F771F7D
:1099A0001A95E1F76E5C7F4E48E050E083E79FE058
:1099B0000E94AC785ACB63E779E0CE0101960E9411
:1099C0009D7DBE016F5F7F4FCE018E960E94FA7B18
:1099D000182FCE0101960E94107D112309F486C034
:1099E0006DE174E0CE0101960E94AF7D47E050E04A
:1099F000BE01625D7F4FCE014C960E94B11EBE013A
:109A0000645E7F4FCE0101960E94D77CCE014C96BA
:109A10000E94107D62E075E0CE014C960E94AF7D01
:109A2000BE01645E7F4FCE0101960E94FA7B182F23
:109A3000CE014C960E94107D112379F141E050E057
:109A4000BE016F5F7F4FCE014C960E94B11ECE01CA
:109A50004C960E94617B8B010A5C1F4FCE014C9695
:109A60000E94107D10934F1100934E1110938F029E
:109A700000938E0284EF91E09093670280936602D8
:109A80006EE170E10E945A0964E670E080E090E0C7
:109A90000E945681CE01019684CD6DEB76E0CE0119
:109AA0004C960E94AF7DBE01645E7F4FCE01019651
:109AB0000E94FA7B182FCE014C960E94107D112334
:109AC00079F041E050E0BE016F5F7F4FCE014C96D0
:109AD0000E94B11ECE014C960E94617B8B01BECFCD
:109AE000CE0101960E94617B8B01BCCF6CE679E0D0
:109AF000CE0101960E949D7DBE016F5F7F4FCE011A
:109B00008E960E94FA7B182FCE0101960E94107D3E
:109B1000112309F4AAC063E476E0CE0101960E9405
:109B2000AF7D46E050E0BE016F5F7F4FCE018E9665
:109B30000E945BA58C01CE0101960E94107D9801C8
:109B400046E050E0BE01625D7F4FCE0101960E946B
:109B5000C47DCE0101960E94617B6B01CE0101960E
:109B60000E94107D6DE174E0CE0101960E94AF7DF0
:109B7000A8014F5F5F4FBE01625D7F4FCE014C96E3
:109B80000E94B11EBE01645E7F4FCE0101960E940D
:109B9000D77CCE014C960E94107D62E075E0CE012C
:109BA0004C960E94AF7DBE01645E7F4FCE01019650
:109BB0000E94FA7B182FCE014C960E94107D112333
:109BC00021F141E050E0BE016F5F7F4FCE014C9626
:109BD0000E94B11ECE014C960E94617B8B010A5CF3
:109BE0001F4FCE014C960E94107DF6013196EE0F6C
:109BF000FF1FE25EFF4E11830083F601EE0FFF1F91
:109C0000E655F44F1183008335CF6DEB76E0CE013E
:109C10004C960E94AF7DBE01645E7F4FCE010196DF
:109C20000E94FA7B182FCE014C960E94107D1123C2
:109C300079F041E050E0BE016F5F7F4FCE014C965E
:109C40000E94B11ECE014C960E94617B8B01C9CF50
:109C5000CE0101960E94617B0091AC0B1091AD0B7F
:109C600001501109060F171FC0CF67E374E0CE0142
:109C70004C960E94AF7DBE01645E7F4FCE018E96F2
:109C80000E94FA7B11E0811115C064E376E0CE01F9
:109C900001960E94AF7DBE016F5F7F4FCE018E9611
:109CA0000E94FA7B11E0811101C010E0CE01019603
:109CB0000E94107DCE014C960E94107D112309F464
:109CC00011C260E476E0CE014C960E94AF7D6BE35A
:109CD00076E0CE0101960E94AF7DAE01445E5F4FFB
:109CE000BE016F5F7F4FCE018E960E9462A4CE01AF
:109CF00001960E94107DCE014C960E94107D60E47A
:109D000076E0CE014C960E94AF7D6DE376E0CE0109
:109D100001960E94AF7DAE01445E5F4FBE016F5F52
:109D20007F4FCE018E960E9462A4CE0101960E94C2
:109D3000107DCE014C960E94107D60E476E0CE014D
:109D40004C960E94AF7D6FE376E0CE0101960E94B3
:109D5000AF7DAE01445E5F4FBE016F5F7F4FCE01AE
:109D60008E960E9462A4CE0101960E94107DCE01C3
:109D70004C960E94107D63E476E0CE014C960E94E2
:109D8000AF7D62E476E0CE0101960E94AF7DAE0128
:109D9000445E5F4FBE016F5F7F4FCE018E960E9483
:109DA00062A4CE0101960E94107DCE014C960E94C5
:109DB000107D63E476E0CE014C960E94AF7D6CE6A8
:109DC00078E0CE0101960E94AF7DAE01445E5F4F08
:109DD000BE016F5F7F4FCE018E960E9462A4CE01BE
:109DE00001960E94107DCE014C960E94107DCE01FE
:109DF0008E960E946C7B0E947D886093F30B70931B
:109E0000F40B8093F50B9093F60B56E0E52EF12CB6
:109E100064E6462E512C612C712C22242394312C83
:109E20005701B3E0AB0EB11C8AA99BA90197A816F4
:109E3000B90608F02AC9B701CE018E960E94C97BE7
:109E4000682FCE014C960E947B7D6701E2E0CE0E2A
:109E5000D11CFFEFEF1AFF0A9601A701BE01625D58
:109E60007F4FCE0101960E94C47DCE0101960E94D3
:109E7000617B8B01CE0101960E94107D013011059E
:109E800021F400913811109139110330110521F49A
:109E900000913A1110913B1160E476E0CE010196F9
:109EA0000E94AF7DA601BE016F5F7F4FCE018E96EF
:109EB0000E945BA56C01CE0101960E94107D6DE1B0
:109EC00074E0CE0101960E94AF7D480181E0881ABE
:109ED00091081C141D042CF59601A501BE01625DBC
:109EE0007F4FCE0182960E94C47DBE016E5D7F4F82
:109EF000CE0101960E94D77CCE0182960E94107DF1
:109F000093E08916910420F17601AFEFEA1AFA0A7C
:109F1000CE0101960E94107DCE014C960E94107DCC
:109F20007FCFA501BE01625D7F4FCE0182960E9468
:109F3000B11EBE016E5D7F4FCE0101960E94D77C9F
:109F4000CE0182960E94107DB3E08B16910400F73B
:109F500070E060E0CE014C960E94C97B823509F02A
:109F600061C0CE0101960E94617B672B682B692B33
:109F7000B1F4F801EE0FFF1FE952FD4F118210827C
:109F8000F801EE0FFF1FEE0FFF1FE154FD4F82E0BF
:109F900090E0A0E0B0E080839183A283B383CE0100
:109FA00001960E94617B6130710581059105A9F5DB
:109FB000F801EE0FFF1FE952FD4F31822082000FA2
:109FC000111F000F111FF801E154FD4F8081918195
:109FD000A281B381181619061A061B0624F04082C6
:109FE000518262827382CE0101960E94617B62304F
:109FF0007105810591053CF0F801E154FD4F608346
:10A000007183828393830E947D8801521D4FD80102
:10A010006D937D938D939C9313971C141D040CF4E6
:10A0200073CF76CF8634E9F5CE0101960E94617B2D
:10A03000672B682B692B39F4F801EE0FFF1FEC5AE0
:10A04000FD4F11821082CE0101960E94617B61302A
:10A0500071058105910539F4F801EE0FFF1FEC5AE7
:10A06000FD4F31822082000F111F000F111FF801D8
:10A07000E154FD4F80819181A281B38118161906A8
:10A080001A061B0624F040825182628273820E946B
:10A090007D8801521D4FF801608371838283938311
:10A0A000BCCF843461F4CE0101960E94617B000F25
:10A0B000111F000F111FF801EC5BFD4FA0CF84357D
:10A0C00009F0ABCFCE0101960E94617B000F111FFA
:10A0D000000F111FF801E154FD4F608371838283EB
:10A0E0009383D5CF66E679E0CE0101960E949D7DEF
:10A0F000BE016F5F7F4FCE018E960E94FA7B182FB4
:10A10000CE0101960E94107D112309F49DC045E007
:10A1100050E067E97FE0CE0101960E94B11EBE01CA
:10A120006F5F7F4F83E79FE00E94D77CCE0101964F
:10A130000E94107D83E79FE00E946C7B60E083E7D4
:10A140009FE00E94687C64E075E0CE014C960E941E
:10A15000AF7D63E77FE0CE0101960E94A67DAE0150
:10A160004E5D5F4FBE01645E7F4FCE0101960E943F
:10A1700077A5182FCE0101960E94107DCE014C9636
:10A180000E94107D112311F40C9445488E010E5D40
:10A190001F4F58E4A52E51E1B52E60E4C62E62E0B3
:10A1A000D62EF12CE12CD8016D918D01F501619332
:10A1B0005F01D6016D936D01CE0101960E94EAA365
:10A1C000CE0101960E94121BCE0101960E94107DC5
:10A1D000B3E0EB16F10471F064E075E0CE01019696
:10A1E0000E94AF7DCE0101960E94121BCE01019606
:10A1F0000E94107DEFEFEE1AFE0AF4E0EF16F10474
:10A2000091F66DE174E0CE0101960E94AF7DCE0122
:10A2100001960E94FB1ACE0101960E94107D6EE10C
:10A2200070E180916602909167020E945A0964E68B
:10A2300070E080E090E00E9456816EE479E0CE010B
:10A2400001960E949D7D46CA69E479E0CE0101969F
:10A250000E949D7DBE016F5F7F4FCE018E960E9452
:10A26000FA7B182FCE0101960E94107D112309F46C
:10A270007CC044E050E067E97FE0CE0101960E9497
:10A28000B11EBE016F5F7F4F83E79FE00E94D77CC6
:10A29000CE0101960E94107D83E79FE00E946C7BB7
:10A2A00060E083E79FE00E94687C4091770F5091C7
:10A2B000780F6AE97BE083E79FE00E94AC7864E076
:10A2C00075E0CE014C960E94AF7D63E77FE0CE0142
:10A2D00001960E94A67DAE014E5D5F4FBE01645E99
:10A2E0007F4FCE0101960E9477A5182FCE010196CF
:10A2F0000E94107DCE014C960E94107D112311F416
:10A300000C9445488E010E5D1F4F4AE4E42E40E157
:10A31000F42E6E0186E2C80ED11CD8016D918D011C
:10A32000F70161937F01CE0101960E94EAA3CE015D
:10A3300001960E94FB1ACE0101960E94107DC01664
:10A34000D10659F784EF91E09093670280936602FB
:10A350006EE170E10E945A0964E670E080E090E0EE
:10A360000E9456816EE379E06ACF67E379E0CE011F
:10A3700001960E949D7DBE016F5F7F4FCE018E963C
:10A380000E94FA7B182FCE0101960E94107D1123A6
:10A39000F1F146E050E067E97FE0CE0101960E94CE
:10A3A000B11EBE016F5F7F4F83E79FE00E94D77CA5
:10A3B000CE0101960E94107D83E79FE00E946C7B96
:10A3C0008091770F9091780F892B11F40C94454868
:10A3D00083E79FE00E94617B709347116093461171
:10A3E00070933F0260933E0284EF91E09093670286
:10A3F000809366026EE170E10E945A0964E670E0A3
:10A4000080E090E00E94568163E279E018CF6CE131
:10A4100079E0CE0101960E949D7DBE016F5F7F4F66
:10A42000CE018E960E94FA7B182FCE0101960E94D3
:10A43000107D1123B9F06FE079E0CE0101960E9402
:10A440009D7D44E650E06FEF7FEFCE0101960E94C4
:10A45000300ACE0101960E94107DF0E0E0E01995EF
:10A460000C94454867E079E0CE0101960E949D7DFD
:10A47000BE016F5F7F4FCE018E960E94FA7B182F30
:10A48000CE0101960E94107D112301F165E476E072
:10A49000CE0101960E94AF7D64E671E1CE01019686
:10A4A0000E942B7CBC0189E79FE00E94C07CCE010A
:10A4B00001960E94107D69E77FE0CE0101960E941F
:10A4C000A67DCE0101960E94FB1A8DC460E079E062
:10A4D000CE0101960E949D7DBE016F5F7F4FCE0130
:10A4E0008E960E94FA7B182FCE0101960E94107D55
:10A4F000112369F061EF78E089E79FE00E949B7C7F
:10A500006AE671E189E79FE00E94947CD4CF60E520
:10A5100076E0CE0101960E94AF7DBE016F5F7F4F56
:10A52000CE018E960E94FA7B182FCE0101960E94D2
:10A53000107D112331F00E94A53010923D020C9441
:10A54000454869E576E0CE014C960E94AF7DBE019C
:10A55000645E7F4F87E99FE00E94FA7B11E08111E2
:10A5600015C06EE576E0CE0101960E94AF7DBE017A
:10A570006F5F7F4F87E99FE00E94FA7B11E08111B6
:10A5800001C010E0CE0101960E94107DCE014C96D4
:10A590000E94107D112309F441C063E476E0CE01EE
:10A5A00001960E94AF7D40919B0F50919C0F8D8131
:10A5B0009E81481B590BBE016F5F7F4F87E99FE06B
:10A5C0000E9414A4AC014F5F5F4F67E97FE0CE01AA
:10A5D0004C960E94B11EBE01645E7F4F83E79FE0F0
:10A5E0000E94D77CCE014C960E94107DCE01019630
:10A5F0000E94107D83E79FE00E94617B61157105D9
:10A6000031F481E08093F0020E94909796CF613000
:10A61000710509F092CF1092F002F6CF63E676E072
:10A62000CE0101960E94AF7DBE016F5F7F4FCE01CC
:10A630008E960E94FA7B182FCE0101960E94107D03
:10A64000112309F43BC143E050E067E97FE0CE010C
:10A6500001960E94B11EBE016F5F7F4F83E79FE0AE
:10A660000E94D77CCE0101960E94107D63E77FE0B7
:10A67000CE0101960E94A67DCE0101960E9467211F
:10A68000CE0101960E94107D84EF91E090936702C5
:10A690008093660263E77FE0CE0101960E94A67D6B
:10A6A00060E0CE0101960E947C7CBC0180E791E1D4
:10A6B0000E94C07CCE0101960E94107D63E77FE07E
:10A6C000CE0101960E94A67D60E0CE0101960E9417
:10A6D0007C7CBC018AE691E10E94C07CCE0101969F
:10A6E0000E94107D40917411509175116EED70E1D2
:10A6F00080E791E10E94AC7840916E1150916F110A
:10A7000069EE70E18AE691E10E94AC786EE170E159
:10A7100080916602909167020E945A0967E676E08E
:10A72000CE0101960E94AF7D63E77FE0CE010196E6
:10A730000E942B7CBC01CE0182960E94A67DCE0198
:10A7400001960E94107D8091DA109091DB10892B88
:10A7500039F4BE016E5D7F4F88E89CE00E94D17E97
:10A7600068EB7BE080E090E00E9456818091DA10F7
:10A770009091DB10029709F087C063E77FE0CE017C
:10A7800088960E94A67D6FE676E0CE0101960E9433
:10A79000AF7DCE0101960E94BC97CE0101960E942A
:10A7A000107D64EF71E080E090E00E94568162E7E6
:10A7B00076E0CE0101960E94AF7DCE0101960E9407
:10A7C000BC97CE0101960E94107D6CED75E080E093
:10A7D00090E00E9456816BE776E0CE0101960E94E0
:10A7E000AF7DCE0101960E94BC97CE0101960E94DA
:10A7F000107D64EF71E080E090E00E94568169E88E
:10A8000076E0CE0101960E94AF7DCE0101960E94B6
:10A81000BC97CE0101960E94107D64EF71E080E04C
:10A8200090E00E94568167E676E0CE0101960E9494
:10A83000AF7DBE01685D7F4FCE0101960E942B7CEB
:10A84000BC01CE014C960E94A67DCE0101960E94CD
:10A85000107DCE014C960E946C7BBE01645E7F4FE2
:10A86000CE0101960E94A67DCE0101960E94BC9762
:10A87000CE0101960E94107DCE014C960E94107D63
:10A88000CE0188960E94107D68EB7BE080E090E02E
:10A890000E9456816EED70E1CE0101960E94AF7D5F
:10A8A000CE0101960E946721CE0101960E94107D83
:10A8B00010923D02CE0182960C94D14A67E976E06F
:10A8C000CE0101960E94AF7DBE016F5F7F4FCE012A
:10A8D0008E960E94FA7B182FCE0101960E94107D61
:10A8E000112309F486C044E050E067E97FE0CE011F
:10A8F00001960E94B11EBE016F5F7F4F83E79FE00C
:10A900000E94D77CCE0101960E94107D6CE976E012
:10A91000CE0101960E94AF7D63E77FE0CE010196F4
:10A920000E942B7CBC01CE014C960E94A67DCE01DC
:10A9300001960E94107D8091DA109091DB10892B96
:10A9400039F4BE01645E7F4F88E89CE00E94D17EAE
:10A9500068E873E180E090E00E9456818091DA100F
:10A960009091DB10029759F563EA76E0CE010196EB
:10A970000E94AF7D8091770F9091780F892B19F508
:10A980006CEA76E0CE0101960E94F37ABE01645E25
:10A990007F4FCE0182960E94A67DCE0182960E94B4
:10A9A000BC97CE0182960E94107D68E873E180E03A
:10A9B00090E00E945681CE0101960E94107D109277
:10A9C0003D020C94CF4ABE016F5F7F4FCE0182964D
:10A9D0000E94A67DCE0182960E94BC97CE018296EF
:10A9E0000E94107D60E777E180E090E00E94568150
:10A9F000CDCF65EB76E0CE0101960E94AF7DBE0122
:10AA00006F5F7F4FCE018E960E94FA7B182FCE018A
:10AA100001960E94107D112309F475C067E97FE05B
:10AA200083E79FE00E94C07C81E080933D0267E95C
:10AA30007FE0CE0101960E94A67DCE0101960E9484
:10AA40006721CE0101960E94107D8091DA109091CD
:10AA5000DB10029709F163E77FE088E89CE00E9441
:10AA6000D17E68EB7BE080E090E00E945681CE01D1
:10AA700001960E945598BE016F5F7F4F87E99FE066
:10AA80000E94D77CCE0101960E94107D60ED77E098
:10AA900080E090E00E9456818091DA109091DB1066
:10AAA000029771F463E77FE0CE0101960E94A67DD4
:10AAB000CE0101960E94BC97CE0101960E94107DA6
:10AAC00080919B0F90919C0F892B09F436CD68ECF7
:10AAD00077E0CE0101960E94AF7D67E97FE0CE016D
:10AAE00001960E942B7CBC01CE014C960E94A67D53
:10AAF000CE014C960E94FB1ACE014C960E94107D0E
:10AB0000CE01019650C269EB76E0CE0101960E941B
:10AB1000AF7DBE016F5F7F4FCE018E960E94FA7BA4
:10AB2000182FCE0101960E94107D112309F495C1C2
:10AB30008091DA109091DB10019709F0FECC6FEB59
:10AB400076E0CE0188960E94AF7DBE01685D7F4FA2
:10AB500088E89CE00E94D17E6CE271E080E090E0A9
:10AB60000E945681CE0182960E94559864E670E05C
:10AB700080E090E00E94568110E000E025E0C22EC7
:10AB8000D12C3AE0A32EB12C6AEC76E0CE010196EE
:10AB90000E94AF7D50E040E0BE016F5F7F4FCE016D
:10ABA00082960E945BA57C01CE0101960E94107DD9
:10ABB000A7014F5F5F4FBE016E5D7F4FCE010196D3
:10ABC0000E94B11EBE016F5F7F4FCE0188960E942A
:10ABD000D77CCE0101960E94107D8CA59DA5892B66
:10ABE00009F170E060E0CE0188960E94C97B082ED2
:10ABF000000C990BC0970A97A8F46CEC76E0CE0194
:10AC000001960E94AF7DBE016F5F7F4FCE01889697
:10AC10000E94FA7BE82ECE0101960E94107DFF244F
:10AC2000F394E110F12C60E977E0CE0101960E94E7
:10AC30009D7D64E170E0CE0101960E9431A6CE01B7
:10AC400001960E94107D0F5F1F4F62E370E080E06D
:10AC500090E00E945681C801B6010E945AB2019745
:10AC6000C1F4CE0101960E9400238D819E81892B23
:10AC700009F4BEC0BE016F5F7F4F87E99FE00E946D
:10AC8000C07C0E942C47FF24F394CE0101960E94C1
:10AC9000107DCE0101960E945598BE016F5F7F4FD7
:10ACA000CE0182960E94D77CCE0101960E94107D33
:10ACB00062E370E080E090E00E9456810436110566
:10ACC00019F0FF2009F460CF80916D0B8823F1F01B
:10ACD00068EC77E0CE014C960E94AF7DBE01685DC6
:10ACE0007F4FCE014C960E942B7CBC01CE01019679
:10ACF0000E94A67DCE0101960E94FB1ACE0101960C
:10AD00000E94107DCE014C960E94107D8CA59DA5C1
:10AD1000892B69F070E060E0CE0188960E94C97BC3
:10AD2000082E000C990BC0970A9708F47AC064EDBE
:10AD300076E0CE0101960E94AF7DCE0182960E9400
:10AD4000107DCE0188960E94107D8D819E81009796
:10AD500009F449C0E981FA812081222309F443C022
:10AD6000079708F440C068EE78E0CE014C960E9448
:10AD70009D7D68EC70E0CE014C960E9431A6CE011C
:10AD80004C960E94107DBE016F5F7F4FCE014C96A6
:10AD90000E94A67D40ED57E06FEF7FEFCE014C960D
:10ADA0000E94300ACE014C960E94107D60EE76E043
:10ADB000CE014C960E94AF7D67E97FE0CE014C96B4
:10ADC0000E942B7CBC01CE0182960E94A67DCE0102
:10ADD00082960E94FB1ACE0182960E94107DCE01BF
:10ADE0004C960E94107DCE0101960E94107DA5CB4D
:10ADF000043111050CF449CFC801B5010E945AB2C3
:10AE0000892B09F042CFBE01685D7F4F88E89CE046
:10AE10000E94D17E68EC70E080E090E00E94568154
:10AE200034CF6CEC76E0CE0101960E94AF7DBE017E
:10AE30006F5F7F4FCE0188960E94FA7B182FCE015C
:10AE400001960E94107D111172CFBE01685D7F4F87
:10AE5000CE0101960E94947D70CF6EEE76E0CE0119
:10AE600001960E94AF7DBE016F5F7F4FCE018E962F
:10AE70000E94FA7B182FCE0101960E94107D1123AB
:10AE800009F4EAC025E030E044E050E067E97FE003
:10AE9000CE0101960E94C47DBE016F5F7F4F83E7A4
:10AEA0009FE00E94D77CCE0101960E94107D67E949
:10AEB0007FE0CE0101960E94A67DCE0101960E9400
:10AEC0006721CE0101960E94107D83E79FE00E94DA
:10AED000617B6130710509F069C07093DB1060938C
:10AEE000DA106FEB77E0CE0101960E949D7DCE01D6
:10AEF00001960E946721CE0101960E94107D63EFAA
:10AF000076E0CE014C960E94AF7D6AE671E1CE01FB
:10AF10004C960E942B7CBC01CE0101960E94A67D1E
:10AF200048EC50E06FEF7FEFCE0101960E94C426FF
:10AF3000CE0101960E94107DCE014C960E94107D9C
:10AF40000E94CDA340E052EC61E070E088E89CE014
:10AF50000E94907784EF91E090936702809366025D
:10AF60006EE170E10E945A0962E077E0CE014C96F2
:10AF70000E94AF7D64E671E1CE014C960E942B7C6D
:10AF8000BC01CE0101960E94A67D40ED57E06FEF17
:10AF90007FEFCE0101960E94300ACE0101960E94F9
:10AFA000107DCE014C960E94107DC7CA61157105B7
:10AFB000D1F51092DB101092DA1061EB77E0CE0140
:10AFC00001960E949D7DCE0101960E946721CE01CF
:10AFD00001960E94107D69EF76E0CE014C960E94AA
:10AFE000AF7D6AE671E1CE014C960E942B7CBC01DC
:10AFF000CE0101960E94A67D48EC50E06FEF7FEFF6
:10B00000CE0101960E94C426CE0101960E94107DB9
:10B01000CE014C960E94107D0E94CDA340E855E2DF
:10B0200060E070E093CF6230710509F086CA7093DA
:10B03000DB106093DA1060EA77E0CE0101960E949F
:10B040009D7DCE0101960E946721CE0101960E944E
:10B05000107D6DEF76E0C1CF67E077E0CE0101961D
:10B060000E94AF7DBE016F5F7F4FCE018E960E9422
:10B07000FA7B182FCE0101960E94107D112309F44E
:10B0800041C047E050E067E97FE0CE0101960E94B1
:10B09000B11EBE016F5F7F4F83E79FE00E94D77CA8
:10B0A000CE0101960E94107D62ED76E0CE01019600
:10B0B0000E94AF7DBE016F5F7F4F83E79FE00E94DC
:10B0C000FA7B182FCE0101960E94107D111110926B
:10B0D0004F0C66ED74E0CE0101960E94AF7DBE017B
:10B0E0006F5F7F4F83E79FE00E94FA7B182FCE01AE
:10B0F00001960E94107D112309F4E9CC81E0809330
:10B100004F0CE5CC6FE077E0CE0101960E94AF7D59
:10B11000BE016F5F7F4FCE018E960E94FA7B182F83
:10B12000CE0101960E94107D112381F146E050E08E
:10B1300067E97FE0CE0101960E94B11EBE016F5FFC
:10B140007F4F83E79FE00E94D77CCE0101960E944B
:10B15000107D83E79FE00E94567B609322117093DD
:10B160002311809324119093251184EF91E0909303
:10B170006702809366026EE170E10E945A0964E6FC
:10B1800070E080E090E00E945681A1CC66E177E01B
:10B19000CE0101960E94AF7DBE016F5F7F4FCE0151
:10B1A0008E960E94FA7B182FCE0101960E94107D88
:10B1B000112301F148E050E067E97FE0CE010196FC
:10B1C0000E94B11EBE016F5F7F4F83E79FE00E9428
:10B1D000D77CCE0101960E94107D83E79FE00E94FC
:10B1E000567B609328117093291180932A119093B4
:10B1F0002B11BBCF6FE177E0CE0101960E94AF7DAE
:10B20000BE016F5F7F4FCE018E960E94FA7B182F92
:10B21000CE0101960E94107D112301F149E050E01A
:10B2200067E97FE0CE0101960E94B11EBE016F5F0B
:10B230007F4F83E79FE00E94D77CCE0101960E945A
:10B24000107D83E79FE00E94567B60932C117093E2
:10B250002D1180932E1190932F1187CF69E277E003
:10B26000CE0101960E94AF7DBE016F5F7F4FCE0180
:10B270008E960E94FA7B182FCE0101960E94107DB7
:10B280001123F1F049E050E067E97FE0CE0101963B
:10B290000E94B11EBE016F5F7F4F83E79FE00E9457
:10B2A000D77CCE0101960E94107D83E79FE00E942B
:10B2B000567B0E940EB2709333116093321155CFBA
:10B2C00063E377E0CE0101960E94AF7DBE016F5F20
:10B2D0007F4FCE018E960E94FA7B182FCE010196E9
:10B2E0000E94107D1123F1F04AE050E067E97FE011
:10B2F000CE0101960E94B11EBE016F5F7F4F83E7B2
:10B300009FE00E94D77CCE0101960E94107D83E7CA
:10B310009FE00E94567B0E940EB2709331116093A1
:10B32000301123CF6EE377E0CE0101960E94AF7D0E
:10B33000BE016F5F7F4FCE018E960E94FA7B182F61
:10B34000CE0101960E94107D112311F14BE050E0D7
:10B3500067E97FE0CE0101960E94B11EBE016F5FDA
:10B360007F4F83E79FE00E94D77CCE0101960E9429
:10B37000107D83E79FE00E94567B0E940EB260938F
:10B380003411709335118093361190933711EDCEAF
:10B390006AE477E0CE0101960E94AF7DBE016F5F47
:10B3A0007F4FCE018E960E94FA7B182FCE01019618
:10B3B0000E94107D1123E1F045E050E067E97FE055
:10B3C000CE0101960E94B11EBE016F5F7F4F83E7E1
:10B3D0009FE00E94D77CCE0101960E94107D83E7FA
:10B3E0009FE00E94617B7093271160932611BDCE70
:10B3F00060E577E0CE0101960E94AF7DBE016F5FF0
:10B400007F4FCE018E960E94FA7B182FCE010196B7
:10B410000E94107D112359F00E947D886093F30BE8
:10B420007093F40B8093F50B9093F60B86C866E54A
:10B4300077E0CE0101960E94AF7DBE016F5F7F4F26
:10B44000CE018E960E94FA7B182FCE0101960E94A3
:10B45000107D112389F143E050E0BE01625D7F4F12
:10B46000CE0101960E94B11EBE016F5F7F4F83E740
:10B470009FE00E94D77CCE0101960E94107D8091B2
:10B48000770F9091780F892B41F083E79FE00E941E
:10B49000617B70936D0260936C0280916C0290915D
:10B4A0006D020197029708F412CB81E090E090932F
:10B4B0006D0280936C020BCB67E377E0CE014C9674
:10B4C0000E94AF7DBE01645E7F4FCE018E960E94CA
:10B4D000FA7B11E0811115C06DE977E0CE0101968C
:10B4E0000E94AF7DBE016F5F7F4FCE018E960E949E
:10B4F000FA7B11E0811101C010E0CE0101960E949B
:10B50000107DCE014C960E94107D112309F468C075
:10B5100067E377E0CE0101960E94AF7DBE016F5FC9
:10B520007F4FCE018E960E94FA7B182FCE01019696
:10B530000E94107D1123A1F046E050E0BE01625D43
:10B540007F4FCE0101960E94B11EBE016F5F7F4FFB
:10B5500083E79FE00E94D77CCE0101960E94107D78
:10B560006DE977E0CE0101960E94AF7DBE016F5F6D
:10B570007F4FCE018E960E94FA7B182FCE01019646
:10B580000E94107D1123A1F042E050E0BE01625DF7
:10B590007F4FCE0101960E94B11EBE016F5F7F4FAB
:10B5A00083E79FE00E94D77CCE0101960E94107D28
:10B5B0008091770F9091780F892B09F488CA63E7FF
:10B5C0007FE0CE0101960E94A67D61E070E0CE0191
:10B5D00001960E941437CE0101960E94107D77CA11
:10B5E00063E677E0CE0182960E94AF7DBE016E5D7C
:10B5F0007F4FCE018E960E94FA7B11E0811129C007
:10B600006AE577E0CE014C960E94AF7DBE01645E94
:10B610007F4FCE018E960E94FA7B11E0811115C0FA
:10B6200062E677E0CE0101960E94AF7DBE016F5FBA
:10B630007F4FCE018E960E94FA7B11E0811101C0EE
:10B6400010E0CE0101960E94107DCE014C960E9422
:10B65000107DCE0182960E94107D112309F4E6C070
:10B6600063E677E0CE0101960E94AF7DBE016F5F79
:10B670007F4FCE018E960E94FA7B182FCE01019645
:10B680000E94107D112309F466C046E050E0BE011F
:10B69000625D7F4FCE0101960E94B11EBE016F5FB9
:10B6A0007F4F83E79FE00E94D77CCE0101960E94E6
:10B6B000107D83E79FE00E94567B6B017C0120E0B8
:10B6C00030E0A9010E9444B218160CF08EC0A70108
:10B6D000960160E070E08AE794E40E949CB10E94C9
:10B6E0000EB26093390270933A0280933B029093BA
:10B6F0003C028091390290913A02A0913B02B091B4
:10B700003C02181619061A061B0664F081E090E048
:10B71000A0E0B0E08093390290933A02A0933B02FC
:10B72000B0933C0280916C0290916D028130910542
:10B7300009F068C08091390290913A02A0913B02D1
:10B74000B0913C028093350290933602A093370269
:10B75000B0933802BCC947E050E0BE01625D7F4F44
:10B76000CE0101960E94B11EBE016F5F7F4F83E73D
:10B770009FE00E94D77CCE0101960E94107D6EE76B
:10B7800074E0CE0101960E94AF7DBE016F5F7F4FD6
:10B79000CE018E960E94FA7B182FCE0101960E9450
:10B7A000107D112331F081E090E090936D02809341
:10B7B0006C0260E776E0CE0101960E94AF7DBE018B
:10B7C0006F5F7F4FCE018E960E94FA7B182FCE01BD
:10B7D00001960E94107D112309F46BCF82E090E066
:10B7E00090936D0280936C0264CF81E090E0A0E0C2
:10B7F000B0E08093390290933A02A0933B02B09359
:10B800003C0277CF029709F062C98091390290918A
:10B810003A02A0913B02B0913C0280933102909396
:10B820003202A0933302B093340251C96AE677E042
:10B83000CE014C960E94AF7DBE01645E7F4FCE016B
:10B840008E960E94DA7B11E0811115C06FE677E0D9
:10B85000CE0101960E94AF7DBE016F5F7F4FCE018A
:10B860008E960E94FA7B11E0811101C010E0CE019A
:10B8700001960E94107DCE014C960E94107D1123EE
:10B8800009F48DC268EF77E0CE0101960E94AF7D8A
:10B89000BE016F5F7F4FCE018E960E94FA7B182FFC
:10B8A000CE0101960E94107D112309F4FBC001E036
:10B8B00010E010936D0200936C0210935D020093F0
:10B8C0005C026AEA75E083E79FE00E94F37A1093D6
:10B8D0005D0200935C0281E090E0A0E0B0E0809324
:10B8E000390290933A02A0933B02B0933C028093BA
:10B8F000350290933602A0933702B093380263E783
:10B900007FE0CE0101960E94A67D62E070E0CE014C
:10B9100001960E941437CE0101960E94107D67EDBA
:10B9200078E0CE0101960E949D7DCE0101960E9495
:10B93000FB1ACE0101960E94107D67EC78E0CE01E3
:10B9400001960E949D7DCE0101960E949927CE010D
:10B9500001960E94107D62ED76E083E79FE00E94F1
:10B96000F37A63E77FE0CE0101960E94A67D63E053
:10B9700070E0CE0101960E941437CE0101960E941C
:10B98000107D82E090E090936D0280936C0266EBF4
:10B9900078E0CE0101960E949D7DCE0101960E9425
:10B9A000FB1ACE0101960E94107D6AEA78E0CE0172
:10B9B00001960E949D7DCE0101960E949927CE019D
:10B9C00001960E94107D6AEA75E083E79FE00E947D
:10B9D000F37A809144119091451197FF06C066E774
:10B9E00077E083E79FE00E94F37A63E77FE0CE0190
:10B9F00001960E94A67D62E070E0CE0101960E9451
:10BA00001437CE0101960E94107D62ED76E083E747
:10BA10009FE00E94F37A82E090E090936D02809321
:10BA20006C0263E77FE0CE0101960E94A67D63E091
:10BA300070E0CE0101960E941437CE0101960E945B
:10BA4000107D84EF91E090936702809366026EE12F
:10BA500070E10E945A0964E670E080E090E00E9484
:10BA6000568181E090E090936D0280936C02109279
:10BA7000DA021092D90282E090E0A0E0B0E0809378
:10BA8000C3029093C402A093C502B093C6020E9461
:10BA90007D886093E3027093E4028093E5029093C3
:10BAA000E60215C86AE677E0CE0101960E94AF7DF6
:10BAB000BE016F5F7F4FCE018E960E94FA7B182FDA
:10BAC000CE0101960E94107D11110C9467556EE70E
:10BAD00074E0CE0101960E94AF7DBE016F5F7F4F83
:10BAE000CE018E960E94FA7B182FCE0101960E94FD
:10BAF000107D112331F081E090E090936D028093EE
:10BB00006C0260E776E0CE0101960E94AF7DBE0137
:10BB10006F5F7F4FCE018E960E94FA7B182FCE0169
:10BB200001960E94107D112331F082E090E0909305
:10BB30006D0280936C0281E090E0A0E0B0E0809321
:10BB4000390290933A02A0933B02B0933C02809159
:10BB50006C0290916D028130910509F099C090932B
:10BB60005D0280935C026FE677E0CE0101960E9451
:10BB7000AF7DBE016F5F7F4FCE018E960E94FA7B34
:10BB8000182FCE0101960E94107D112319F146E075
:10BB900050E0BE01625D7F4FCE014C960E94B11E07
:10BBA0006AE777E0CE0101960E94AF7DBE01645E38
:10BBB0007F4FCE0101960E942B7CBC0183E79FE062
:10BBC0000E94C07CCE0101960E94107DCE014C9651
:10BBD0000E94107D8091390290913A02A0913B021F
:10BBE000B0913C028093350290933602A0933702C5
:10BBF000B09338026AEA75E083E79FE00E94F37A27
:10BC000063E77FE0CE0101960E94A67D62E070E0CE
:10BC1000CE0101960E941437CE0101960E94107D3C
:10BC200069E978E0CE0101960E949D7DCE010196E2
:10BC30000E94FB1ACE0101960E94107D81E090E0E7
:10BC400090935D0280935C0262ED76E083E79FE073
:10BC50000E94F37A63E77FE0CE0101960E94A67D01
:10BC600063E070E0CE0101960E941437CE01019688
:10BC70000E94107D69E878E0CE0101960E949D7DCA
:10BC8000CE0101960E949927CE0101960E94107D57
:10BC900080916C0290916D02029711F00C9467559F
:10BCA0006AEA75E083E79FE00E94F37A809144118D
:10BCB0009091451197FF06C066E777E083E79FE024
:10BCC0000E94F37A01E010E010935D0200935C02A1
:10BCD00063E77FE0CE0101960E94A67D62E070E0FE
:10BCE000CE0101960E941437CE0101960E94107D6C
:10BCF00062ED76E083E79FE00E94F37A68E778E000
:10BD0000CE0101960E949D7DCE0101960E94FB1AF4
:10BD1000CE0101960E94107D63E77FE0CE0101967F
:10BD20000E94A67D63E070E0CE0101960E94143768
:10BD3000CE0101960E94107D6CE678E0CE0101965E
:10BD40000E949D7DCE0101960E949927CE01019609
:10BD50000E94107D8091441190914511919581959B
:10BD60009109909345118093441110935D020093C3
:10BD70005C0284EF91E090936702809366026EE12B
:10BD800070E10E945A0964E670E080E090E00E9451
:10BD9000568110936D0200936C020C9467556CE70A
:10BDA00077E0CE0188960E94AF7DBE01685D7F4F2F
:10BDB000CE018E960E94FA7B01E081113DC06DECB0
:10BDC00077E0CE0182960E94AF7DBE016E5D7F4F0F
:10BDD000CE018E960E94FA7B01E0811129C06CECA5
:10BDE00077E0CE014C960E94AF7DBE01645E7F4F2E
:10BDF000CE018E960E94FA7B01E0811115C063E8A6
:10BE000077E0CE0101960E94AF7DBE016F5F7F4F4C
:10BE1000CE018E960E94FA7B01E0811101C000E004
:10BE2000CE0101960E94107DCE014C960E94107D9D
:10BE3000CE0182960E94107DCE0188960E94107DD0
:10BE4000002309F41FC26CE777E0CE0101960E943F
:10BE5000AF7DBE016F5F7F4FCE018E960E94FA7B51
:10BE6000082FCE0101960E94107D46E050E001119E
:10BE700017C06DEC77E0CE0101960E94AF7DBE0148
:10BE80006F5F7F4FCE018E960E94FA7B082FCE0106
:10BE900001960E94107D002309F48BC042E050E01F
:10BEA000BE01625D7F4FCE0101960E94B11EBE01B0
:10BEB0006F5F7F4F83E79FE00E94D77CCE010196A2
:10BEC0000E94107D8091770F9091780F892B11F44B
:10BED0000C9467556AE777E0CE014C960E94AF7DDF
:10BEE000BE01645E7F4F83E79FE00E94FA7B811171
:10BEF00014C06CEB78E0CE0101960E94AF7DBE01CC
:10BF00006F5F7F4F83E79FE00E94FA7B11E0811112
:10BF100010E0CE0101960E94107DCE014C960E9449
:10BF2000107DC12CD12C7601112309F46AC183E75D
:10BF30009FE00E94567B6B017C0180916C02909186
:10BF40006D02019709F09FC083E79FE00E94567B36
:10BF50009B01AC016091960B7091970B8091980BAF
:10BF60009091990B0E9430B16093960B7093970B50
:10BF70008093980B9093990B8090960B9090970BD1
:10BF8000A090980BB090990B20E030E044EB53E484
:10BF9000C501B4010E9444B287FD86C020E030E0B4
:10BFA00044EB53E4C501B4010E942FB14B015C0185
:10BFB000EBCF43E050E0BE01625D7F4FCE010196C2
:10BFC0000E94B11EBE016F5F7F4F83E79FE00E941A
:10BFD000D77CCE0101960E94107D6EE774E0CE0101
:10BFE00001960E94AF7DBE016F5F7F4FCE018E969E
:10BFF0000E94FA7B082FCE0101960E94107D00233B
:10C00000B1F081E090E090936D0280936C0280919A
:10C01000E10B9091E20BA091E30BB091E40B8093C4
:10C02000960B9093970BA093980BB093990B60E7A6
:10C0300076E0CE0101960E94AF7DBE016F5F7F4F1B
:10C04000CE018E960E94FA7B082FCE0101960E94A7
:10C05000107D002309F436CF82E090E090936D02CA
:10C0600080936C028091DD0B9091DE0BA091DF0B31
:10C07000B091E00B8093960B9093970BA093980B45
:10C08000B093990B1FCF83E79FE00E94567B9B01E3
:10C09000AC016091960B7091970B8091980B9091E9
:10C0A000990B0E942FB160CF20E030E0A901C501BB
:10C0B000B4010E9482AF87FF0BC020E030E044EB68
:10C0C00053E4C501B4010E9430B14B015C01ECCFD7
:10C0D0008092960B9092970BA092980BB092990B2E
:10C0E00020E030E0A901C701B6010E9444B287FDFB
:10C0F00015C06CEB78E0CE0101960E94AF7D63E73E
:10C100007FE0CE0101960E942B7CBC0183E79FE07B
:10C110000E94C07CCE0101960E94107D20E030E09C
:10C12000A901C701B6010E9482AF87FF6AC0809152
:10C130006C0290916D02019799F520E030E0A90121
:10C14000C701B6010E9444B218160CF092C020E05C
:10C1500030E040E251E4C701B6010E9430B122E074
:10C16000AB01BC01CE014C960E94187D6AE777E0D6
:10C17000CE0101960E94AF7DBE01645E7F4FCE016D
:10C1800001960E942B7CBC0183E79FE00E94C07C4B
:10C19000CE0101960E94107DCE014C960E94107D2A
:10C1A00080916C0290916D02019759F120E030E08E
:10C1B000A901C701B6010E9444B2B701A601181631
:10C1C0000CF0705822E0CE014C960E94187D6AE770
:10C1D00077E0CE0101960E94AF7DBE01645E7F4F85
:10C1E000CE0101960E942B7CBC0183E79FE00E9458
:10C1F000C07CCE0101960E94107DCE014C960E941B
:10C20000107D81E090E090935D0280935C0263E793
:10C210007FE0CE0101960E94A67D62E070E0CE0133
:10C2200001960E941437CE0101960E94107D20E0F5
:10C2300030E0A901C701B6010E9482AF87FD02C0AC
:10C240000C94675580916C0290916D02019711F0EA
:10C250000C94675567E877E083E79FE00E94F37AE4
:10C2600063E77FE0CE0101960E94A67D62E070E068
:10C27000AEC9A701960160E070E080E291E40E94FF
:10C280002FB16DCF6CE877E0CE0182960E94AF7D32
:10C29000BE016E5D7F4FCE018E960E94FA7B11E04B
:10C2A000811129C06BE877E0CE014C960E94AF7DEA
:10C2B000BE01645E7F4FCE018E960E94FA7B11E034
:10C2C000811115C062E977E0CE0101960E94AF7D31
:10C2D000BE016F5F7F4FCE018E960E94FA7B11E008
:10C2E000811101C010E0CE0101960E94107DCE01A7
:10C2F0004C960E94107DCE0182960E94107D1123E3
:10C3000009F49BC0CE018E960E946C7B6AEA75E0B0
:10C3100083E79FE00E94F37A6EE774E0CE01019616
:10C320000E94AF7DBE016F5F7F4FCE018E960E944F
:10C33000FA7B182FCE0101960E94107D112331F057
:10C3400081E090E090936D0280936C0260E776E06C
:10C35000CE0101960E94AF7DBE016F5F7F4FCE017F
:10C360008E960E94FA7B182FCE0101960E94107DB6
:10C37000112391F082E090E090936D0280936C0223
:10C38000809144119091451197FF06C066E777E0D0
:10C3900083E79FE00E94F37A81E090E090935D0252
:10C3A00080935C0263E77FE0CE0101960E94A67D48
:10C3B00062E070E0CE0101960E941437CE01019632
:10C3C0000E94107D6CE877E0CE0101960E94AF7D5F
:10C3D000BE016F5F7F4FCE018E960E94FA7B182FB1
:10C3E000CE0101960E94107D45E050E0111102C07F
:10C3F00046E050E0BE01625D7F4FCE0101960E9493
:10C40000B11EBE016F5F7F4F83E79FE00E94D77C24
:10C41000CE0101960E94107D8091770F9091780F48
:10C42000892B11F40C94675563E77FE0CE010196E8
:10C430000E94A67D63E070E0CAC86AE977E0CE0199
:10C4400082960E94AF7DBE016E5D7F4FCE018E96BB
:10C450000E94FA7B11E0811129C069E977E0CE01E1
:10C460004C960E94AF7DBE01645E7F4FCE018E96DA
:10C470000E94FA7B11E0811115C060EA77E0CE01DD
:10C4800001960E94AF7DBE016F5F7F4FCE018E96F9
:10C490000E94FA7B11E0811101C010E0CE010196EB
:10C4A0000E94107DCE014C960E94107DCE01829696
:10C4B0000E94107D112309F426C16AE977E0CE01BC
:10C4C00001960E94AF7DBE016F5F7F4FCE018E96B9
:10C4D0000E94FA7B182FCE0101960E94107D112335
:10C4E00009F443C045E050E0BE01625D7F4FCE01DC
:10C4F00001960E94B11EBE016F5F7F4F83E79FE0F0
:10C500000E94D77CCE0101960E94107D8091770F0A
:10C510009091780F892B61F083E79FE00E94567B12
:10C520006093960B7093970B8093980B9093990B55
:10C53000C090960BD090970BE090980BF090990BD1
:10C5400020E030E044EB53E4C701B6010E9444B25E
:10C5500087FD55C020E030E044EB53E4C701B6014D
:10C560000E942FB16B017C01EBCF46E050E0BE0191
:10C57000625D7F4FCE0101960E94B11EBE016F5FCA
:10C580007F4F83E79FE00E94D77CCE0101960E94F7
:10C59000107D6EE774E0CE0101960E94AF7DBE0172
:10C5A0006F5F7F4FCE018E960E94FA7B182FCE01CF
:10C5B00001960E94107D112331F081E090E090936C
:10C5C0006D0280936C0260E776E0CE0101960E94D6
:10C5D000AF7DBE016F5F7F4FCE018E960E94FA7BCA
:10C5E000182FCE0101960E94107D112309F48ECFE1
:10C5F00082E090E090936D0280936C0287CF20E000
:10C6000030E0A901C701B6010E9482AF87FF0BC0CD
:10C6100020E030E044EB53E4C701B6010E9430B1A2
:10C620006B017C01ECCFC092960BD092970BE092FD
:10C63000980BF092990B80916C0290916D0201978A
:10C6400071F4C092E10BD092E20BE092E30BF09216
:10C65000E40B61E175E089E79FE00E94F37A809145
:10C66000960B9091970BA091980BB091990B2091FC
:10C670006C0230916D022230310571F48093DD0B34
:10C680009093DE0BA093DF0BB093E00B61E275E0BB
:10C6900089E79FE00E94F37A4091960B5091970BA7
:10C6A0006091980B7091990B21E0CE014C960E94FD
:10C6B000187D69E77FE0CE0101960E94A67DBE014C
:10C6C000645E7F4FCE0101960E942B7C6CE175E089
:10C6D0000E94157CBC0189E79FE00E94C07CCE01CE
:10C6E00001960E94107DCE014C960E94107D69E754
:10C6F0007FE0CE0101960E94A67DCE0101960E94A8
:10C7000099270C94EB5A68EA77E0CE0182960E9452
:10C71000AF7DBE016E5D7F4FCE018E960E94FA7B8B
:10C7200011E0811129C067EA77E0CE014C960E94A2
:10C73000AF7DBE01645E7F4FCE018E960E94FA7B74
:10C7400011E0811115C06DEA77E0CE0101960E94DB
:10C75000AF7DBE016F5F7F4FCE018E960E94FA7B48
:10C7600011E0811101C010E0CE0101960E94107D00
:10C77000CE014C960E94107DCE0182960E94107DC3
:10C78000112309F412C2C0903902D0903A02E0900D
:10C790003B02F0903C0263EB77E0CE0101960E94F1
:10C7A000AF7DBE016F5F7F4FCE018E960E94FA7BF8
:10C7B000182FCE0101960E94107D112309F465C047
:10C7C00044E050E0BE01625D7F4FCE0101960E94C1
:10C7D000B11EBE016F5F7F4F83E79FE00E94D77C51
:10C7E000CE0101960E94107D80916C0290916D02A5
:10C7F0008130910509F093C0C0903502D090360287
:10C80000E0903702F090380281E090E0A0E0B0E0E4
:10C810008093350290933602A0933702B09338028A
:10C820008091770F9091780F892B09F090C068EB79
:10C8300077E083E79FE00E94F37A8091770F9091F1
:10C84000780F892B81F063E77FE0CE0101960E948B
:10C85000A67D70E060E0CE0101960E941437CE0103
:10C8600001960E94107D80916C0290916D02813042
:10C87000910509F08CC1C0923502D0923602E09247
:10C880003702F09238020C94675545E050E0BE0143
:10C89000625D7F4FCE0101960E94B11EBE016F5FA7
:10C8A0007F4F83E79FE00E94D77CCE0101960E94D4
:10C8B000107D6EE774E0CE0101960E94AF7DBE014F
:10C8C0006F5F7F4FCE018E960E94FA7B182FCE01AC
:10C8D00001960E94107D112331F081E090E0909349
:10C8E0006D0280936C0260E776E0CE0101960E94B3
:10C8F000AF7DBE016F5F7F4FCE018E960E94FA7BA7
:10C90000182FCE0101960E94107D112309F46CCFDF
:10C9100082E090E090936D0280936C0265CF029765
:10C9200009F07ECFC0903102D0903202E090330205
:10C93000F090340281E090E0A0E0B0E0809331021A
:10C9400090933202A0933302B093340269CF6EEB1E
:10C9500077E0CE0101960E94AF7DBE016F5F7F4FF1
:10C9600083E79FE00E94DA7B182FCE0101960E9498
:10C97000107D112309F477CF83E79FE00E94567B57
:10C9800020E030E0A9010E9482AF811128C080918F
:10C990006C0290916D02019731F461EC77E083E7CE
:10C9A0009FE00E94F37A80916C0290916D02029751
:10C9B00031F468EB77E083E79FE00E94F37A80919F
:10C9C000770F9091780F892B09F44DCF63E77FE0C3
:10C9D000CE0101960E94A67D61E070E03CCF63E449
:10C9E00076E0CE0101960E94AF7DBE016F5F7F4F62
:10C9F00083E79FE00E94DA7B182FCE0101960E9408
:10CA0000107D112309F42FCF41E050E063E77FE070
:10CA1000CE0101960E94B11ECE0101960E94567B66
:10CA20004B015C01CE0101960E94107D20E030E0B8
:10CA3000A901C501B4010E9482AF181634F0812CFF
:10CA4000912C90E8A92E9FE3B92E00916C021091D1
:10CA50006D020130110509F075C0A501940160E077
:10CA600070E48CE995E40E949CB160932D02709370
:10CA70002E0280932F029093300260933C117093AA
:10CA80003D1180933E1190933F1160932902709362
:10CA90002A0280932B0290932C02B801CE014C966F
:10CAA0000E94FD7A66EC77E0CE0101960E94AF7D90
:10CAB000BE01645E7F4FCE0101960E942B7CBC01BB
:10CAC000CE0182960E94A67DCE0182960E94121B04
:10CAD000CE0182960E94107DCE0101960E94107DAB
:10CAE000CE014C960E94107D6AE578E0CE01019659
:10CAF0000E949D7DCE0101960E94121BCE010196DF
:10CB00000E94107D40912D0250912E0260912F02C3
:10CB10007091300225E0CE0101960E94187DCE0171
:10CB200001960E94FB1ACE0101960E94107D84EFAF
:10CB300091E090936702809366026EE170E10E943B
:10CB40005A0991CE0230110509F0A7CFA501940131
:10CB500060E070E48CE196E40E949CB160932D0249
:10CB600070932E0280932F029093300260934011B5
:10CB70007093411180934211909343116093250269
:10CB800070932602809327029093280286CF029703
:10CB900011F00C946755C0923102D0923202E092AB
:10CBA0003302F09234020C9467556BEC77E0CE01BF
:10CBB00082960E94AF7DBE016E5D7F4FCE018E9644
:10CBC0000E94FA7B11E0811129C06AEC77E0CE0166
:10CBD0004C960E94AF7DBE01645E7F4FCE018E9663
:10CBE0000E94FA7B11E0811115C060ED77E0CE0163
:10CBF00001960E94AF7DBE016F5F7F4FCE018E9682
:10CC00000E94FA7B11E0811101C010E0CE01019673
:10CC10000E94107DCE014C960E94107DCE0182961E
:10CC20000E94107D112309F429C18AA99BA90597A7
:10CC300010F40C94675544E050E0BE01625D7F4FF4
:10CC4000CE0101960E94B11EBE016F5F7F4F83E748
:10CC50009FE00E94D77CCE0101960E94107D6BEC74
:10CC600077E0CE0101960E94AF7DBE016F5F7F4FDE
:10CC7000CE018E960E94FA7B182FCE0101960E945B
:10CC8000107D112309F49BC044E050E0BE01625DB9
:10CC90007F4FCE0101960E94B11EBE016F5F7F4F94
:10CCA00083E79FE00E94D77CCE0101960E94107D11
:10CCB00083E79FE00E94567B20E030E0A9010E94BC
:10CCC00044B2181614F00C94675583E79FE00E9455
:10CCD000567B60932D0270932E0280932F029093C7
:10CCE000300220916C0230916D022130310509F043
:10CCF000B0C060933C1170933D1180933E119093AE
:10CD00003F116093290270932A0280932B02909323
:10CD10002C02B901CE014C960E94FD7A66EC77E0B8
:10CD2000CE0101960E94AF7DBE01645E7F4FCE01B1
:10CD300001960E942B7CBC01CE0182960E94A67DAA
:10CD4000CE0182960E94121BCE0182960E94107D17
:10CD5000CE0101960E94107DCE014C960E94107D5E
:10CD600068E478E0CE0101960E949D7DCE01019697
:10CD70000E94121BCE0101960E94107D40912D024F
:10CD800050912E0260912F027091300225E0CE0169
:10CD900001960E94187DCE0101960E94FB1ACE01D9
:10CDA00001960E94107D84EF91E09093670280933A
:10CDB00066026EE170E10E945A090C94675545E0E5
:10CDC00050E0BE01625D7F4FCE0101960E94B11E10
:10CDD000BE016F5F7F4F83E79FE00E94D77CCE014B
:10CDE00001960E94107D6EE774E0CE0101960E94CC
:10CDF000AF7DBE016F5F7F4FCE018E960E94FA7BA2
:10CE0000182FCE0101960E94107D112331F081E090
:10CE100090E090936D0280936C0260E776E0CE0123
:10CE200001960E94AF7DBE016F5F7F4FCE018E964F
:10CE30000E94FA7B182FCE0101960E94107D1123CB
:10CE400009F436CF82E090E090936D0280936C02FB
:10CE50002FCF2230310509F05CCF609340117093E1
:10CE60004111809342119093431160932502709376
:10CE7000260280932702909328024BCF65ED75E040
:10CE8000CE014C960E94AF7DBE01645E7F4FCE0105
:10CE90008E960E94FA7B11E0811115C066ED77E055
:10CEA000CE0101960E94AF7DBE016F5F7F4FCE0124
:10CEB0008E960E94FA7B11E0811101C010E0CE0134
:10CEC00001960E94107DCE014C960E94107D112388
:10CED00009F463C065ED75E0CE0101960E94AF7D57
:10CEE000BE016F5F7F4FCE018E960E94FA7B182F96
:10CEF000CE0101960E94107D112399F042E050E08E
:10CF000067E97FE0CE0101960E94B11EBE016F5F0E
:10CF10007F4F83E79FE00E94D77CCE0101960E945D
:10CF2000107D66ED77E0CE0101960E94AF7DBE01D7
:10CF30006F5F7F4FCE018E960E94FA7B182FCE0135
:10CF400001960E94107D112399F043E050E067E9BB
:10CF50007FE0CE0101960E94B11EBE016F5F7F4F40
:10CF600083E79FE00E94D77CCE0101960E94107D4E
:10CF700083E79FE00E94617B653B710510F40C9490
:10CF8000675565E378E0CE0101960E949D7DCE0154
:10CF900001960E94121B0C94EB5A6AED77E0CE01C9
:10CFA00001960E94AF7DBE016F5F7F4FCE018E96CE
:10CFB0000E94FA7B182FCE0101960E94107D11234A
:10CFC00009F474C026E030E044E050E067E97FE017
:10CFD000CE0101960E94C47DBE016F5F7F4F83E743
:10CFE0009FE00E94D77CCE0101960E94107D63E4F1
:10CFF00076E0CE0101960E94AF7D40919B0F50914B
:10D000009C0F8D819E81481B590BBE016F5F7F4F26
:10D0100087E99FE00E9414A4AC014F5F5F4F67E96E
:10D020007FE0CE014C960E94B11EBE01645E7F4F30
:10D0300083E79FE00E94D77CCE014C960E94107D32
:10D04000CE0101960E94107D83E79FE00E94567BEF
:10D0500088E2EEE6FBE0A5EFB0E101900D928A9543
:10D06000E1F784EF91E090936702809366026EE1AE
:10D0700070E10E945A0964E178E089E79FE00E942C
:10D080009B7C44E050E067E97FE0CE0101960E947E
:10D09000B11EBE016F5F7F4F89E79FE00E94947CC5
:10D0A000CE0101960E94107D0C945B526EED77E0EC
:10D0B000CE0101960E94AF7DBE016F5F7F4FCE0112
:10D0C0008E960E94FA7B182FCE0101960E94107D49
:10D0D00011110C94415866EE77E0CE0101960E9442
:10D0E000AF7DBE016F5F7F4FCE018E960E94FA7BAF
:10D0F000182FCE0101960E94107D112371F141E09D
:10D1000068E972E0CE0101960E94E494BE016F5F6F
:10D110007F4F82E891E10E94221E82E891E10E9405
:10D120005B0D811104C068EC77E00C941F5182E81C
:10D1300091E10E94A007892B51F082E891E10E94C1
:10D14000C50D682F85E29DE00E94AA74F0CF82E8A9
:10D1500091E10E94670D0C9445486DEE77E0CE0199
:10D1600001960E94AF7DBE016F5F7F4FCE018E960C
:10D170000E94FA7B182FCE0101960E94107D112388
:10D18000E9F08DB79EB7825391400FB6F8949EBFD9
:10D190000FBE8DBFADB7BEB7119682E391E0EEE151
:10D1A000F0E101900D920197E1F70E94C6320FB6AF
:10D1B000F894DEBF0FBECDBF0C94454866EF77E014
:10D1C000CE0101960E94AF7DBE016F5F7F4FCE0101
:10D1D0008E960E94FA7B182FCE0101960E94107D38
:10D1E000112309F457C0EDB7FEB7E253F1400FB673
:10D1F000F894FEBF0FBEEDBFADB7BEB7119682E388
:10D2000091E0EEE1F0E101900D920197E1F70E94CB
:10D21000452C0FB6F894DEBF0FBECDBF63E078E0BB
:10D22000CE0101960E949D7DADB7BEB7A253B1401D
:10D230000FB6F894BEBF0FBEADBF119682E391E06A
:10D24000EEE1F0E101900D920197E1F70E944B248D
:10D250000FB6F894DEBF0FBECDBF8DB79EB7825319
:10D2600091400FB6F8949EBF0FBE8DBFADB7BEB74D
:10D27000119682E391E0EEE1F0E101900D920197C9
:10D28000E1F70E94C6320FB6F894DEBF0FBECDBFE5
:10D290000C944A4D68EF77E0CE0101960E94AF7D75
:10D2A000BE016F5F7F4FCE018E960E94FA7B182FD2
:10D2B000CE0101960E94107D1123F9F061EF77E015
:10D2C000CE0101960E949D7DBE016F5F7F4FCE0112
:10D2D0004C960E94A67DCE014C960E94FB1ACE0170
:10D2E0004C960E94107DEDB7FEB7E253F1400FB6A9
:10D2F000F894FEBF0FBEEDBFB9CF6CEF77E0CE0163
:10D3000001960E94AF7DBE016F5F7F4FCE018E966A
:10D310000E94FA7B182FCE0101960E94107D1123E6
:10D3200009F4F5C065ED77E0CE0182960E949D7DFF
:10D33000BE016E5D7F4FCE0101960E94A67DAE01BB
:10D340004F5F5F4F62E070E08FE792E00E94F82D40
:10D35000182FCE0101960E94107D111122C0BE012E
:10D360006E5D7F4FCE014C960E94A67D60E078E016
:10D37000CE014C960E94157C6AEC7FE00E942B7CCB
:10D38000BC01CE0101960E94A67DCE0101960E94AD
:10D39000FB1ACE0101960E94107DCE014C960E9490
:10D3A000107D68EE73E080E090E00E945681BE013F
:10D3B0006E5D7F4FCE0101960E94A67DAE014F5F4C
:10D3C0005F4F63E070E082E792E00E94F82D182F33
:10D3D000CE0101960E94107D111122C0BE016E5D2A
:10D3E0007F4FCE014C960E94A67D60E178E0CE0191
:10D3F0004C960E94157C6AEC7FE00E942B7CBC015D
:10D40000CE0101960E94A67DCE0101960E94FB1AD4
:10D41000CE0101960E94107DCE014C960E94107D97
:10D4200068EE73E080E090E00E9456816EEB7FE052
:10D43000CE0101960E94A67DAE014F5F5F4F61E075
:10D4400070E082EB92E00E94F82D182FCE01019639
:10D450000E94107D111121C06EEB7FE0CE014C9631
:10D460000E94A67D60E178E0CE014C960E94157C7A
:10D470006AEC7FE00E942B7CBC01CE0101960E94E9
:10D48000A67DCE0101960E94FB1ACE0101960E9454
:10D49000107DCE014C960E94107D68EE73E080E016
:10D4A00090E00E94568180914F0C882311F40C94D7
:10D4B0005A5443E162EB72E0CE0101960E94E4947B
:10D4C000BE016F5F7F4F88EB91E10E94221E88EBC7
:10D4D00091E10E945B0D882311F40C945A546EEB79
:10D4E0007FE088EB91E10E94DF7E66E970E080E0FA
:10D4F00090E00E94568188EB91E10E94670D62E303
:10D5000070E080E090E00E9456810C945A546CE1E7
:10D5100078E0CE0101960E94AF7DBE016F5F7F4F24
:10D52000CE018E960E94FA7B182FCE0101960E94A2
:10D53000107D1123C1F00CEA1BE082EBE82E8BE09A
:10D54000F82ED8018C910E5F1F4F60E00E94E37FA0
:10D550006CE271E080E090E00E945681E016F106F6
:10D5600081F70C94454860E278E0CE0101960E9474
:10D57000AF7DBE016F5F7F4FCE018E960E94FA7B1A
:10D58000182FCE0101960E94107D1123A9F00CEAFC
:10D590001BE0F80180810E5F1F4F61E00E94E37F76
:10D5A0006CE271E080E090E00E945681FBE0023B7B
:10D5B0001F0779F70C94454865E278E0CE010196A3
:10D5C0000E94AF7DBE016F5F7F4FCE018E960E949D
:10D5D000FA7B182FCE0101960E94107D112311F4C1
:10D5E0000C94454827E030E046E050E067E97FE0F2
:10D5F000CE0101960E94C47DBE016F5F7F4F83E71D
:10D600009FE00E94D77CCE0101960E94107D83E7A7
:10D610009FE00E94617B672B71F410926D0B67E9AC
:10D620007FE0CE0101960E94A67DCE0101960E9468
:10D6300067210C94F35681E080936D0BF0CF2F920D
:10D640003F924F925F926F927F928F929F92AF9292
:10D65000BF92CF92DF92EF92FF920F931F93CF93DF
:10D66000DF9300D000D01F921F92CDB7DEB760913C
:10D670008E0270918F0280918C0290918D020E9497
:10D68000291B84E1482E512C612C712C312C212C2A
:10D690008FEF281A380AC301B2010E9456816091A7
:10D6A0008E0270918F0280918C0290918D020E9467
:10D6B000291B8C0183E02816310434F08EE12816F2
:10D6C000310444F4012B51F084E1480E511C611CDB
:10D6D000711CDECF0115110509F0A6C080918C02E6
:10D6E00090918D028B30910509F086C08090541185
:10D6F00090905511A0905611B0905711C0905011B4
:10D70000D0905111E0905211F090531164E670E006
:10D7100080E090E00E94568161E275E0CE010196C2
:10D720000E949D7DCE0101960E949927CE0101960F
:10D730000E94107D61E082E00E94418C21E0B501F1
:10D74000A401CE0101960E94187DBE016F5F7F4F3C
:10D7500084ED91E10E94D17ECE0101960E94107D60
:10D760006FED84ED91E10E94198C6CE175E084ED20
:10D7700091E10E94F37E20E0B701A601CE0101965F
:10D780000E94187DBE016F5F7F4F84ED91E10E9482
:10D79000D17ECE0101960E94107D6CE278E084ED8E
:10D7A00091E10E94C97E89829A82AB82BC82CD823D
:10D7B000DE82EF82F88629813A814B815C816D811E
:10D7C0007E818F81988528960FB6F894DEBF0FBEB4
:10D7D000CDBFDF91CF911F910F91FF90EF90DF9020
:10D7E000CF90BF90AF909F908F907F906F905F9001
:10D7F0004F903F902F9008958631910509F476CF90
:10D800000C9709F083CF8090920A9090930AA09091
:10D81000940AB090950AC0908E0AD0908F0AE0903A
:10D82000900AF090910A72CF0F3F8FEF1807CCF05B
:10D830006EE075E0CE0101960E949D7D4AE050E0C9
:10D8400070E060E0CE0101960E94C426CE010196F0
:10D850000E94107D6BEE74E089E79FE00E949B7C44
:10D8600032C00E3F8FEF1807B9F16DED74E0CE01B5
:10D8700001960E949D7D4AE050E070E060E0CE019C
:10D8800001960E94C426CE0101960E94107D6EEC86
:10D8900074E089E79FE00E949B7CB801CE0101966D
:10D8A0000E94FD7ABE016F5F7F4F89E79FE00E9473
:10D8B000947CCE0101960E94107D68EB74E089E7AC
:10D8C0009FE00E943E7C19821A821B821C821D826C
:10D8D0001E821F8218866FCF6DEA74E0CE0101961A
:10D8E0000E949D7D4AE050E070E060E0CE0101962C
:10D8F0000E94C426CE0101960E94107D6DE874E05E
:10D90000ABCF2F923F924F925F926F927F928F9206
:10D910009F92AF92BF92CF92DF92EF92FF920F93BE
:10D920001F93CF93DF93CDB7DEB7AC970FB6F894C4
:10D93000DEBF0FBECDBF8C017B018091DB0B9091D0
:10D94000DC0B01969093DC0B8093DB0B2091F80BA2
:10D95000222341F06AE070E00E945AB218161906BC
:10D960000CF4C0C281E08093F80B1092DC0B109293
:10D97000DB0B50E040E06EE174E0C8010E946C1ED9
:10D9800082E0E816F10409F4C6C26DE174E088EBA8
:10D990009FE00E94F37A60918E0270918F028091D5
:10D9A0008C0290918D020E94291B1C0163E17BE097
:10D9B000C8010E94531E6EE278E0C8010E94C97E31
:10D9C0006EE571E1CE0101960E94A67DBE016F5FFA
:10D9D0007F4FC8010E94D17ECE0101960E94107D2A
:10D9E00067E378E0C8010E94C97E68E176E0C8017B
:10D9F0000E94F37E64E671E1CE0101960E94A67D4D
:10DA0000BE016F5F7F4FC8010E94D17E6EE076E05D
:10DA1000C8010E94F37E66E770E1CE0109960E947C
:10DA2000AF7DBE01675F7F4FC8010E94D17E61E07C
:10DA300076E0C8010E94F37E6EED70E1CE010F9694
:10DA40000E94AF7DBE01615F7F4FC8010E94D17E01
:10DA50006AEF75E0C8010E94F37ECE010F960E9426
:10DA6000107DCE0109960E94107DCE0101960E9484
:10DA7000107D0E94258428EE33E040E050E00E94B3
:10DA8000CCB029013A0160EF75E0C8010E94F37E35
:10DA9000CE0101960E941422BE016F5F7F4FC80124
:10DAA0000E94D17ECE0101960E94107DC301B20179
:10DAB00020E13EE040E050E00E94EEB04B015C010E
:10DAC000B901CE0187960E94BD1E4CE3C42ED12C15
:10DAD000E12CF12CC501B401A70196010E94EEB022
:10DAE000B901CE0101960E94BD1E60E077E0CE0133
:10DAF00009960E94AF7DBE016F5F7F4FCE010996F0
:10DB00000E942B7CBC01CE0187960E94947CCE01A2
:10DB100009960E94107DCE0101960E94107DC301DE
:10DB2000B201A70196010E94EEB0CE0101960E94BB
:10DB3000BD1E60E077E0CE0109960E94AF7DBE0178
:10DB40006F5F7F4FCE0109960E942B7CBC01CE01F6
:10DB500087960E94947CCE0109960E94107DCE018A
:10DB600001960E94107D6DE378E0CE0109960E9437
:10DB7000AF7DBE01695D7F4FCE0109960E942B7C6F
:10DB800060E478E00E94157CBC01CE0101960E9401
:10DB9000A67DBE016F5F7F4FC8010E94D17ECE017E
:10DBA00001960E94107DCE0109960E94107D6EE4C0
:10DBB00078E0C8010E94C97ECE0101960E94F31947
:10DBC000B801CE0101960E946B7E69E478E0C8013D
:10DBD0000E94B57E0E941F6B29833A834B835C832E
:10DBE0006D837E838F83988749815A816B817C8185
:10DBF00021E0CE010F960E94187DBE01615F7F4F2C
:10DC0000CE0109960E94A67D66E578E0CE010996D0
:10DC10000E94157CBC0188EB9FE00E94C07CCE0175
:10DC200009960E94107DCE010F960E94107D6DE531
:10DC300078E0CE010F960E94AF7D68EB7FE0CE01C9
:10DC40000F960E942B7CBC01CE0109960E94A67DF6
:10DC5000BE01675F7F4FC8010E94D17ECE01099649
:10DC60000E94107DCE010F960E94107D4D815E8135
:10DC70006F81788521E0CE0109960E94187DBE0152
:10DC8000675F7F4F88EB9FE00E94D77CCE010996AB
:10DC90000E94107D6FE678E0CE010F960E94AF7D66
:10DCA00068EB7FE0CE010F960E942B7C60E878E065
:10DCB0000E94157CBC01CE0109960E94A67DBE0182
:10DCC000675F7F4FC8010E94D17ECE0109960E94F6
:10DCD000107DCE010F960E94107D4091E10B509176
:10DCE000E20B6091E30B7091E40B22E0CE010F9602
:10DCF0000E94187D67E878E0CE0145960E94AF7DCE
:10DD0000BE01615F7F4FCE0145960E942B7C69E981
:10DD100078E00E94157CBC01CE0109960E94A67D88
:10DD2000BE01675F7F4FC8010E94D17ECE01099678
:10DD30000E94107DCE0145960E94107DCE010F9667
:10DD40000E94107D4091DD0B5091DE0B6091DF0B46
:10DD50007091E00B22E0CE010F960E94187D62EADE
:10DD600078E0CE0145960E94AF7DBE01615F7F4F96
:10DD7000CE0145960E942B7C69E978E00E94157CD3
:10DD8000BC01CE0109960E94A67DBE01675F7F4F50
:10DD9000C8010E94D17ECE0109960E94107DCE015D
:10DDA00045960E94107DCE010F960E94107DE6EFF1
:10DDB0002E16EFEF3E062CF46EE07CE0C8010E94C8
:10DDC000531E6BEE7AE0C8010E94531E9EE1E92EBD
:10DDD00090E1F92E27EDA22E22E0B22ECC24C3949E
:10DDE000D12C4701F8E08F0E911C82E0A80EB11CE7
:10DDF00080911E1090911F108C159D050CF464C02D
:10DE0000B601CE010F960E94FD7A68EC77E0CE0154
:10DE100045960E94AF7DBE01615F7F4FCE01459662
:10DE20000E942B7C60E476E00E94157CBC01CE0150
:10DE300009960E94A67DBE01675F7F4FC8010E94C0
:10DE4000D17EB701645E7F4FCE014B960E94AF7DBD
:10DE5000BE01655E7F4FC8010E94D17E60EB78E015
:10DE6000C8010E94C97EF50160817181660F771F2C
:10DE7000660F771F665D7F4ECE0181960E94AF7D53
:10DE8000BE016F5D7F4FC8010E94D17E65EB78E0D7
:10DE9000C8010E94C97ECE0181960E94107DCE01EC
:10DEA0004B960E94107DCE0109960E94107DCE01F6
:10DEB00045960E94107DCE010F960E94107DFFEFC7
:10DEC000CF1ADF0A74018DCFCE0187960E94107D94
:10DED00081E08093520C6CEC7BE0C8010E94531EE1
:10DEE0001092F80BAC960FB6F894DEBF0FBECDBF04
:10DEF000DF91CF911F910F91FF90EF90DF90CF9026
:10DF0000BF90AF909F908F907F906F905F904F9059
:10DF10003F902F9008956EE07CE0C8010E94531E50
:10DF2000DACF8F929F92AF92BF92CF92DF92EF9211
:10DF3000FF920F931F93CF93DF93CDB7DEB7A097D8
:10DF40000FB6F894DEBF0FBECDBF6DE174E082EE78
:10DF50009FE00E94F37A6DE174E086ED9FE00E94FD
:10DF6000F37A48E4842E42E0942E5EE1C52E50E11F
:10DF7000D52E61EDA62E62E0B62E77EDE72E72E08B
:10DF8000F72E01E010E0F40181919191A191B191FE
:10DF90004F01892B8A2B8B2B19F5F70182819381F5
:10DFA000F5012081318182179307D1F0880F991FE5
:10DFB000FC01E759F44FD801AA0FBB1FA655B44F77
:10DFC00060818C910E94E37FF70182819381F5014A
:10DFD0009183808364E670E080E090E00E94568147
:10DFE000F501619171915F0180911E1090911F1058
:10DFF000801791070CF4E2C2CE0145960E94FD7A8B
:10E00000B801CE010F960E94FD7AB601645E7F4F83
:10E01000CE0109960E94AF7D60E476E0CE010196C4
:10E020000E94AF7DBE01675F7F4FCE0101960E94C7
:10E030002B7C6BEB78E00E94157CBE01615F7F4F0B
:10E040000E942B7C63E476E00E94157CBE016B5E2F
:10E050007F4F0E942B7CBC0182EE9FE00E94947C4B
:10E06000CE0101960E94107DCE0109960E94107D7E
:10E07000CE010F960E94107DCE0145960E94107D24
:10E080000F5F1F4FF8E0CF0ED11C22E0E20EF11C13
:10E090000430110509F077CFE0913811F091391172
:10E0A000EE0FFF1FE153FD4F60817181CE0101969C
:10E0B0000E94FD7A46E050E0BE016F5F7F4FCE01C7
:10E0C00009960E94B922BE01675F7F4F86ED9FE0EF
:10E0D0000E94947CCE0109960E94107DCE0101968B
:10E0E0000E94107DE0913A11F0913B11EE0FFF1F5D
:10E0F000E153FD4F60817181CE0101960E94FD7A4E
:10E1000046E050E0BE016F5F7F4FCE0109960E944E
:10E11000B922BE01675F7F4F86ED9FE00E94947C2D
:10E12000CE0109960E94107DCE0101960E94107DBD
:10E1300060E476E0CE0145960E94AF7D0E94258482
:10E1400028EE33E040E050E00E94CCB069017A0153
:10E150006DE174E0CE014B960E94AF7D6DE174E0FD
:10E1600088EE9FE00E94F37ACE0101960E9414226D
:10E1700044E150E0BE016F5F7F4FCE0109960E94DF
:10E18000B922BE01675F7F4F88EE9FE00E94D77C77
:10E19000CE0109960E94107DCE0101960E94107D4D
:10E1A0002AE0B701A601CE0109960E944E7D48E003
:10E1B00050E0BE01675F7F4FCE010F960E94B922EB
:10E1C00068EE7FE0CE0101960E94A67DBE01615FF0
:10E1D0007F4FCE0101960E942B7CBC018CED9FE00D
:10E1E0000E94C07CCE0101960E94107DCE010F9648
:10E1F0000E94107DCE0109960E94107D2AE0B70191
:10E20000A601CE0109960E944E7D6EEB78E0CE010C
:10E2100001960E94AF7DBE01675F7F4FCE010196E0
:10E220000E942B7CBE016B5E7F4F0E942B7CBC0149
:10E2300088EE9FE00E94947CCE0101960E94107DA2
:10E24000CE0109960E94107D4091E10B5091E20BA6
:10E250006091E30B7091E40B21E0CE0101960E94E6
:10E26000187DBE016F5F7F4FCE014B960E94D77C19
:10E27000CE0101960E94107D65EC78E0CE010196FA
:10E280000E94AF7DBE01655E7F4FCE0101960E9468
:10E290002B7CBE016B5E7F4F0E942B7CBC0188EE05
:10E2A0009FE00E94947CCE0101960E94107DBE01E9
:10E2B000655E7F4FCE0101960E94A67D46E050E04C
:10E2C000BE016F5F7F4FCE0109960E94B922BE0149
:10E2D000675F7F4F8CED9FE00E94947CCE01099692
:10E2E0000E94107DCE0101960E94107D4091DD0BB1
:10E2F0005091DE0B6091DF0B7091E00B21E0CE01BD
:10E3000001960E94187DBE016F5F7F4FCE014B9634
:10E310000E94D77CCE0101960E94107D63ED78E0CB
:10E32000CE0101960E94AF7DBE01655E7F4FCE019A
:10E3300001960E942B7CBE016B5E7F4F0E942B7C5E
:10E34000BC0188EE9FE00E94947CCE0101960E9461
:10E35000107DBE01655E7F4FCE0101960E94A67DB5
:10E3600046E050E0BE016F5F7F4FCE0109960E94EC
:10E37000B922BE01675F7F4F8CED9FE00E94947CC5
:10E38000CE0109960E94107DCE0101960E94107D5B
:10E3900060918E0270918F0280918C0290918D021B
:10E3A0000E94291B9093EE0B8093ED0B892B71F04B
:10E3B00060918E0270918F0280918C0290918D02FB
:10E3C0000E94291B9093EE0B8093ED0B8091ED0B37
:10E3D0009091EE0B8C3F9F4F0CF410C10E941F6B6D
:10E3E00029833A834B835C836D837E838F839887F5
:10E3F00049815A816B817C8121E0CE0109960E947E
:10E40000187DBE01675F7F4FCE014B960E94D77C7F
:10E41000CE0109960E94107D6DED78E0CE0109963F
:10E420000E94AF7DBE01655E7F4FCE0109960E94BE
:10E430002B7CBE016B5E7F4F0E942B7CBC0188EE63
:10E440009FE00E94947CCE0109960E94107DBE013F
:10E45000655E7F4FCE0109960E94A67D46E050E0A2
:10E46000BE01675F7F4FCE010F960E94B922BE01A9
:10E47000615F7F4F8CED9FE00E94947CCE010F96F0
:10E480000E94107DCE0109960E94107D4D815E8113
:10E490006F81788521E0CE0109960E94187DBE012A
:10E4A000675F7F4FCE014B960E94D77CCE010996C5
:10E4B0000E94107D68EE78E0CE0109960E94AF7D43
:10E4C000BE01655E7F4FCE0109960E942B7CBE0186
:10E4D0006B5E7F4F0E942B7CBC0188EE9FE00E9408
:10E4E000947CCE0109960E94107DBE01655E7F4F2F
:10E4F000CE0109960E94A67D46E050E0BE01675F0E
:10E500007F4FCE010F960E94B922BE01615F7F4FFF
:10E510008CED9FE00E94947CCE010F960E94107DAE
:10E52000CE0109960E94107D62EE7FE088EE9FE0AA
:10E530000E94947C60E476E0CE0101960E94AF7D5B
:10E5400066ED7FE0CE0101960E942B7CBC018CED34
:10E550009FE00E94947CCE0101960E94107D6CED9C
:10E560007FE0CE0101960E94A67DCE0101960E9419
:10E57000FB1ACE0101960E94107D6AE070E080E0F7
:10E5800090E00E945681CE014B960E94107DCE01F4
:10E5900045960E94107DA0960FB6F894DEBF0FBE80
:10E5A000CDBFDF91CF911F910F91FF90EF90DF9042
:10E5B000CF90BF90AF909F908F900895CE014596D9
:10E5C0000E94FD7AB801CE010F960E94FD7AB60135
:10E5D0006C5E7F4FCE0109960E94AF7D60E476E0CD
:10E5E000CE0101960E94AF7DBE01675F7F4FCE01D5
:10E5F00001960E942B7C6AEB78E01DCD6EEE78E0F0
:10E6000088EE9FE00E948A7C6DEF78E08CED9FE0C1
:10E610000E948A7C64E079E088EE9FE00E948A7C18
:10E620006DEF78E08CED9FE00E948A7C7DCFBF92F9
:10E63000CF92DF92EF92FF920F931F93CF93DF93CE
:10E64000CDB7DEB7C455D1090FB6F894DEBF0FBE03
:10E65000CDBF6C018B0165965FAF4EAF6597809122
:10E66000DB0B9091DC0B01969093DC0B8093DB0B22
:10E670008091F80B81113CC0BB24B394B092F80B8D
:10E680001092DC0B1092DB0B6DE174E0CE01895B24
:10E690009F4F0E94AF7D6DE174E0CE01835B9F4F81
:10E6A0000E94AF7D50E040E06EE174E0C6010E9440
:10E6B0006C1E0130110509F0A6C06DE174E088EE12
:10E6C0009FE00E94F37A6596EEADFFAD659780817D
:10E6D000811124C00E94916FB092520CCE01835BD5
:10E6E0009F4F0E94107DCE01895B9F4F0E94107D3D
:10E6F0000FB6F894DEBF0FBECDBFCC5ADF4F0FB6BA
:10E70000F894DEBF0FBECDBFDF91CF911F910F9167
:10E71000FF90EF90DF90CF90BF9008956596EEAD9B
:10E72000FFAD65978081882309F467C000E210E09F
:10E730009E012F5F3F4F40E250E0BE016F5D7F4F73
:10E74000CE018D5A9F4F0E94D477049739F3BE01B2
:10E750006F5D7F4FCE018F5B9F4F0E94AF7DBE01EB
:10E760006F5B7F4FCE01895B9F4F0E94D77CCE01AC
:10E770008F5B9F4F0E94107DBE016F5F7F4FCE0168
:10E780008F5B9F4F0E94AF7DBE016F5B7F4FCE01BD
:10E79000835B9F4F0E94D77CCE018F5B9F4F0E946F
:10E7A000107DBE01695B7F4F88EE9FE00E94947CE4
:10E7B00063968EAD9FAD6397892B09F4AFCF63E469
:10E7C00076E0CE018F5B9F4F0E94AF7DBE01635B01
:10E7D0007F4FCE018F5B9F4F0E942B7C60E476E0E1
:10E7E0000E94157CBC0188EE9FE00E94947CCE01C3
:10E7F0008F5B9F4F0E94107D91CF68EE7FE084EC8D
:10E800009FE00E94C07C1092F80B68CF0895089595
:10E8100008950895AF92BF92CF92DF92EF92FF9248
:10E820000F931F93CF93DF936C017B018B01040F38
:10E83000151FEB015E01AE18BF08C017D10759F0D4
:10E840006991D601ED91FC910190F081E02DC60116
:10E850001995892B79F7C501DF91CF911F910F9100
:10E86000FF90EF90DF90CF90BF90AF900895FC01A4
:10E87000538D448D252F30E0842F90E0821B930B25
:10E88000541710F0CF96089501970895FC01918DCB
:10E89000828D981761F0A28DAE0FBF2FB11D5D96CE
:10E8A0008C91928D9F5F9F73928F90E008958FEF70
:10E8B0009FEF0895FC01918D828D981731F0828D24
:10E8C000E80FF11D858D90E008958FEF9FEF08957B
:10E8D000FC01918D228D892F90E0805C9F4F821BDF
:10E8E00091098F739927089588E89CE00E946874C5
:10E8F00021E0892B09F420E0822F089585E29DE034
:10E900000E94687421E0892B09F420E0822F089589
:10E91000FC01A48DA80FB92FB11DA35ABF4F2C9194
:10E92000848D90E001968F739927848FA689B7898B
:10E930002C93A089B1898C91837080648C93938D82
:10E94000848D981306C00288F389E02D80818F7D25
:10E9500080830895EF92FF920F931F93CF93DF93DD
:10E96000EC0181E0888F9B8D8C8D98131AC0E8890B
:10E97000F989808185FF15C09FB7F894EE89FF89DA
:10E980006083E889F98980818370806480839FBF78
:10E9900081E090E0DF91CF911F910F91FF90EF9078
:10E9A0000895F62E0B8D10E00F5F1F4F0F73112788
:10E9B000E02E8C8D8E110CC00FB607FCFACFE889C3
:10E9C000F989808185FFF5CFCE010E948874F1CF4F
:10E9D000EB8DEC0FFD2FF11DE35AFF4FF0829FB737
:10E9E000F8940B8FEA89FB8980818062CFCFCF9327
:10E9F000DF93EC01888D8823B9F0AA89BB89E88967
:10EA0000F9898C9185FD03C0808186FD0DC00FB60C
:10EA100007FCF7CF8C9185FFF2CF808185FFEDCF8A
:10EA2000CE010E948874E9CFDF91CF91089580E0F4
:10EA300090E0892B29F00E947E7481110E940000D1
:10EA400080E090E0892B49F080E090E0892B29F06C
:10EA50000E94000081110E94000080E090E0892B5C
:10EA600049F080E090E0892B29F00E94000081119C
:10EA70000E94000080E090E0892B29F00E947474CD
:10EA800081110C94000008958150823108F05AC021
:10EA9000E82FF0E08827E05BFA488F4F0C946EB2C5
:10EAA00070757475627568756C75A27577757D750E
:10EAB000817587758B758F7595759975A2759D751F
:10EAC000A375A775809180008F778093800008954B
:10EAD000809180008F7DF9CF80918000877FF5CF76
:10EAE00084B58F7784BD089584B58F7DFBCF8091E9
:10EAF000B0008F778093B00008958091B0008F7D33
:10EB0000F9CF809190008F77809390000895809145
:10EB100090008F7DF9CF80919000877FF5CF809115
:10EB2000A0008F778093A00008958091A0008F7D32
:10EB3000F9CF8091A000877FF5CF809120018F775A
:10EB4000809320010895809120018F7DF9CF8091DD
:10EB50002001877FF5CFCF93DF93282F30E0F90195
:10EB6000E35AF34F8491F901E25EF24FD491F90137
:10EB7000EC59F24FC491CC23A1F081110E9444754D
:10EB8000EC2FF0E0EE0FFF1FED5BF34FA591B4917A
:10EB9000EC91ED2381E090E009F480E0DF91CF91EA
:10EBA000089580E090E0FACF20910C12260F3327D1
:10EBB000331F21323105ECF420917D0CFC0190E0F3
:10EBC00080E0243069F082E00895A0910C12219138
:10EBD000AC0144515E4EA40FB52FB11D2C9301968C
:10EBE000861798F380910C12680F60930C1280E0E6
:10EBF000089581E00895E091460C8091450CE81756
:10EC000030F4F0E0EE54F44F808190E008958FEFFF
:10EC10009FEF08959091460C8091450C2FEF3FEFA8
:10EC2000981748F4E92FF0E0EE54F44F208130E0DB
:10EC30009F5F9093460CC90108958091450C909177
:10EC4000460C891B990B0895CF92DF92EF92FF92A9
:10EC50000F931F93CF93DF937C01CB018A01209107
:10EC6000830C222389F0EB016B01C40ED51ECC1559
:10EC7000DD0569F06991D701ED91FC910190F0817A
:10EC8000E02DC7011995F3CF642F0E94D475C801F8
:10EC9000DF91CF911F910F91FF90EF90DF90CF9078
:10ECA0000895CF93DF931F92CDB7DEB7698320918C
:10ECB000830C2223F9F02091860C203258F021E0B9
:10ECC00030E0FC013383228390E080E00F90DF91FD
:10ECD000CF9108958091840CE82FF0E0EB56FA4E26
:10ECE000998190838F5F8093840C8093860C81E060
:10ECF00090E0ECCF61E0CE0101960E94D475F7CF91
:10ED00000E9497B40F931F93CF93DF93EC018881F8
:10ED10009981009759F02A813B812617370730F0F7
:10ED200081E0DF91CF911F910F9108958B016F5F6B
:10ED30007F4F0E94B6B3009759F0998388831B8355
:10ED40000A832C813D81232B59F7FC011082E8CFE7
:10ED500080E0E7CFEF92FF920F931F93CF93DF9363
:10ED60006115710541F480E0DF91CF911F910F9102
:10ED7000FF90EF90089541155105B1F07B01EC0132
:10ED80000C811D81040F151FB8010E948276882313
:10ED900051F3288139818C819D81B701820F931FA6
:10EDA0000E94E7B41D830C8381E0DECFCF93DF9315
:10EDB000EC0188819981009711F00E942DB319828E
:10EDC00018821D821C821B821A82DF91CF910895C6
:10EDD000EF92FF920F931F93CF93DF93EC017B0190
:10EDE0008A01BA010E94827681110BC0CE010E9475
:10EDF000D676CE01DF91CF911F910F91FF90EF90CA
:10EE000008951D830C83B701888199810E94E7B41E
:10EE1000F0CF8091E6118823A9F1409168025091CA
:10EE2000690260916A0270916B0229E233E180917C
:10EE3000291590912A150E949E0C811102C080E034
:10EE400008954091E7115091E8116091E911709196
:10EE5000EA11411551056105710591F029E233E18F
:10EE60008091291590912A150E949E0C882339F3D0
:10EE70001092E7111092E8111092E9111092EA1124
:10EE80001092E61181E008958F929F92AF92BF9207
:10EE9000EF92FF920F931F93CF934B015C01C42F0E
:10EEA0008091680290916902A0916A02B0916B0210
:10EEB00088159905AA05BB0549F10E9409778111BA
:10EEC0000BC080E0CF911F910F91FF90EF90BF900A
:10EED000AF909F908F90089589E2E82E83E1F82EFD
:10EEE00000E012E030E020E0B501A4018091291596
:10EEF00090912A150E94F70B882319F380926802DB
:10EF000090926902A0926A02B0926B024091E6115F
:10EF10004C2B4093E61181E0D5CF8CBD9DBD08956B
:10EF2000CF93DF93EC019A01AB01E889F98982E084
:10EF30008083211581EE38074105510581F160E09C
:10EF400079E08DE390E00E94CCB021503109410975
:10EF500051095695479537952795EC85FD85108283
:10EF6000EE85FF852083188EEC89FD8986E08083FD
:10EF7000EA89FB89808180618083EA89FB898081BD
:10EF800088608083EA89FB89808180688083EA8940
:10EF9000FB8980818F7D8083DF91CF910895E889FF
:10EFA000F989108220E1D9CF2F923F924F925F9240
:10EFB0006F927F928F929F92AF92BF92CF92DF9289
:10EFC000EF92FF920F931F93CF93DF9300D0CDB7B3
:10EFD000DEB71C013B014A0129015801FC01C08038
:10EFE000D18070E060E0C3010E94CCB4A80170E061
:10EFF00060E0C2010E94CCB4F601808110E000E024
:10F00000811162C004E010E004C07601F101F182D8
:10F01000E082C8010F900F900F90DF91CF911F9168
:10F020000F91FF90EF90DF90CF90BF90AF909F90A7
:10F030008F907F906F905F904F903F902F900895AA
:10F040006B3209F482C06D3309F04EC08181882390
:10F05000E9F2F7018FEFE81AF80A6081653209F4E6
:10F0600052C00CF048C0662309F456C082E0A816CE
:10F07000B1040CF061C0012B09F46BC003E010E097
:10F08000E8CF81818983882309F282818A8376018E
:10F09000811104C0F2E0EF0EF11CB8CF83E0E80E5E
:10F0A000F11C1B8240E150E070E060E0CE0101966F
:10F0B0000E9445A719C0F3016083F1E08F1A9108FF
:10F0C000C30101963C0167017601FFEFEF1AFF0AC9
:10F0D000F6016081663209F499CF0CF0B1CF662356
:10F0E00009F493CF653269F2F2E08F1691041CF7B0
:10F0F00001E010E0E8CF663209F488CF6B3209F006
:10F10000B5CF60E2B3CF81818983882301F1828109
:10F110008A83811103C032967F0178CF7F0193E00B
:10F12000E90EF11C1B8240E150E070E060E0CE018E
:10F1300001960E9445A79ACFF2016083F1E0AF1AD1
:10F14000B108C20101962C0184CF60E2CDCFF70156
:10F15000E3CF02E010E07DCF0F931F93CF93DF93B7
:10F160004115510541F0FC0104811581011511057E
:10F1700039F4FB011082DF91CF911F910F91089517
:10F18000415051094017510708F48A01EB01FC0175
:10F1900060817181A801CE010E94FCB4C00FD11F13
:10F1A0001882E9CF20E3FC0120833296862F8295D6
:10F1B0008F706F706A3030F4605D6293682F8111D8
:10F1C000F5CF0895695CF9CF8F929F92AF92BF926D
:10F1D000CF92DF92EF92FF92CF932EEC3DE03093EF
:10F1E0002A1520932915882309F46DC040E060E0BA
:10F1F00070E0CB010E94447781110BC080E0CF9179
:10F20000FF90EF90DF90CF90BF90AF909F908F9046
:10F2100008958091E7148F7789F78091F314909186
:10F22000F414A091F514B091F61484369105A1055B
:10F23000B10520F3C090EF14D090F014E090F114D9
:10F24000F090F214C114D104E104F104B9F240E0E9
:10F25000C701B6010E944477882381F2809134135C
:10F26000909135138115924049F6A0913913AA2344
:10F2700029F260913713709138136115710509F403
:10F28000BDCF20913613222309F4B8CFA093EC0D03
:10F290002093DE0D90E080E030E0E1E0F0E0C82F68
:10F2A000AF01082E02C0440F551F0A94E2F724173D
:10F2B000350769F041E0480F01968930910579F7EB
:10F2C0004093E70D9BCFC12CD12C7601C0CF80930A
:10F2D000E70D20913F133091401350E040E021159D
:10F2E000310541F420914D1330914E1340914F134D
:10F2F000509150132093DF0D3093E00D4093E10DBA
:10F300005093E20D46015701860E971EA11CB11CB9
:10F310008092ED0D9092EE0DA092EF0DB092F00D57
:10F32000E0913A13F0913B13F093F30DE093F20D5B
:10F33000B0E00E940DB1DC01CB01880D991DAA1D22
:10F34000BB1D8093F40D9093F50DA093F60DB09333
:10F35000F70D25E0EE0FFF1F2A95E1F7E150FE4F74
:10F36000EF2FFF27E6958E0F9F1FA11DB11D8093E4
:10F37000E80D9093E90DA093EA0DB093EB0D80900A
:10F380003C1390903D13B12CA12C8114910441F4B5
:10F390008090491390904A13A0904B13B0904C1357
:10F3A000C81AD90AEA0AFB0AC80CD91CEA1CFB1CB9
:10F3B00004C0F694E794D794C794CA95D2F7C09244
:10F3C000E30DD092E40DE092E50DF092E60D85EFAD
:10F3D000C8168FE0D806E104F10428F48CE080938D
:10F3E000F10D81E00CCF80E125EFC2162FEFD206A0
:10F3F000E104F104A0F38091551390915613A0916C
:10F400005713B09158138093F40D9093F50DA0937A
:10F41000F60DB093F70D80E2E2CF8F929F92AF92FC
:10F42000BF92CF92DF92EF92FF920F931F93CF93F1
:10F43000DF93CDB7DEB760970FB6F894DEBF0FBE8F
:10F44000CDBF7C0190914A0C992351F108E0933390
:10F4500009F404E06B0180E591E00E948D779E0144
:10F460002F5F3F4F5901490110E0812F0E948F0FFC
:10F47000F40181934F018823D9F01F5F0113F5CF69
:10F4800000E0F50181915F018D3161F0883151F02B
:10F490008A51823038F00F5F1013F3CF0E940A11A7
:10F4A00018E08AC060E170E0802F0E94ED0F102FFD
:10F4B000A12EB12CF501EE0FFF1FEB5CF34F118273
:10F4C000108283EE93E00197F1F742E870E060E08C
:10F4D000812F0E94D00F4FEF62E070E0812F0E94D9
:10F4E000D00FB601C114D10491F480919002909193
:10F4F000910201968115F0EC9F0708F471C090937A
:10F500009102809390026091900270919102812FFC
:10F510000E94BA0F86E0E5E2F3E0DE011996019061
:10F520000D928A95E1F7F70183818F778C8784812B
:10F530008D8785818E87A7014E5F5F4F24E030E085
:10F540006CE070E0812F0E94930FB601812F0E9422
:10F55000A40F26E030E0AE01475F5F4F66E070E049
:10F56000812F0E94930F61E070E0812F0E94ED0FC8
:10F5700027E02A9DC0012B9D900D11249C01235052
:10F58000344F7901F9011182108222E030E0AE019E
:10F59000415F5F4F68E270E0812F0E94FD0F8F8511
:10F5A0009889982789279827F70193838283168261
:10F5B000158214820E940A11812F60960FB6F8946A
:10F5C000DEBF0FBECDBFDF91CF911F910F91FF9096
:10F5D000EF90DF90CF90BF90AF909F908F90089565
:10F5E00080E090EC8CCFFB0101900020E9F731978F
:10F5F000AF01461B570B0C94E8760F931F93CF93E4
:10F60000DF93CDB7DEB762970FB6F894DEBF0FBEBB
:10F61000CDBF8C01CB01F8011182108213821282BE
:10F62000158214824AE0BE016F5F7F4F0E948CA852
:10F63000BE016F5F7F4FC8010E94F37A62960FB6DA
:10F64000F894DEBF0FBECDBFDF91CF911F910F9118
:10F6500008950F931F93CF93DF93CDB7DEB7A19794
:10F660000FB6F894DEBF0FBECDBF8C01CB01BA013F
:10F67000F8011182108213821282158214822AE00C
:10F68000AE014F5F5F4F0E94C6A8BE016F5F7F4F04
:10F69000C8010E94F37AA1960FB6F894DEBF0FBEA0
:10F6A000CDBFDF91CF911F910F910895FC01808113
:10F6B0009181009711F00C9448A860E070E0CB01B4
:10F6C0000895FC0180819181009711F00C944CA861
:10F6D00060E070E0CB010895AF92BF92CF92DF92CD
:10F6E000EF92FF920F931F93CF93DF93DC01CD90A6
:10F6F000DC901197C114D10439F01496CD91DC91AE
:10F700008C017601209761F4DF91CF911F910F91C9
:10F71000FF90EF90DF90CF90BF90AF90089575016C
:10F720005701BFEFAB1ABB0AF7018081082E000C0E
:10F73000990B0E9473A8892B91F72197CC0DDD1DA1
:10F740008881082E000C990B0E9473A8892B29F040
:10F75000CE15DF0510F02197F3CFAE014F5F5F4F5D
:10F760004E195F09D80115965C934E931497CE14E9
:10F77000DF0420F4B701C6010E94B1B4D801ED91B5
:10F78000FC91119714968D919C91E80FF91F1082AE
:10F79000BBCFFC01248135816217730748F4808157
:10F7A0009181009729F0860F971FFC0180810895B1
:10F7B00080E00895FC0124813581FB01448155815D
:10F7C00024173507A0F0FC0180819181009779F022
:10F7D000FB01608171816115710549F0241B350BB6
:10F7E000820F931F0E94DEB421E0892B09F020E0F4
:10F7F000822F0895FB0144815581FC0124813581CC
:10F800002417350778F080819181009759F0FB012A
:10F81000608171816115710529F00E94EEB421E0CB
:10F82000892B09F020E0822F0895CF93DF93EC011C
:10F83000FB0101900020E9F73197AF01461B570B00
:10F840000E94AA76811103C0CE010E94D676CE0115
:10F85000DF91CF910895CF93DF93EC01FB014481B9
:10F860005581608171810E94AA76811103C0CE0109
:10F870000E94D676CE01DF91CF910895EF92FF924C
:10F880000F931F93CF93DF93EC017B01CB010E9479
:10F8900083A80097A9F00C811D81080F191FB801DA
:10F8A000CE010E948276882361F0288139818C8183
:10F8B0009D81B701820F931F0E947CA81D830C833A
:10F8C00081E0DF91CF911F910F91FF90EF9008950C
:10F8D000CF93DF931F921F92CDB7DEB769831A8251
:10F8E00041E050E0BE016F5F7F4F0E94AA760F900B
:10F8F0000F90DF91CF910895CF93DF93EC010E9499
:10F90000687C811103C0CE010E94D676CE01DF91C2
:10F91000CF910895FB0101900020E9F73197AF01E5
:10F92000461B570B0C94AA76FB01448155816081DC
:10F9300071810C94AA76EF92FF920F931F93CF934D
:10F94000DF93EC018B01CB010E9483A87C01BC01F9
:10F95000CE010E94827681110BC0CE010E94D67624
:10F96000CE01DF91CF911F910F91FF90EF900895FD
:10F97000FD82EC82B801888199810E947CA8F0CF39
:10F98000CF93DF93EC01FB018617970749F0608165
:10F9900071816115710541F0448155810E94E876BD
:10F9A000CE01DF91CF9108950E94D676F9CF0F93C3
:10F9B0001F93CF93DF938C01EB01FC018081918138
:10F9C0000097E1F06881798161157105A9F04281A4
:10F9D00053812C813D814217530770F00E94E7B498
:10F9E0008C819D81F801958384831D821C82DF9127
:10F9F000CF911F910F9108950E942DB38881998115
:10FA0000F801918380838A819B81938382838C8197
:10FA10009D8195838483198218821B821A82E5CF87
:10FA2000FC0180819181009711F00C942DB3089511
:10FA3000EF92FF920F931F93CF93DF93CDB7DEB773
:10FA4000A1970FB6F894DEBF0FBECDBF7C01CB01EE
:10FA5000BA01F70111821082138212821582148278
:10FA600042E0420F8E010F5F1F4F0E9483A6009756
:10FA700089F0BC01C7010E94F37AA1960FB6F894F1
:10FA8000DEBF0FBECDBFDF91CF911F910F91FF90D1
:10FA9000EF900895C7010E94D676EFCF0F931F9382
:10FAA000CF93DF93CDB7DEB7A2970FB6F894DEBF42
:10FAB0000FBECDBF8C01CB01BA01F80111821082BB
:10FAC000138212821582148230E0AE014F5F5F4FC5
:10FAD0000E9497A8BE016F5F7F4FC8010E94F37A12
:10FAE000A2960FB6F894DEBF0FBECDBFDF91CF91C7
:10FAF0001F910F910895CF93DF931F921F92CDB75F
:10FB0000DEB7FC01118210821382128215821482E8
:10FB100069831A82BE016F5F7F4F0E94F37A0F9054
:10FB20000F90DF91CF910895FC0111821082138212
:10FB30001282158214820C94D77CFC0111821082EF
:10FB400013821282158214820C949B7CFC01118218
:10FB5000108213821282158214820C94C07CFC01E4
:10FB6000118210821382128215821482611571052E
:10FB700051F0FB0101900020E9F73197AF01461BDE
:10FB8000570B0C94E8760895AF92BF92CF92DF9214
:10FB9000EF92FF920F931F93CF93DF936C015B0162
:10FBA0007A0189012417350720F48F2D7901042F5C
:10FBB000182F6DE174E0C6010E94AF7DD501149647
:10FBC000CD91DC91EC16FD06E0F40C171D0708F44E
:10FBD000E801D501ED91FC911197EC0FFD1F10810B
:10FBE00010826D917C916E0D7F1DC60161157105AE
:10FBF000A1F00E94F37AF50180819181C80FD91F8D
:10FC00001883C601DF91CF911F910F91FF90EF9064
:10FC1000DF90CF90BF90AF9008950E94D676EBCF43
:10FC2000FB0101900020E9F73197AF01461B570B0C
:10FC3000DC01ED91FC910280F381E02D19948F920B
:10FC40009F92AF92BF92EF92FF920F931F93CF9329
:10FC5000DF93CDB7DEB7A1970FB6F894DEBF0FBE26
:10FC6000CDBF7C01FA01CB0119A2223008F42AE0B1
:10FC70008E010F5D1F4F822E912CB12CA12CBF0144
:10FC8000A50194010E94CCB0F901CA016A300CF5BB
:10FC9000605DD8016E938D01232B242B252B79F7E2
:10FCA00090E080E0109721F0BD01C7010E94107E16
:10FCB000A1960FB6F894DEBF0FBECDBFDF91CF91F6
:10FCC0001F910F91FF90EF90BF90AF909F908F90FA
:10FCD0000895695CDECF8F929F92AF92BF92CF92D0
:10FCE000DF92EF92FF920F931F93CF93DF937C01EC
:10FCF000EB016C0182E0C80ED11C4701E5E08E0EDD
:10FD0000911C10E000E0F60141916F0150E070E0BD
:10FD100060E02AE0CE010E941F7E5C01E881F9814B
:10FD20000190F081E02D6EE2CE0119958A0D9B1DA8
:10FD3000080F191FC814D90431F7F701458150E0A5
:10FD400070E060E02AE0CE010E941F7E800F911FCC
:10FD5000DF91CF911F910F91FF90EF90DF90CF90A7
:10FD6000BF90AF909F908F9008950F931F93CF9364
:10FD7000DF93EC010E94107E8C0167E779E0CE01F1
:10FD80000E94107E800F911FDF91CF911F910F91E4
:10FD900008956115710511F00C94107E90E080E0DB
:10FDA0000895DB0114964D915C9115976D917C91AE
:10FDB000DC01ED91FC910280F381E02D19940F9309
:10FDC0001F93CF93DF93EC010E94D17E8C0167E7F4
:10FDD00079E0CE010E94107E800F911FDF91CF91BC
:10FDE0001F910F910895EF92FF920F931F93CF935E
:10FDF000DF938C017B01D0E0C0E0F701EC0FFD1F29
:10FE00006491662361F0D801ED91FC910190F0813D
:10FE1000E02DC8011995892B11F02196EECFCE0166
:10FE2000DF91CF911F910F91FF90EF900895DC012A
:10FE300082E194E08D939D9384E0FB0101900D920B
:10FE40008A95E1F708951F920F920FB60F92112431
:10FE50000BB60F922F933F934F935F936F937F93C4
:10FE60008F939F93AF93BF93EF93FF9388E89CE0AA
:10FE70000E948874FF91EF91BF91AF919F918F91F4
:10FE80007F916F915F914F913F912F910F900BBE9A
:10FE90000F900FBE0F901F9018951F920F920FB6E4
:10FEA0000F9211240BB60F922F938F939F93EF9382
:10FEB000FF93E091980CF091990C8081E0919E0C59
:10FEC000F0919F0C82FD1DC090818091A10C8F5FED
:10FED0008F732091A20C821741F0E091A10CF0E009
:10FEE000E857F34F958F8093A10CFF91EF919F916D
:10FEF0008F912F910F900BBE0F900FBE0F901F9000
:10FF000018958081F2CF1F920F920FB60F92112495
:10FF10000BB60F922F933F934F935F936F937F9303
:10FF20008F939F93AF93BF93EF93FF9385E29DE0F1
:10FF30000E948874FF91EF91BF91AF919F918F9133
:10FF40007F916F915F914F913F912F910F900BBED9
:10FF50000F900FBE0F901F9018951F920F920FB623
:10FF60000F9211240BB60F922F938F939F93EF93C1
:10FF7000FF93E091350DF091360D8081E0913B0DBE
:10FF8000F0913C0D82FD1DC0908180913E0D8F5FF0
:10FF90008F7320913F0D821741F0E0913E0DF0E00C
:10FFA000EB5DF24F958F80933E0DFF91EF919F9106
:10FFB0008F912F910F900BBE0F900FBE0F901F903F
:10FFC00018958081F2CF1F93CF93DF93282F30E0D5
:10FFD000F901E35AF34F8491F901E25EF24FD491B3
:10FFE000F901EC59F24FC491CC23A9F0162F8111DD
:10FFF0000E944475EC2FF0E0EE0FFF1FE651F34F27
:020000040001F9
:10000000A591B4918FB7F894EC91111108C0D095D7
:10001000DE23DC938FBFDF91CF911F910895DE2BFC
:10002000F8CFAF92BF92CF92DF92EF92FF920F93F1
:100030001F93CF93DF936B017A01EC01CE5EDC4E10
:1000400028813CE0389F8001399F100D1124A09039
:10005000E515B12C27FF1FC0FB011182108288819A
:100060008F5F888388819801280F311D87FD3A951D
:10007000F6012A153B051CF488818C30C4F180817F
:100080009181049680349C4908F473C0F601808104
:100090009181049670C088819801280F311D87FDD9
:1000A0003A952A153B05DCF68881A801480F511DB9
:1000B00087FD5A95FA01EE0FFF1FE40FF51FE35E6F
:1000C000F14F808186FFCBCF8881F801E80FF11DC9
:1000D00087FDFA95CF01EE0FFF1FE80FF91FE35ED2
:1000E000F14F808160E08F730E94E37FB8CF808101
:1000F00091812881A801420F511D27FD5A959A012F
:10010000FA01EE0FFF1FE20FF31FE35EF14F2181B3
:100110003281820F931FF701918380838881980138
:10012000280F311D87FD3A95F901EE0FFF1FE20FF1
:10013000F31FE35EF14F808186FF22C08881080FA4
:10014000111D87FD1A95F801EE0FFF1FE00FF11F3B
:10015000E35EF14F808161E08F73DF91CF911F915A
:100160000F91FF90EF90DF90CF90BF90AF900C94E5
:10017000E37F80E49CE9F701918380838FEF88839C
:10018000DF91CF911F910F91FF90EF90DF90CF9073
:10019000BF90AF90089510927D0C81E080937C0C0D
:1001A0001092570C61E084E10E94E37F61E085E1F9
:1001B0000E94E37FE9EBF0E080818E7F8083808185
:1001C0008D7F808388E48093B80085E48093BC00B1
:1001D00008951092460C1092450C1092840C1092C7
:1001E000860C0E94CB8087E094E79093281380933D
:1001F000271388E094E7909326138093251308959E
:10020000CF93DF9390E0FC01E25EF24F24918C5992
:10021000924FFC0184918823D1F090E0880F991FC0
:10022000FC01EC5FF24FA591B491FC01E651F34F54
:10023000C591D49161110EC09FB7F8948C91E22FB3
:10024000E0958E238C932881E223E8839FBFDF9182
:10025000CF9108958FB7F894EC91E22BEC938FBF78
:10026000F6CF3FB7F89480911B1390911C13A09187
:100270001D13B0911E1326B5A89B05C02F3F19F082
:100280000196A11DB11D3FBFBA2FA92F982F882716
:10029000BC01CD01620F711D811D911D42E0660FF1
:1002A000771F881F991F4A95D1F708958F929F92C3
:1002B000AF92BF92CF92DF92EF92FF926B017C01DF
:1002C0000E9431814B015C01C114D104E104F104AD
:1002D000B9F00E943181681979098A099B09683E41
:1002E00073408105910580F321E0C21AD108E1082D
:1002F000F10888EE880E83E0981EA11CB11CE4CFA3
:10030000FF90EF90DF90CF90BF90AF909F908F9035
:100310000895AF92BF92CF92DF92EF92FF920F9328
:100320001F93CF93DF93C82FD62F1092581110929E
:10033000591110925A1110925B1110925C1161E0E8
:100340000E94008160E08C2F0E94E37F6D2F70E09F
:1003500090E080E00E94568160E08C2F0E94008136
:100360008BE990E00197F1F700E911E08C2F0E94F2
:10037000AB75892B81F401501109C1F78EEF9FEF06
:10038000DF91CF911F910F91FF90EF90DF90CF9071
:10039000BF90AF90089500E911E08C2F0E94AB75DB
:1003A000019721F401501109C1F7E8CF18E2D0E814
:1003B00000E090E9E92EFF24F3948C2F0E94AB75A6
:1003C000892B29F481E0E81AF108B9F7D7CF0E9408
:1003D00031816B017C0180E9A82EBB24B3948C2F62
:1003E0000E94AB75019729F481E0A81AB108B9F70A
:1003F000C5CF0E9431816C197D098E099F09693230
:1004000071058105910538F0E02FF0E0E05BFE4ECC
:1004100080858D2B8087D69511F40F5FD0E8115021
:1004200041F690E080E0ACCF0F931F93CF93DF9322
:1004300000D000D01F921F92CDB7DEB780918B15F0
:1004400081112AC0109273151092721588EE93E0F4
:10045000A0E0B0E08093741590937515A093761585
:10046000B09377158CE993E0909371158093701594
:1004700082E194E090937F1580937E151092801511
:1004800010928115109282151092831588E0809346
:10049000881581E080938B158DE295E190934D0C4A
:1004A00080934C0C80912C1581119DC060E372E00B
:1004B00080E090E00E9456811FB7F89480912B1540
:1004C000811127C0E9E9FDE08491E3E5FDE0949125
:1004D000E82FF0E0EE0FFF1FEC5FF24FA591B49113
:1004E000EC91E92321F461E085E30E94E37F61E080
:1004F00085E30E9400818CB580618CBD8CB58064E1
:100500008CBD61E084E30E94008161E083E30E948E
:10051000008180912B158F5F80932B151FBFEEE616
:10052000FDE0E491F0E0EE0FFF1FE651F34F8591FF
:1005300094919093490C8093480CE8E2FDE0E4919B
:10054000E093470C61E08AE00E9400810E94F30D75
:1005500080E591E00E948D7784E380934A0C80E8E7
:100560000E947C0F0E94660F882309F4F5C088E082
:100570000E947C0F0E94530F883009F0EDC080E18B
:100580000E947C0F0E94530F803109F0E5C080E08B
:100590000E947C0F0E94530F182F8111DDC041E093
:1005A00050E0BE016F5F7F4F8FE190E00E94FD0D34
:1005B0008981833009F0D0C080E480934B0C42E005
:1005C0006EE170E0812F0E94D00F42E06FE170E099
:1005D000812F0E94D00F1F5F183089F70E940A11E7
:1005E00081E080932C1580E591E00E948D7746E0B4
:1005F00050E062E972E089E090E00E94A50E82E19D
:1006000094E09A8389831B821C821D821E82CE0104
:1006100003960E9403110E940A1180914C0C909144
:100620004D0CDC0192961D921D921D921C92959785
:10063000FC0116A217A210A611A69A961D921D9251
:100640001D921C929D9740E65AEE60E070E046AB2A
:1006500057AB60AF71AF40EA5FE060E070E0DA9600
:100660004D935D936D937C93DD973E9624E1DF017E
:100670001D922A95E9F726E0E2E9F2E0DC011896FE
:1006800001900D922A95E1F7FC01EE5BFF4F10827D
:100690000E94A8298C01019709F0CBC080E591E068
:1006A0000E948D7760914C0C70914D0C625F7F4F72
:1006B000CE0101960E94177FCE0103960E9403117E
:1006C00060914C0C70914D0C6A5E7F4FCE0101968B
:1006D0000E94177F44E050E0BE016D5F7F4F81E0D4
:1006E00090E00E94A50E60914C0C70914D0C6E5ED6
:1006F0007F4FCE0101960E94177F44E050E0BE017B
:100700006D5F7F4F85E090E00E94A50E0E940A1168
:1007100060914C0C70914D0C625E7F4FCE01019642
:100720000E94177F8B819C81AD81BE818093190EC1
:1007300090931A0EA0931B0EB0931C0E0E94318151
:100740007F7380919002909191026827792770932E
:100750009102609390026DC087E380934A0C80E819
:100760000E947C0F0E94660F882329F188E00E9476
:100770007C0F0E94530F8830F1F480E10E947C0FBF
:100780000E94530F182F8031B1F480E00E947C0F3B
:100790000E94530F81110FC041E050E0BE016F5F16
:1007A0007F4F89E390E00E94FD0D8981843019F428
:1007B00010934B0C13CF83E380934A0C80E80E9484
:1007C0007C0F0E94660F882371F180E10E947C0FEC
:1007D0000E94530F803139F582E10E947C0F0E9404
:1007E000530F823101F580E00E947C0F0E94530F6D
:1007F000811119C084E080934B0C15E5188741E006
:1008000050E0BE01685F7F4F8BE190E00E94A50E33
:100810001F8341E050E0BE01695F7F4F8AE190E0B5
:100820000E94A50EDBCE10924A0C0E940A1110E025
:1008300000E0C80128960FB6F894DEBF0FBECDBF0A
:10084000DF91CF911F910F9108952FB7F894609188
:100850001713709118138091191390911A132FBFC9
:100860000895CF92DF92EF92FF92CF93DF93809122
:10087000C90E883050F0CFEFDFEFCE01DF91CF917E
:10088000FF90EF90DF90CF900895E091EE0EE11190
:1008900042C00E9425846B017C0128EEC20E23E039
:1008A000D21EE11CF11C8DEB9EE00E947015882386
:1008B00011F38091240F882331F08091EF0E9091F5
:1008C000F00E892BC1F28DEB9EE00E94D313EC0158
:1008D000CF3FDC0771F08091240F882371F2809163
:1008E000EF0E9091F00E01979093F00E8093EF0E23
:1008F000C4CF0E942584C616D706E806F90698F6E6
:100900001092EE0E8DEB9EE00E94CB158DEB9EE0DB
:100910000E949215B2CFE150E093EE0EF0E0ED545C
:10092000F14FC38DD0E0A9CF0F931F93CF93DF93E7
:10093000EC018C01F80181918F018823A1F10E94C3
:100940003184F8012291022E000C330B8217930799
:1009500089F38F3F980781F0A091EE0E91E09A0FF6
:100960009093EE0EB0E0AD54B14F5B968C93903205
:1009700019F48FE18093EE0E2FE1EC17FD07C9F01B
:1009800092919F3FD1F3A091EE0E81E08A0F809368
:10099000EE0EB0E0AD54B14F5B969C93803269F798
:1009A0002093EE0EEACF81E0DF91CF911F910F915E
:1009B000089580E0F9CF0F931F93CF93DF93EC015D
:1009C0000E9425848B010E94A00B8F3F69F00E943A
:1009D0002584601B710B6C177D07A8F380E0DF9105
:1009E000CF911F910F91089581E0F9CF4F925F92BF
:1009F0006F927F928F929F92AF92BF92CF92DF922F
:100A0000EF92FF920F931F93CF93DF93CDB7DEB793
:100A100063970FB6F894DEBF0FBECDBF7C016B01AC
:100A20003A01FB0120E090E080E06AE0319133235D
:100A300009F461C040ED430F4A3008F04DC0689F93
:100A4000A001699F500D1124CA01C097830F911D09
:100A500037FD9A958F3F910549F340F3F7014281A5
:100A60005381648175818091DB159091DC15A09193
:100A7000DD15B091DE15481759076A077B0709F4A1
:100A80000DC28701085F1F4F0E9425846F70772772
:100A90007C5FC8010E942317813009F004C282E103
:100AA00094E09A838983F70182819381A481B5813F
:100AB0008B839C83AD83BE8345E350E0BE016F5FB3
:100AC0007F4FC8010E94AC17892BA9F5D12CC12CEE
:100AD000C8010E944F1417C03E3209F0BFCF233027
:100AE00009F4BCCFD301A20FB11D12968C932F5FD6
:100AF00090E080E09BCF233009F0B0CFF3018583F5
:100B0000CC24C394D12CC60163960FB6F894DEBFF3
:100B10000FBECDBFDF91CF911F910F91FF90EF904E
:100B2000DF90CF90BF90AF909F908F907F906F900D
:100B30005F904F9008950E942584F7017783668324
:100B400042E050E0B7016A5F7F4FC8010E94411741
:100B500081E090E09A83898342E050E0BE016F5FBC
:100B60007F4FC8010E94411780E091E09A838983FA
:100B700042E050E0BE016F5F7F4FC8010E94411705
:100B80001A82198242E050E0BE016F5F7F4FC801B8
:100B90000E94411742E050E0BE016F5F7F4FC801E5
:100BA0000E94411742E050E0BE016F5F7F4FC801D5
:100BB0000E9441175601F6018081882301F16501E9
:100BC000F60181912F01882311F08E32B1F4460194
:100BD0008A189B081814190474F48D8641E050E0BB
:100BE000BE01635F7F4FC8010E944117A401B50198
:100BF000C8010E9441175201DECF6201E1CF1D867C
:100C000041E050E0BE01635F7F4FC8010E94411781
:100C1000C12CDD24D394DA82C98242E050E0BE01C7
:100C20006F5F7F4FC8010E944117DA82C98242E09C
:100C300050E0BE016F5F7F4FC8010E944117C8019D
:100C40000E947B17892B09F441CFF3E0AF2EB12C22
:100C5000230122E0420E511CD4C0F701428153818E
:100C600064817581808D918DA28DB38D4817590750
:100C70006A077B0709F008C1848D958DC59709F037
:100C800003C181A192A15DEFC52EDD24DA940C97FA
:100C90000CF4ADC04CE050E0BE016F5F7F4FC80167
:100CA0000E942E138B819C819827892798279A8BE5
:100CB000898BF7014681578129813A814217530771
:100CC00009F0E7C097FFE5C08F7092703BEFC32E2D
:100CD000DD24DA94892B09F08AC06F807884762429
:100CE000672476242AEFC22EDD24DA94611471047D
:100CF00009F47DC0D12CC12C8D819E819827892734
:100D00009827C816D906F8F441E050E0BE01635FA9
:100D10007F4FC8010E942E134D85442331F050E0CF
:100D200070E060E0C8010E942E138D858111ECCF28
:100D300044E050E070E060E0C8010E942E13FFEF35
:100D4000CF1ADF0AD9CF912C812C41E050E0BE01AF
:100D50006D5E7F4FC8010E942E134B89842F807CCB
:100D600009F06CC0442331F050E070E060E0C8014D
:100D70000E942E138B898111E8CF42E050E0BE0122
:100D8000615F7F4FC8010E942E1342E050E0BE0118
:100D9000635F7F4FC8010E942E1344E050E070E073
:100DA00060E0C8010E942E1342E050E0BE016F5E79
:100DB0007F4FC8010E942E138F85988949895A89CF
:100DC0008115914009F043C0CD84DE84DC24CD241C
:100DD000DC2481E0C816D104D1F54115544009F056
:100DE0004AC044E050E0B201C8010E942E1321E045
:100DF000A21AB10809F46CCEFFEFCF16DF0609F096
:100E000067CE0E9425843B014C01C8010E947713E4
:100E1000181619060CF421CF0E942584661977094B
:100E200088099909693873418105910548F562E39C
:100E300070E080E090E00E945681E7CF41E050E012
:100E400070E060E0C8010E942E131B8A93CF5427E4
:100E50004527542770E060E0C8010E942E13FFEF81
:100E60008F1A9F0A6814790409F06FCF96EFC92E84
:100E7000DD24DA94BCCFE7EFCE2EDD24DA94B7CFB1
:100E8000CC24CA94DC2CB3CF6EEFC62EDD24DA94CA
:100E9000AECF4CEFC42EDD24DA94A9CF8EEFC82E4E
:100EA000DD24DA9430CED12CC12C2DCE1F920F929E
:100EB0000FB60F9211242F933F938F939F93AF936D
:100EC000BF938091171390911813A0911913B091AB
:100ED0001A133091161323E0230F2D3758F501967E
:100EE000A11DB11D2093161380931713909318130F
:100EF000A0931913B0931A1380911B1390911C1394
:100F0000A0911D13B0911E130196A11DB11D8093D8
:100F10001B1390931C13A0931D13B0931E13BF912A
:100F2000AF919F918F913F912F910F900FBE0F9096
:100F30001F90189526E8230F0296A11DB11DD2CF50
:100F40001F920F920FB60F9211240BB60F922F9390
:100F50003F934F935F936F937F938F939F93AF9341
:100F6000BF93EF93FF9348E251E064E271E090E0B9
:100F700080E00E941180FF91EF91BF91AF919F910E
:100F80008F917F916F915F914F913F912F910F9032
:100F90000BBE0F900FBE0F901F9018951F920F92CF
:100FA0000FB60F9211240BB60F922F933F934F93CE
:100FB0005F936F937F938F939F93AF93BF93EF93C1
:100FC000FF9348EA50E064EA70E083E090E00E941A
:100FD0001180FF91EF91BF91AF919F918F917F9180
:100FE0006F915F914F913F912F910F900BBE0F909A
:100FF0000FBE0F901F9018951F920F920FB60F9271
:1010000011240BB60F922F933F934F935F936F93DF
:101010007F938F939F93AF93BF93EF93FF9348E991
:1010200050E064E970E082E090E00E941180FF915E
:10103000EF91BF91AF919F918F917F916F915F9150
:101040004F913F912F910F900BBE0F900FBE0F90BD
:101050001F9018951F920F920FB60F9211240BB686
:101060000F922F933F934F935F936F937F938F9341
:101070009F93AF93BF93EF93FF9348E850E064E8EA
:1010800070E081E090E00E941180FF91EF91BF91AC
:10109000AF919F918F917F916F915F914F913F9110
:1010A0002F910F900BBE0F900FBE0F901F901895B1
:1010B00060930E1370930F1380931013909311137A
:1010C000645D7E4F8F4F9F4F60930A1370930B1395
:1010D00080930C1390930D1382E090E0909309138A
:1010E000809308130E942584609304137093051362
:1010F00080930613909307130895CF92DF92EF9297
:10110000FF920F931F930E9425848B019C01C09036
:101110000413D0900513E0900613F090071360912C
:101120000E1370910F1380911013909111130C19DD
:101130001D092E093F09083E134021053105E0F045
:10114000DC01CB010196A11DB11D80930E1390937C
:101150000F13A0931013B0931113B701A6014851B8
:101160005C4F6F4F7F4F4093041350930513609370
:10117000061370930713C7CF1F910F91FF90EF9045
:10118000DF90CF900895CF93DF93EC010E947D888C
:101190009E01220F331F220F331FF901E152FD4F31
:1011A0006083718382839383CE01880F991FFC0132
:1011B000E952FD4F408151811416150644F4FC019B
:1011C000E153FD4F408151811416150614F1FC01C5
:1011D000E952FD4F41E050E05183408381539D4FE0
:1011E000FC015183408321543D4F88E097E0A0E00B
:1011F000B0E0F90180839183A283B383CE010E9482
:101200000F1A64EF71E080E090E0DF91CF910C94D1
:101210005681DF91CF9108954F925F926F927F92A6
:101220008F929F92AF92BF92CF92DF92EF92FF92F6
:101230000F931F93CF93DF934B015C0180910013B9
:1012400090910113A0910213B09103138815990591
:10125000AA05BB0509F4C6C08CE3C82ED12CE12C2D
:10126000F12CC501A70196010E94CCB06093D20B6E
:10127000CA01B901A70196010E94CCB06093D30BBB
:10128000C501B40120E13EE040E050E00E94CCB056
:10129000CA01B90128E130E040E050E00E94CCB042
:1012A0006093D40BC501B40120E831E541E050E082
:1012B0000E94CCB069017A01CA01B9016C5F7F4F0D
:1012C0008F4F9F4F27E030E040E050E00E94CCB0CD
:1012D0006F5F6093D50B412C512C320140E004E646
:1012E00010E0C0E9D1E0242F30E02E54384FF9014E
:1012F000E370FF273097F9F4C901B8010E945AB290
:10130000892B31F4C901BE010E945AB2892B99F48C
:101310008EE691E0A0E0B0E0480E591E6A1E7B1EEA
:10132000D301C201AA27BB27C816D906EA06FB06C5
:1013300038F04F5FD8CF8DE691E0A0E0B0E0ECCF81
:101340004093D80BC90164E670E00E945AB2EC01E8
:10135000C90160E971E00E945AB2309721F42097E8
:10136000D9F40097C9F04DE651E060E070E0441A0E
:10137000550A660A770AC418D508E608F708A5E3EF
:10138000B3E020E0213069F43097E9F5209711F4BB
:101390000097C9F54DE106C04EE651E060E070E00F
:1013A000E6CF4C9150E070E060E031E0320FC416BF
:1013B000D506E606F70640F0C41AD50AE60AF70A8B
:1013C0001196232F3C30F1F62F5F2093D70BC39457
:1013D000C092D60B8092001390920113A092021338
:1013E000B0920313DF91CF911F910F91FF90EF9077
:1013F000DF90CF90BF90AF909F908F907F906F9035
:101400005F904F9008954CE1CDCF0E947D880E945F
:101410000C898091D80B90E08E54984F08950E94CB
:101420007D880E940C898091D70B90E008950E94DE
:101430007D880E940C898091D60B90E008950E94CF
:101440007D880E940C898091D30B90E008950E94C2
:101450007D880E940C898091D40B90E008951F92A2
:101460000F920FB60F9211240BB60F922F933F934A
:101470004F935F936F937F938F939F93AF93BF939C
:10148000EF93FF93809130120E94AB75209133123D
:10149000309134122F5F3F4F309334122093331228
:1014A00090913212953618F096E090932F12909109
:1014B0002F12943009F46EC0F8F4923031F1933069
:1014C00009F44CC090913112992319F0811171C027
:1014D0002F9AFF91EF91BF91AF919F918F917F9143
:1014E0006F915F914F913F912F910F900BBE0F9095
:1014F0000FBE0F901F901895953009F457C0963085
:1015000009F791E09093FF124FC08111DBCF20913A
:101510003312309134122436310528F410923412EB
:1015200010923312CFCF1092FF1210923212E0912C
:10153000321291E09E0F90933212F0E0209133121C
:1015400030913412EE0FFF1FEB5CFD4E3183208390
:10155000109234121092331293E019C0813009F0C6
:10156000B1CFE091321291E09E0F90933212F0E0F1
:101570002091331230913412EE0FFF1FEB5CFD4EC1
:1015800031832083109234121092331294E090939E
:101590002F1298CF882359F22091331230913412B0
:1015A0002536310508F48ECF95E0F1CF81118ACF31
:1015B000B5CF2F988ECFCF93DF9391E09093EB111F
:1015C0008823B9F0C091B800D091BA008091BC00D6
:1015D0008A7B8093BC0060E084E10E94E37F60E04E
:1015E00085E10E94E37F0E94CB80D093BA00C09334
:1015F000B800DF91CF9108958F929F92AF92BF92E2
:10160000CF92DF92EF92FF920F931F93CF93DF93CE
:10161000D091860CD13208F0D7C0182FC091850C1C
:101620000E9431816B017C0180917D0C81116BC026
:1016300082E080937D0C10937C0C8FEF80937B0C69
:1016400010927A0CD093790CA5E9B5E1E9E5FCE0BC
:1016500080E0D81391C01092580C8091580CCC0F98
:10166000C82BC093580C8091570C813009F088C06A
:101670001092570C0E9431816B017C018091580CB3
:101680008093BB0080917F0C9091800CA091810C85
:10169000B091820C892B8A2B8B2BA1F00E94318177
:1016A00000917F0C1091800C2091810C3091820C64
:1016B0006C197D098E099F09061717072807390736
:1016C00008F442C08091BC0083FDD8CF85EC8093A4
:1016D000BC000E9431816B017C0180917D0C8230C5
:1016E00009F450C080917B0C8F3F09F46FC080914A
:1016F0007B0C803209F46CC080917B0C803309F440
:1017000069C084E026C080917F0C9091800CA091EC
:10171000810CB091820C892B8A2B8B2B09F484CFFE
:101720000E94318180907F0C9090800CA090810C61
:10173000B090820C6C197D098E099F098616970658
:10174000A806B90608F070CF80917E0C0E94DB8A53
:1017500085E01092840C1092860C1092830CDF911D
:10176000CF911F910F91FF90EF90DF90CF90BF909E
:10177000AF909F908F9008959D9191938F5F69CFC7
:1017800085EEA5CF80917F0C9091800CA091810C6B
:10179000B091820C892B8A2B8B2B09F49ECF0E944F
:1017A000318100917F0C1091800C2091810C30913F
:1017B000820C6C197D098E099F09061717072807E7
:1017C000390708F08ACFC0CF81E0C3CF80E0C1CF16
:1017D00082E0BFCF83E0BDCFFC01248131E03093B4
:1017E000830C2093850C1092840C1092860C8385B8
:1017F000682B82EC9DE00E94517681E00C94FC8A7B
:101800000F931F93CF938C01C62F0E94EC8B6C2FEC
:101810006460C8010E94EC8B6C2F6B7FC8010E9432
:10182000EC8B83EC90E00197F1F7CF911F910F9132
:1018300008950F931F93CF938C01C62F607F616033
:101840000E94008C80E1C89FB00111246160C80132
:101850000E94008C81E090E0CF911F910F9108953C
:10186000CF93C82F682F607F84ED91E10E94008C98
:1018700080E1C89FB001112484ED91E1CF910C94D7
:10188000008CCF93DF9300D000D01F921F92CDB772
:10189000DEB798E0EBE2F3E0DE01119601900D92E5
:1018A0009A95E1F79091DD11961708F46FEF70E0CB
:1018B000660F771F21E030E02C0F3D1F620F731F72
:1018C000FB019081890F806828960FB6F894DEBFDF
:1018D0000FBECDBFDF91CF910C94308C85ED8093FE
:1018E000BC0080917F0C9091800CA091810CB091F4
:1018F000820C0796A11DB11D23E0B695A79597957B
:1019000087952A95D1F72091BC0024FD03C0109241
:101910007D0C089540917F0C5091800C6091810C5A
:101920007091820C452B462B472B69F30097A1053C
:10193000B10541F025E32A95F1F700000197A109CF
:10194000B109E1CF80917E0C0C94DB8A1F920F923B
:101950000FB60F9211240BB60F922F933F934F9314
:101960005F936F937F938F939F93AF93BF93EF9307
:10197000FF938091B900887F803609F44DC008F04C
:1019800040C0883209F4A9C028F5803109F49DC00F
:10199000C8F4882309F4FBC0883009F496C0FF918D
:1019A000EF91BF91AF919F918F917F916F915F91D7
:1019B0004F913F912F910F900BBE0F900FBE0F9044
:1019C0001F901895883109F488C0803241F78093C0
:1019D0007B0C14C0803409F49DC040F48033B9F30B
:1019E0008833E9F680937B0C85ECB0C0803509F430
:1019F00085C0883509F496C0883489F60E946E8CBB
:101A0000CECF883909F48CC038F5883729F050F4E6
:101A1000883611F0803719F683E080937D0C1092A0
:101A20002E1257C0883809F47BC0803919F08038ED
:101A300009F0B5CF80912E12803208F071C0E0918C
:101A40002E1281E08E0F80932E128091BB00F0E069
:101A5000E25FFD4E80833DC0803B39F0E0F4803A88
:101A600009F479C0883A09F09ACF84E080937D0C1C
:101A700010920D1210920C12E0912713F09128137E
:101A8000199580910C1281110FC081E080930C1286
:101A90001092EC1109C0803C09F4A6CF883C09F4EF
:101AA000A3CF883B09F07BCFE0910D1281E08E0F30
:101AB00080930D12F0E0E451FE4E80818093BB00D4
:101AC00090910D1280910C1229C08091580C809336
:101AD000BB0085EC8093BC0062CF90917A0C809122
:101AE000790C981758F5E0917A0C81E08E0F80936D
:101AF0007A0CF0E0E75AF34F8081E9CFE0917A0C5D
:101B000081E08E0F80937A0C8091BB00F0E0E75A61
:101B1000F34F808390917A0C8091790C9817C8F2DA
:101B200085E8D8CFE0917A0C81E08E0F80937A0C13
:101B30008091BB00F0E0E75AF34F808380917C0CEA
:101B400081115CCF81E08093570C84EA8093BC00C4
:101B500010927D0C24CF85EC8093BC0010927D0CFC
:101B600080912E12803230F4E0912E12F0E0E25F8C
:101B7000FD4E108260912E1270E0E0912513F091DD
:101B800026138EE092E1199510922E1208CF109232
:101B90007B0C34CF4F925F926F927F928F929F9285
:101BA000AF92BF92CF92DF92EF92FF920F931F936B
:101BB000CF93DF93EC01423051056105710590F43C
:101BC00080E0DF91CF911F910F91FF90EF90DF9018
:101BD000CF90BF90AF909F908F907F906F905F90CD
:101BE0004F90089589859A85AB85BC850196A11D86
:101BF000B11D84179507A607B70710F3CB88DC88BB
